:020000040000FA
:040000006FD00400B9
:101000006F00907C00000000000000009020002095
:10101000AA220020A9BDF9F56C23002000000000E1
:10102000000000006C230020902000200000000041
:101030000000000090200020000000009020002010
:101040000000000090200020902000209020002030
:101050009020002090200020382F002074240020B1
:101060000000000090200020902000200C24002090
:1010700090200020D22300209020002090200020EB
:101080009020002090200020902000209020002020
:101090009020002001A04111B7170040985F3AC688
:1010A000945F3247E39CE6FE3245410182800111A4
:1010B00013078008F337078093F787083EC20100C3
:1010C0000100B7170040930570052380B70413068D
:1010D00080FA2380C7040100010083C6B70493F699
:1010E000F60DA385D704238007049246F3A6068055
:1010F0000100010093760502D5CEF336078093F602
:10110000860836C4010001002380B7042380C70489
:1011100001000100B70614007D89558D88C70100C4
:1011200001000100010023800704A246F3A6068007
:101130000100010073370780137787083AC6010062
:1011400001002380B7042380C704010001000100CF
:1011500001003727004093061005A303D7802380A2
:101160000704B247F3A70780010001009307800836
:10117000F3B7078093F787083ECE01000100B71749
:101180000040130770052380E704130780FA2380CB
:10119000E7040100010003C7B70413670708A3852C
:1011A000E70423800704F247F3A70780010001004A
:1011B0000561828093760504BDC6F336078093F6F9
:1011C000860836C8010001002380B7042380C704C5
:1011D00001000100B7061400938606047D89558D31
:1011E00088C7010001000100010023800704C246F6
:1011F000F3A6068001000100733707801377870884
:101200003ACA010001002380B7042380C70401000B
:1012100001003727004093062005A303D7802380D1
:101220000704D24781B773370780137787083ACC12
:10123000010001002380B7042380C70401000100DE
:1012400098471367070C98C723800704E24719BF24
:101250000111814601468145114506CE97000000E7
:10126000E780605693078008F3B7078093F78708F5
:101270003EC601000100B717004013077005238028
:10128000E704130780FA2380E7040100010003C785
:101290006704136717002383E70423800704B2471A
:1012A000F3A7078001000100F2400561828041112F
:1012B000814601468145114597000000E780A05016
:1012C00013078008F337078093F787083EC40100AF
:1012D0000100B7170040130670052380C70493066A
:1012E00080FA2380D70401000100FD552396B70240
:1012F00023800704A245F3A5058001000100733790
:101300000780137787083AC6010001002380C704CD
:101310002380D7040100010003C767041367170087
:101320002383E70423800704B247F3A70780010063
:10133000010001A0BD473305F50201007D1575FDD3
:101340008280411122C426C206C6AA8401446317C2
:101350009400B24022449244410182800504130566
:10136000803E420497000000E78000FD4180C5B741
:101370009305000273A04580824573901534924016
:101380002242B2424243D2436244F2440255925551
:101390002256B2564257D2576258F25806499649D9
:1013A000264AB64A464BD64B664CF64C065D965DD1
:1013B000265EB65E465FD65F09617300203041113C
:1013C000B7170040985F3AC6945F3247E39CE6FE49
:1013D000324541018280B71700401307000323887C
:1013E000E702854717170000232AF77073002030A3
:1013F000411122C406C637040020976000E0E78050
:10140000605A974000E0E780A0781C408297F5B7CB
:10141000B737004003C7470091463D8B6309D700AB
:1014200099466314D70083C757407300203017379D
:101430000000034767519306E00763ECE60293065A
:101440001700173600002301D65083C68700973750
:10145000000093876747BA972380D700B7E7040057
:10146000BC4F09468945171500000345E5F48297EE
:101470006DBF83C78700DDB7B787004003C767002C
:10148000098B6309071003C77700930600031377DE
:101490000703630DD708174800000348389A17461A
:1014A00000001306E6980547B30606012380E60010
:1014B00083C577001747000013070798429793F5F5
:1014C000F50F2300B70003C58700974500009385FB
:1014D0006596C2951375F50F2380A5000347070095
:1014E00089451377F703630CB70C63E7E50A6306D6
:1014F000071A8545630CB7129747000083C71794F6
:101500003307F600034707001377F70F19CB85075A
:1015100093F7F70F0D476363F71A17470000A30F00
:10152000F790B787004009472383E700B78700405B
:1015300083C77700E207E18763DE0704974700006F
:1015400083C7D78F174700001307878E3E978546BE
:101550002300D700174700001307078E3E97930616
:1015600000032300D700174700001307A78C3E97FE
:10157000A14685072300D70093F7F70F0D47636453
:10158000F71417470000A30BF78AB78700400947F5
:101590002383E70073002030930610026300D70E08
:1015A000930620026305D70693060002E316D7F4DC
:1015B00003C727021377C70F13672700D5A803C7F0
:1015C00067001377070465CB03C7A702173800002D
:1015D0001308886F173500001305C5661347070801
:1015E0002385E70203C7A7021377370F1367870026
:1015F0002385E702814713070004B305F5008C41FA
:10160000B306F80091078CC2E399E7FEF5B503C76E
:10161000A702134707042385E70203C7A70213772E
:10162000C70F136727002385E702F9B503C76700D3
:101630001377070449C303C767021738000013086C
:10164000685C173500001305A5531347070823836B
:10165000E70203C767021377370F136787002383F7
:10166000E702814713070004B305F5008C41B30678
:10167000F80091078CC2E399E7FEBDBD03C767027E
:10168000134707042383E70203C767021377C70FD3
:10169000136727002383E70285B503C76700137725
:1016A000070411CB03C727021377370F136787008F
:1016B0002381E70291B5238006003DBD97370000E6
:1016C000A38E0776B9BD97370000A389077675BD4D
:1016D0002303048015472303E48001002302A48030
:1016E000828083076480E3CE07FE23030480828028
:1016F00083076480E3CE07FE03454480828083072E
:101700006480E3CE07FE2302A4808280411126C4B8
:101710004AC24EC006C61377F50BAD47AA892E897B
:101720009544630CF700194597000000E78080FAA4
:1017300097000000E78020FB8D444E859700000055
:10174000E78040F9FD59FD1463983401B240A2448A
:101750001249824941018280135509011375F50F21
:1017600097000000E780E0F92209F1BF011126CCC3
:1017700006CEB704080097000000E780C0F61545C4
:1017800097000000E78000F597000000E78080F6F2
:1017900097000000E78000F62AC697000000E78067
:1017A00080F432459377150089EB136515001375A6
:1017B000F50FF240E24405618280FD14E9F0014535
:1017C000CDBF397126DC4ADA4ED852D656D45AD219
:1017D0005ED006DE62CE66CCB7E700E07D5783AA16
:1017E000070022C603AA470023A0E71823A2E71890
:1017F000B7170040130770052380E704130780FA2A
:101800002380E70483C74704930B75FFB684E20780
:1018100093FBFB0F8546AA892E8B32893724004023
:10182000E187015763FA76016308D50089461307FB
:1018300000026313D5000157D98F93F7F70FB71C38
:1018400000402382FC0411472303E4801305F00FBA
:1018500097000000E78000E8094C97000000E7804F
:1018600080E863657C15B7050700DA9537870700C0
:10187000795563FEE504B3879500636AF704370B77
:101880000800A94733EB65016395F90881E88144B5
:1018900097000000E78020E5268515A8DA85094530
:1018A00097000000E780C0E605090345F9FFFD1435
:1018B000050B97000000E780C0E481C49377FB0F1D
:1018C000E5F797000000E780A0EA69F17D55B717BA
:1018D0000040130770052380E704130780FA238074
:1018E000E70403C74704418B2382E704F250B7E7BC
:1018F00000E023A0571123A24711E2543244525969
:10190000C259325AA25A125B825B724CE24C21617C
:101910008280A547639BF90685691309F00FB3061A
:101920009900B3742B01B6941349F9FFB37499006D
:10193000856B33796901416B9387F9FFB3F7270111
:1019400099E363FC340193D94900C147E3E637FFCB
:101950003DBF0569C1697D19D9B71305800D63883D
:101960006901130500026384790113051008CA8513
:1019700097000000E780C0D997000000E78040DFB3
:1019800031D54E99B38434416DBFDA852D4597002A
:101990000000E780E0D7CA94E30B99EE05099700B1
:1019A0000000E78020D5A30FA9FEFDB79387F9FFBC
:1019B00093F7F70F636DFC0C83C71C041307300803
:1019C0006315F706370708006361EB06B3079B0052
:1019D000B706100063FBD704334BEB0089476399CC
:1019E000F9068980D549E38404EADA850945970038
:1019F0000000E780E0D111090327C9FF91472320A8
:101A0000E48003076480E34E07FE23033481FD175F
:101A1000EDFBFD14110B81C49377FB0FE9FF9700D9
:101A20000000E780E0D461F155B5B717004003C767
:101A30005704B70708001377070219E3B7870700B1
:101A40007955E376FBE833079B00E3F9E7F841B506
:101A50008547E380F9F0DA852D4597000000E7809F
:101A600020CB9389F4FFE38404E297000000E78031
:101A700060C893F7390091EB83260480032709009F
:101A800093074900E396E6E03E89CE84D9BFB54787
:101A90006399F9001305900B97000000E78080C35D
:101AA000FDB3B1471305B00AE388F9FE9947639780
:101AB000F904B7050800B365BB002D459700000089
:101AC000E78000C581448D4BA14997000000E78065
:101AD00060C263967401832704802320F900850483
:101AE000E39534FF8327048013172B016355070008
:101AF0002312F90069BB2322F90051BB9D47639F64
:101B0000F90281451305B00497000000E78040C04A
:101B1000BD442320090023220900FD59970000003D
:101B2000E78040BD93F77400CA9703C70700FD1410
:101B3000398D2380A700E39334FF91BBA1476397BE
:101B4000F90697000000E780A0C28144630D0B00F6
:101B50008D479304C0036308FB00930400056304EE
:101B60008B01930440041375C507E30295D2194510
:101B700097000000E78000B697000000E780A0B65D
:101B8000054597000000E780E0B426859700000037
:101B9000E78020B7094597000000E78080B69700EE
:101BA0000000E780E0BCE31405CE0DB39147639FCE
:101BB000F9001305600697000000E780A0B19700C8
:101BC0000000E78040B213059009F9B5E38109CC24
:101BD000F1547DB9BD660147173600001306464330
:101BE000938606A685458347060093F7F70F91C3B2
:101BF00082800507E3F9E6FE97370000238AB740A5
:101C0000DDB77D166206618693178601E18763D48E
:101C1000070001458280931726003307F500AE9731
:101C200018439C4363E7E7007D16E37FF7FC7D558F
:101C3000828005458280FD15E205E18513978501C7
:101C4000618793F7F50F63480700FD15139725008B
:101C50002A97584365D713851700620561858280EE
:101C60003308B5021C4283A80600B335B502C297FB
:101C700033B50701AE98469585486367B500639410
:101C8000A50063E3070181480C43C6950CC388C2D5
:101C90001CC2828081471397870161876343B70025
:101CA0008280139727002A97232007008507E5B72E
:101CB0008147014793968701E18663C5B6001335D6
:101CC0001700828093962700AA9694428507558F25
:101CD000D5B793D755408A07AA979C430545331536
:101CE000B5007D8D828017F3FFDFE702833D2A84F4
:101CF00097000000E78060F405C5931725003E9427
:101D00000327C4FF814711EB7D1516053E9542055B
:101D1000418517F3FFDF6700033D05838507E5B7BE
:101D20000145C5BF81471397870161876343C7009A
:101D3000828013972700B386E50094422A9785078F
:101D400014C3D5B77D1662066186014793178601D5
:101D5000E18763D5070013351700828093172600AB
:101D6000B306F500AE9794429C437D16B58F5D8F08
:101D7000F1BF8A05AA9501476363B500828083A6F7
:101D8000C5FFF11593D71600D98F9CC11397F601A3
:101D9000E5B72A830148014701456343D7008280A4
:101DA000B387050183A80700B30706019C43C697C4
:101DB000AA976384F80033B517010507B308030138
:101DC000620723A0F80061871108C1BF2A83014779
:101DD0008147014563C3D70082803388E5008328AB
:101DE0000800330EE600032E0E003388A8403308A7
:101DF000C8416384080133B508018507B308E300CF
:101E0000E20723A00801E1871107E9B717F3FFDF15
:101E1000E702232B0111B286B2842E86AA850A8599
:101E200097000000E780C0FA2A84A6850A859700FB
:101E30000000E78020E833348000060413351500E5
:101E4000018D056117F3FFDF6700E32917F3FFDF5B
:101E5000E702A3244111AA89AE8A328BB68402C25A
:101E600002C402C60144131C8401135C8C41634903
:101E70009C02939B1400FD1B0549138CF4FFF15C3D
:101E800033048901620461846340740792478E04BD
:101E9000CE9423AEF4FE410117F3FFDF6700632306
:101EA00013192400B30B2B01014A93172A00D6976C
:101EB00083A50B0088437800340050009700000091
:101EC000E78040DA050A93178A01E187F11BE35E98
:101ED000FCFC92474E9905042320F900A2473EC21C
:101EE000B24702C63EC441B7131A8901135A8A4148
:101EF000131D240093178A01E18763CF970092474F
:101F00000A044E941CC0A24705091379F90F3EC27A
:101F1000B24702C63EC4ADB7B3079A0313152A00F1
:101F200056950841780034005000050AEA97DA9780
:101F30008C4397000000E780E0D26DBF197106C2A4
:101F400012C416C61AC81ECA22CC26CE2AD02ED239
:101F500032D436D63AD83EDA42DC46DECAC0CEC2E9
:101F6000D2C4D6C6DAC8DECAE2CCE6CEEAD0EED219
:101F7000F2D4F6D6FAD8FEDA97150000938585B725
:101F80008841E700050092402242B2424243D243D8
:101F90006244F244025592552256B2564257D257E5
:101FA0006258F25806499649264AB64A464BD64BDD
:101FB000664CF64C065D965D265EB65E465FD65F65
:101FC0000961730020300000972100209381810374
:101FD000175100201301018317F5FFFF1305C502F8
:101FE0009705002093850502171600201306C6FDED
:101FF00063FAC5008322050023A055001105910551
:10200000E3EAC5FE17150200130545B29715002037
:102010009385C5FB171600201306467C63FAC5009E
:102020008322050023A0550011059105E3EAC5FEB2
:10203000171500201305857A9745002093850549DB
:102040006377B500232005001105E36DB5FEFD4261
:10205000739002BC8D4273904280B722000093823D
:10206000828873900230970200209382A2F993E253
:10207000320073905230974200009382226E739028
:1020800012346FB0F47773002030397101436EC69B
:1020900019A0397141536AC866CA62CC5ECE19A0D4
:1020A000397101535AD056D252D44ED64AD826DA74
:1020B00022DC06DE33016140828241114AC026C221
:1020C00022C406C68282B24D4101024D924C224C7E
:1020D000B24B4101024B924A224AB24941010249A4
:1020E00092442244B240410182803D432A87637377
:1020F000C3029377F700BDEFADE5937606FF3D8A07
:10210000BA960CC34CC30CC74CC74107E36BD7FE50
:1021100011E28280B306C3408A06970200009696B9
:102120006780A6002307B700A306B7002306B70001
:10213000A305B7002305B700A304B7002304B70025
:10214000A303B7002303B700A302B7002302B7001D
:10215000A301B7002301B700A300B7002300B70015
:10216000828093F5F50F93968500D58D93960501A2
:10217000D58D61B7939627009702000096968682C8
:10218000E78086FA9680C1171D8F3E96E374C3F8E8
:10219000A5B73367B500FD530D8B79E7B7877F7F10
:1021A0009387F7F710419441B372F6003363F6005A
:1021B000BE92B3E262006397720C6318D606504178
:1021C000D441B372F6003363F600BE92B3E262000C
:1021D0006398720A631BD60410459445B372F600E7
:1021E0003363F600BE92B3E262006391720A631E2B
:1021F000D6025045D445B372F6003363F600BE9262
:10220000B3E26200639A72086311D60210499449DE
:10221000B372F6003363F600BE92B3E262006393DA
:1022200072085105D105E30FD6F6131706019397EF
:102230000601631CF7001357060193D70601330507
:10224000F7409375F50F91E982804183C18333058F
:10225000F7409375F50F91E182801377F70F93F7AD
:10226000F70F3305F74082800346050083C605005B
:10227000050585056313D60065FA3305D6408280CF
:1022800011059105E312D6FE014582802105A105C5
:10229000E31CD6FC014582803105B105E316D6FC6E
:1022A000014582804105C105E310D6FC01458280CD
:1022B000B717004003C777051377E70FA38BE70431
:1022C000130700F8A38DE7043D47238CE7041307A9
:1022D0005003A38CE70403C7A7051377D70F238DFB
:1022E000E7048280B717004003C7E7020D89411158
:1022F0001377C70F498F93068008F3B6068093F6CD
:10230000860836C601000100930670052380D704B5
:10231000930680FA2380D704010001002387E70297
:1023200023800704B247F3A70780010001004101A1
:10233000828041112A83014E930E407E130F0019B3
:10234000930F400663E56E129308001913034006CD
:10235000B3781503854E0D4FA14F337365020D8978
:102360001335150063EFBE121308F6FF7946729815
:102370004208135808013307C70213D61700BE07D7
:1023800032976146B3F6C60213068070B386C60262
:102390003697A166F58F42075D8FB716004083C759
:1023A000F60293F70708A303F1000346710083C701
:1023B000F60293F70708E394C7FE83477100B71648
:1023C000004093F7F70F6388071293078008F3B76D
:1023D000078093F787083EC401000100B71700404B
:1023E000930670052380D704930680FA2380D704D0
:1023F0000100010023AA070383C6170393E606081A
:10240000A388D70223800704A247F3A7078001000F
:1024100001001166B71700407D16D45BC85F938535
:102420004703A98EF18EF5FA93068008F3B606806D
:1024300093F6860836C601000100930670052380D6
:10244000D704930680FA2380D7040100010098C1C5
:1024500003C7170313670704A388E7022380070451
:10246000B247F3A7078001000100410182807D137C
:102470003368E3039308E016630E08003368F30340
:102480009308D016630808009378330093B81800B7
:102490009388D81633081E01131E0801135E0E011F
:1024A00055B56393E5030548638608000148630357
:1024B00003002A8871087298FD15131E0801C205D1
:1024C000135E0E01C18179BD13F8150063F4BF00DE
:1024D0007908D5B713381800E5BF83C7F60293F71C
:1024E0000708A303F1000346710083C7F60293F7C0
:1024F0000708E394C7FE8347710093F7F70FF1DFF6
:10250000E9B531714AD966CB06DF22DD26DB4ED72D
:1025100052D556D35AD15ECF62CD6AC96EC7AA8C46
:1025200002D897100000E780009F2A89930780084F
:10253000F3B7078093F787083EDA01000100B71769
:102540000040130770052380E704130780FA2380F7
:10255000E7040100010003C7F7021377770FA38791
:10256000E70203C7F70213678700A387E702238008
:102570000704D257F3A70780010001000545970023
:102580000000E78060D6130780C13347E902116A73
:1025900093070AE893065002BD69930BA004814A91
:1025A000014B13048008930470057D1AB347F902A8
:1025B0003307D7023EC0FD873ECC938709A6930917
:1025C000803E3347F7023AC27D873AC43347390326
:1025D0008549B399990193D93940B306D702B30B12
:1025E0007703B3C6F602B3CBFB0236C6FD8636C808
:1025F00093D6FB4136CEB7460F0093860624334967
:10260000D9028566938606FAB3969601B389E902E4
:10261000130760553309D90293060010B389E90204
:102620003349D902B3C9F9029316390036CA3719AA
:102630000040FD8636D0930D090493D7F9413ED270
:10264000F336048093F6860836DC01000100930718
:1026500070052380FD00930680FA2380DD000100D1
:1026600001008346390593F6860FA309D9048346F2
:10267000390593E61600A309D90423800D00E2561C
:10268000F3A6068001000100130C80FA116DF336E9
:10269000048093F6860836DE01000100930770057A
:1026A0002380FD0023808D01010001008346390550
:1026B000216693E60602A309D90483560905B3E609
:1026C000A6012318D90483560905D18E2318D904ED
:1026D00023800D00F256F3A6068001000100834618
:1026E000390593F606026381061A03463905218AE5
:1026F0006DDE081897100000E780E08573360480CF
:1027000013768608B2C20100010023809D00238059
:102710008D0101000100B717004003C6370513768D
:10272000F60DA389C70403C6370513660602A389FD
:10273000C704835609052166B3E6A6012318D90408
:1027400083560905D18E2318D90423800D0096469F
:10275000F3A60680010001008346390593F60602C0
:10276000638B061483463905A18AEDFE970000208D
:10277000E7806092AA8636D497000020E780A09177
:10278000A256E30AD5FE835609054255B3E6A601D3
:102790002318D90497000000E780A07D83463905FF
:1027A000A18AEDDE03560905834629058247337663
:1027B000CA00B306DA0293D5F641B296B388F64062
:1027C000E24733B8C6002E983308F840A247B3B6A4
:1027D00016013308D84063C70701631DF80092470C
:1027E00063FA1701C247634FF80E63950701B247BA
:1027F00063EAF80E894663E9660FF24693151800FE
:1028000013D3F8015E8613951800B365B30042D662
:1028100046D497C00100E78080F03258050B137B47
:10282000FB0F63470001631A0838A2586387083812
:1028300013081500B336A800B69513D6F5013298E3
:10284000B336C800AE9613581800FE06B3E606016C
:102850007336048013768608B2C601000100238017
:102860009D0023808D01010001000356C902B2962C
:10287000C206C1822316D90223800D00B646F3A6F4
:1028800006800100010021B5F336048093F6860826
:10289000B6C00100010023809D0023808D0101004E
:1028A00001008346390593E60602A309D904238073
:1028B0000D0086460DB5F336048093F68608B6C43F
:1028C0000100010023809D0023808D010100010093
:1028D0008346390593E60602A309D90423800D0037
:1028E000A646BDB5E30B0BF0F336048093F68608DD
:1028F000B6C801000100930680FA23809D00238062
:10290000DD00010001008346390593F5FC0F93F6C5
:10291000860FA309D90483463905CD8EA309D904AE
:1029200023800D00C646F3A60680010001001305B2
:1029300080FA03463905930639051D8A631C9629DA
:102940007336048013768608B2CC010001001306AA
:1029500080FA23809D002380CD000100010003C682
:1029600006001376F60D2380C60003C60600136624
:1029700006022380C600835609051166D18E2318EE
:10298000D904835609052166D18E2318D9042380E2
:102990000D00E646F3A6068001000100130680FA4A
:1029A0008346390593F60602638006268346390579
:1029B000130C3905A18AFDDA081897000000E7809A
:1029C0008059F336048093F68608B6D001000100E2
:1029D000930680FA23809D002380DD000100010022
:1029E00083460C00116693F6F60D2300DC00834647
:1029F0000C0093E606022300DC0083560905D18E05
:102A00002318D904835609052166D18E2318D904C9
:102A100023800D008656F3A60680010001001306F0
:102A200080FA8346390593F60602638A06208346B8
:102A30003905A18AEDFE97F0FF1FE780C0652A8C5B
:102A400097F0FF1FE7802065E30C85FF835609059B
:102A500011664255D18E2318D90497000000E780F3
:102A600040518346390513063905A18AFDDAF3364C
:102A7000048093F68608B6D401000100930680FA1C
:102A800023809D002380DD000100010083460600B5
:102A900093F6F60D2300D60023800D00A656F3A66C
:102AA0000680010001008356090503462905D24727
:102AB000B376DA003306CA021305800C9355F6414B
:102AC0003696330DF6408257333CD6002E9C333673
:102AD000A601330CFC40330CCC40330885039256DE
:102AE0004E86B335A5033305A503C29597C00100F3
:102AF000E780E0C263468001631E0C16630C0D166E
:102B0000130615003335A6002E959356F50136961B
:102B1000B335D600AA959396F50105828585D18EA9
:102B20006346B000639D051A638B061A0356C902FB
:102B300015823305D6003336C500B2956348B00020
:102B4000639105241306F00F637DA622894663F383
:102B5000561593078008F3B7078093F78708BED60A
:102B60000100010037170040930770052300F704A8
:102B7000930780FA2300F704010001008356C7027F
:102B800089678117D58FC207C1832316F7022300F7
:102B90000704B657F3A7078001000100FA506A54F2
:102BA000DA544A59BA592A5A9A5A0A5BFA4B6A4C69
:102BB000DA4C4A4DBA4D296182801308F5FF33354E
:102BC000A800FD152E951356F5013298B336C800AE
:102BD000AA9695B9F336048093F68608B6CA010022
:102BE000010023809D002380AD0001000100834689
:102BF0003905CD8EA309D90423800D00D646F3A64E
:102C000006800100010035B3F336048093F6860890
:102C1000B6CE0100010023809D002380CD0001007D
:102C200001008346390593E60602A309D9042380EF
:102C30000D00F646F3A606800100010095B3F336B9
:102C4000048093F68608B6D20100010023809D001F
:102C50002380CD00010001008346390593E606027A
:102C6000A309D90423800D009656F3A6068001001F
:102C7000010045BB9306F5FF33B5A600FD152E9563
:102C80009355F501AE96B3B5B600AA951396F50126
:102C9000858269B5F336048093F68608B6D80100BC
:102CA0000100930680FA23809D002380DD0001004F
:102CB00001008356C9020566011693F6F60FD18E00
:102CC000C206C1822316D90223800D00C656F3A680
:102CD000068001000100850A93FAFA0F95B233E6E7
:102CE000B60045C20356C9023305D0403338A000B0
:102CF000B305B040B385054115826345B000D1E10D
:102D00006371A608894663F0560593078008F3B7F8
:102D1000078093F78708BEDA01000100B71700406B
:102D2000130770052380E704130780FA2380E70464
:102D30000100010003D7C7027D8B2396E7022380A1
:102D40000704D65781BDF336048093F68608B6DCB7
:102D500001000100930680FA23809D002380DD009E
:102D6000010001008356C9020566011693F6F60FAD
:102D7000D18EC206C1822316D90223800D00E656E9
:102D8000B9B793078008F3B7078093F78708BEDECB
:102D90000100010037170040930770052300F70476
:102DA000930780FA2300F704010001000356C702CD
:102DB00093975600B297C207C1832316F7022300E8
:102DC0000704F657C1BB914763EEB70217E701004E
:102DD000130747A48A05BA959C41BA978287B7170B
:102DE000004003A7470B1345F5FF698F23AAE70AA5
:102DF00003A7070B698F23A8E70A03A7070A798DA2
:102E000023A0A70A8280B717004083A6470B134769
:102E1000F5FFF98E23AAD70A83A6070B558D23A8A1
:102E2000A70A83A6070A758F23A0E70A8280B7172F
:102E3000004003A7470B498F23AAE70A03A7070B04
:102E40001345F5FF45BFB717004083A6470B13474F
:102E5000F5FF758F23AAE70A03A7070A598D4DB717
:102E6000B717004003A7470B498FEDB7914763EEB3
:102E7000B70217E701001307279B8A05BA959C4103
:102E8000BA978287B717004003A7470D1345F5FF90
:102E9000698F23AAE70C03A7070D698F23A8E70C06
:102EA00003A7070C798D23A0A70C8280B7170040D9
:102EB00083A6470D1347F5FFF98E23AAD70C83A6E7
:102EC000070D558D23A8A70C83A6070C758F23A08B
:102ED000E70C8280B717004003A7470D498F23AA4C
:102EE000E70C03A7070D1345F5FF45BFB7170040D3
:102EF00083A6470D1347F5FF758F23AAE70C03A799
:102F0000070C598D4DB7B717004003A7470D498FE0
:102F1000EDB7B71700408847420541819377050414
:102F200091EB9377F5013755E8011305058033459B
:102F3000F50282809377050C130700046397E7007E
:102F40009377F50137459C1CCDB72165130505D056
:102F5000828037E700E01C435443A183E206D58F0B
:102F60001CC1FD572320F7182322F718828013175E
:102F70008500B7E700E023A0E710618123A2A71036
:102F80008280B7F700E08847CC4782808147373797
:102F90000040A14663C4C700328582800345B74024
:102FA000E38EA6FE3385F50003450500850723045F
:102FB000A740CDB797070020938747019C43173759
:102FC00000201307A7503E95636EE50017370020D9
:102FD000130747636368A700170700202328A7FE8D
:102FE0003E858280FD57EDBF411122C406C62A846A
:102FF00097000000E78020F22947B307E502B240BE
:103000008D83B3D7870222449507B3D7E7023737BA
:103010000040C207C1832316F70041018280716519
:1030200041111305052006C697000000E78000FC4B
:10303000B7370040130770F82381E7000D47A381DD
:10304000E70013070004A380E70005472387E70094
:10305000B2404101828037370040834727001A057C
:1030600093F7F703C98F93F7F70F2301F7008280D7
:10307000B737004003C7170019C9D98DA380B7001F
:1030800003C70700136787002380E700828093C58A
:10309000F5FFF98DA380B7008280AE872A87B73607
:1030A000004021463738004089E717430000670099
:1030B000E32183C8B600E30916FF05078348F7FF3D
:1030C000FD17C20723041801C183F9BF411122C4AF
:1030D00006C62A8497000000E780E0E32947B3078B
:1030E000E502B2408D83B3D7870222449507B3D758
:1030F000E70237370040C207C1832316F74041017A
:103100008280716541111305052006C697000000F5
:10311000E78000FCB7370040130770F82381E740D1
:103120000D47A381E74013070004A380E74005474C
:103130002387E740B24041018280CC41411106C65D
:10314000328503C6150083C5050022064D8E420652
:103150008D654186138875A2630C0611634BC80404
:10316000138845A26300060D634AC800938535A203
:103170006301B6082390060029464DA0138855A286
:103180006305060D938565A2E316B6FE8D451D46C3
:1031900063E6E5081146198E63F3C7003E86B7E77C
:1031A00004002390C600FC4797D501009385056A6B
:1031B0009DA0138895A263030611634E060D138824
:1031C000A5A263000613938505A5E315B6FA9945F4
:1031D0001D4663E5E504198E63F3C7003E86B7E735
:1031E00004002390C600FC4797050020938545E81E
:1031F0001DA09D451D4663E3E5022146198E63F33C
:10320000C7003E86B7E70400FC472390C600970539
:1032100000209385255DBA9582970146B24032859C
:1032200041018280AD451D46E3EAE5FE3146198E37
:1032300063F3C7003E86B7E704002390C600FC474F
:1032400097D5010093850563F9B7B1451D46E3E7BE
:10325000E5FC3546198E63F3C7003E86B7E70400E8
:103260002390C600FC4797D501009385A56165B7FB
:103270008D451D46E3E4E5FA1146198E63F3C70058
:103280003E86B7E704002390C600FC4797D50100AF
:103290009385855C49B78D451D46E3E1E5F8114608
:1032A000198E63F3C7003E86B7E704002390C6007B
:1032B000FC4797D501009385A55EB1BFA5451D4686
:1032C000E3EEE5F42946198E63F3C7003E86B7E7BF
:1032D00004002390C600FC4797D5010093858558CC
:1032E0001DBFB5451D46E3EBE5F23946198E63F384
:1032F000C7003E86B7E704002390C600FC4797D579
:1033000001009385A55301BFB7E7040003A307138A
:10331000970600209386C6D44146A5451705002090
:10332000130505CB02832D4559EF03C50500094759
:103330006317E50803A84500411106C603471800B6
:1033400032850346080022074168518F930828FE02
:103350006308170363E9E800051863030705239072
:10336000060029451DA8130648FE630BC702151861
:10337000E31707FF15463E87637BF602154705A84E
:103380003E8691C30546B7E70400FC472390C6007C
:103390004206CC45418282970145B240410182807C
:1033A0001306700F3E876374F6001307700FB7E7BC
:1033B00004002390E600FC4713160701D9BF2390B1
:1033C0000600054582808280416779176304E50421
:1033D000411122C406C685472A84639FF500B7E7DA
:1033E000040022852244B24003A3871397050020DE
:1033F0009385856E4101028389476399F500B7E79C
:10340000040083A7070B8545829771D9B2402244F7
:10341000410182808280797122D452CC2E842A8A02
:1034200097D501009385C54917D501001305C54BF4
:1034300006D63AC626D24AD0B68432894ECE97B046
:103440000100E7800079A68517D501001305C54A5C
:1034500097B00100E780E077294597B00100E78049
:10346000207C8347840093F70702E1E78349040047
:103470008947054532476396F908544083C71600CB
:1034800083C60600A207D58FC166138616FE638C1D
:10349000C7028D16638FD7068D66938626902945C1
:1034A0006391D706B7E70400A285225403A347140B
:1034B000B250F249A6864A86925402595285624A0F
:1034C0008547456102832D450DEF9307700F354504
:1034D00063E99702B7E70400FC4748441306700FFE
:1034E000CA8582978149970700209387A75F9C43ED
:1034F000014581CB9C4391C74E852686CA8582971C
:103500000145B250225492540259F249624A45612F
:1035100082802D457DF79307700F3545E3E397FED5
:10352000B7E70400FC4748441306700FCA8582972A
:103530005DBF2145F9B7411122C437E40400832758
:10354000841326C2AA84416506C697050020938588
:10355000A5587D1582978327C40A17050000130517
:10356000E5E68588829795C0032304132244B24080
:10357000924497060020938626C14146C54517050B
:103580000020130565AF41010283B24022449244FA
:1035900001454101828019C59707002023A4A75443
:1035A00001458280454582801147636AA70A97D604
:1035B00001009386A62F0A0536951841411106C6CB
:1035C0003697AE87B28502871307700F6145639DFA
:1035D000E700B7E70400FC471306700F170500204B
:1035E0001305C52082970145B240410182800547FD
:1035F0006145E39BE7FEB7E70400FC470546170576
:1036000000201305252EF9BF1307700F6145E39DB8
:10361000E7FCB7E70400FC471306700F170500200E
:103620001305852CC1B71307700F6145E39EE7FAB8
:10363000B7E70400FC471306700F170500201305B9
:10364000253A4DB715476145E390E7FAB7E704001F
:10365000FC471546170500201305454861B7094585
:103660008280411126C2B7E4040083A7C41322C498
:103670004AC006C62E84970500209385E5452A8911
:103680008297058905C5970700209387E79E83D712
:10369000A70BA28503A3440D2310F4002244B240DB
:1036A00092444A850249014641010283B2402244C4
:1036B00092440249494541018280970700202385B1
:1036C00007429707002023A30742B717004003A72C
:1036D000070CB706C0FFFD16758F23A0E70C03A7E4
:1036E000070DB7064000558F23A8E70C03A7070C6A
:1036F0003D9B23A0E70C03A7070D1367070123A831
:10370000E70C8280B717004003A5470C83A7470C3E
:10371000598113451500C18B058999E3136525006F
:103720009707002083C7473C6380A70297070020C4
:10373000238CA73A11C9970700209387273B03A33F
:1037400007006303030002838280114517F3FFFF24
:10375000670063DB411193962500AA852D4506C6B7
:1037600097F0FF1FE780E005B240014541018280EC
:10377000011122CC06CE3714004026CA4AC84EC6D4
:1037800052C483447405034AB4058349840503493C
:10379000940597F0FFFFE780E0B18347A40593F419
:1037A000F40F137AFA0F93E71700230DF40493F93B
:1037B000F90F1379F90FB717004003C7A705058B59
:1037C0006DFF03D5C705A38D4705238C3705A38C53
:1037D0002705A38B9704F2406244D2444249B24980
:1037E000224A0561828041119397050122C406C6D1
:1037F00026C2C1872E8463DC0700B7E40400FC54B2
:10380000829719C1BC5482972165218D15A893F721
:10381000150013C515008DE793F725009DC7970088
:103820000000E78060EEB7E70400BC4F1306000A13
:103830008945170500200345E52B82971345240091
:10384000B24022449244410182809397250163D87B
:103850000702B7E4040083A7C41E82979700000004
:10386000E780E0EEBC4C37F60200130606E08965FF
:1038700017050020034505288297096579B79397B6
:1038800015010145E3DE07FA17D501001305C50E42
:1038900097B00100E780C04BB7E70400BC4F1306A8
:1038A00000649165170500200345C52482971165C2
:1038B000A9BF2D71232A9110FD74E98C232C81104E
:1038C00023282111232631112A84AE8932899306B7
:1038D00000100A86A6852D45232E111097F0FF1F94
:1038E000E78020EE13154401B7E70400FC4751813F
:1038F0000A0513962900CA850A958297A6858566CA
:103900000146254597F0FF1FE780A0EB0A86A685B4
:1039100093060010294597F0FF1FE78080EA832077
:10392000C111032481118324411103290111832929
:10393000C11015618280B7F7070003C70701411165
:1039400006C622C426C24AC0A547631DF7009700D9
:103950000000E78040F6B24022449244024901450B
:103960004101828013942500AA843289A286AA8507
:103970000146254597F0FF1FE780A0E4A2864A860E
:10398000A685294597F0FF1FE780A0E3E9B71D71E1
:10399000A2CC37E404005C5C485886CE494697D5F3
:1039A00001009385E5F8829711E917D50100130509
:1039B00065F997B00100E780A03901A0B7F600E0F3
:1039C000795798CAFD57DCCA0567B7E700E023A01E
:1039D000E7101306F00290C223A0E71801000100CF
:1039E000370700201847130600048145970600207A
:1039F00023A0E6104157A38AE7403C440808829779
:103A0000971700209387C7AB3EC885671387074089
:103A1000231AE1001D673ACC370701051307071089
:103A20003ACE9387B7D31307B00F2310E1022312C6
:103A3000F102054797F7FFFF9387E7542301E1025F
:103A40003ED817070000130727D197070000938778
:103A500067D2B7F50700BAC23EDC170700001307AC
:103A6000C7ED97070000938787CE81463000E105B8
:103A70001945BAC43EDE97F0FF1FE78080D41808CE
:103A80008147994630003E960346060085070507A4
:103A9000A30BC700E398D7FEC24791C70357410164
:103AA00085676373F70001A0B7E7040083A7470A9F
:103AB00008088297AA8511C917D501001305C5E921
:103AC00097B00100E780E01001A0F6406644256150
:103AD0008280411126C2B7E4040083A7040806C609
:103AE00022C417050000130545D082971704002053
:103AF000130444002300A40097000000E780800224
:103B000097000000E780A0BB03450400224403A304
:103B10008405B24092441306003289654101028354
:103B2000797106D622D413078008F337078093F7FC
:103B300087083EC201000100B717004093057005D9
:103B40002380B704130680FA2380C7040100010014
:103B500083C6F70293F6A60FA387D7022380070434
:103B60009246F3A6068001000100733707801377A1
:103B700087083AC4010001002380B7042380C704EA
:103B80000100010003C7F70213672700A387E702BC
:103B900023800704A247F3A7078001000100054521
:103BA00097E0FFFFE780407497000000E78020BAAD
:103BB000014781468147054685451305407E97E0CC
:103BC000FFFFE780407737E404003C44680051463B
:103BD00081458297B707C0A83EC8B787E803938797
:103BE00007D03ECA97E7FF1F9387677D3EC67C5884
:103BF00068008297B250225445618280411197D566
:103C000001009385A53D17D501001305E5CD06C636
:103C100097B00100E780E0FB17D501001305C554FC
:103C200097B00100E780E0FAB2402945410117B39F
:103C300001006700E3FE411197D501009385453BE4
:103C400017D50100130545CA06C697B00100E780E5
:103C500040F817D501001305E54F97B00100E78044
:103C600040F7B2402945410117B30100670043FB0B
:103C7000411122C406C6834705002A849DC797D5F3
:103C800001009385A53C17D501001305E5C597B044
:103C90000100E78000F44C4017D5010013050561D1
:103CA00097B00100E780E0F23DA058410DEF97D5B5
:103CB00001009385A53917D501001305E5C297B01A
:103CC0000100E78000F117D501001305A55F97B04B
:103CD0000100E78000F02244B2402945410117B3BA
:103CE00001006700E3F3A1679386D7036313D7024C
:103CF00097D501009385853517D501001305C5BEFD
:103D000097B00100E780E0EC17D501001305855C52
:103D10007DBFED0797D501009385453317D5010089
:103D2000130585BC631BF70097B00100E78060EACC
:103D300017D501001305455B59BF97B00100E78017
:103D400040E94C4017D501001305055C91BF4111B6
:103D500097D501009385052B17D501001305C5B82C
:103D600006C697B00100E780C0E6B2402945410190
:103D700017B301006700C3EA797122D426D24AD072
:103D80002E842A898145B2844800714606D697E080
:103D9000FFFFE780C03597F7FF1F9387A75FDC47DA
:103DA00083D70700231421012313F100975000004B
:103DB000E780E0039547A305F1009307401F3EC647
:103DC000FD572305A100230AF10097500000E7806A
:103DD00040162686A285480097500000E780000420
:103DE000B250225492540259456182809727002094
:103DF000239B07B497270020238407ACB7E7040070
:103E0000BC47411106C641468145170500201305F0
:103E1000A559829797200000E780805C97200000DA
:103E2000E7800037014597600000E78000A317078F
:103E30000020034767599307F00A6315F7029307B9
:103E4000F0F88945170500201305055817070020CD
:103E5000230CF75697070020A388075697600000A9
:103E6000E78000D097600000E780E0E181453705FA
:103E700004009707002023A70752970700202391EB
:103E8000075297070020238E075097070020239F93
:103E9000074897070020239D074697070020239097
:103EA0000750970700202399075097300000E780BC
:103EB0000042014597600000E78080D397D501005C
:103EC0009385C51617D50100130505A297B001000B
:103ED000E78020D017D501001305454997B00100B0
:103EE000E78020CFB2402945410117B301006700A8
:103EF00023D3411122C406C626C293F715002E848F
:103F0000638F0710814617F6FF1F1306E6458545A8
:103F1000170500200355853F97C00000E780203D2E
:103F200015C997D501009385251117D501001305F3
:103F3000A59B97B00100E780C0C917D50100130504
:103F400065B297B00100E780C0C8294597B001006D
:103F5000E78000CD97D501009385050E17D50100A8
:103F60001305859897B00100E780A0C617D501001A
:103F7000130585B097B00100E780A0C5294597B02B
:103F80000100E780E0C917F5FF1F1305A5405C4558
:103F900005472390E70097400100E780A0ED97D503
:103FA00001009385650917D501001305E59397B0C6
:103FB0000100E78000C217D50100130525AD97B0B9
:103FC0000100E78000C1294597B00100E78040C5A6
:103FD000930710F8170700202308F73E97070020E3
:103FE00083D7873217070020A300F73E170500206C
:103FF0001305853DA1839145170700202307F73C52
:1040000097070020A383073C97600000E78040B536
:1040100013451400B240224492444101828093F738
:104020002500E1C3170700200357873745CB9706C4
:10403000002093862637944297D70100938707354F
:10404000170600200346E6358145170500201305B5
:10405000A53597700000E780E048AA8441C197D554
:1040600001009385250417D501001305E58797B056
:104070000100E78000B6A68517D50100130585A2CB
:1040800097B00100E780E0B4294597B00100E780D0
:1040900020B99707002023950730930710F81707DA
:1040A00000202303F7329707002083D7E72517075F
:1040B0000020A30BF730A183170700202307F73058
:1040C00091458D471705002013050530170700207F
:1040D000A30DF72E97600000E78080A81345240009
:1040E00015BF93F74500D1C397D50100938585FB94
:1040F00017C501001305457F97B00100E78060AD4B
:1041000017D501001305C59B97B00100E78060AC8F
:10411000294597B00100E780A0B0930720F8170762
:1041200000202303F72A9707002083D727201707AB
:104130000020A30BF728A183170700202307F728E7
:10414000854717070020A302F72897500000E78053
:1041500040DE1705002013052527914597600000D4
:10416000E78000A01345440075B593F78500A9C703
:1041700097D50100938505F317C501001305C57692
:1041800097B00100E780E0A417D5010013058594DE
:1041900097B00100E780E0A3294597B00100E780D0
:1041A00020A897070020239D071E97700000E78036
:1041B000404313458400B9BD93F70501D1C385453C
:1041C000170500200355851697600100E78060F50C
:1041D00097D50100938505ED17C501001305C5703E
:1041E00097B00100E780E09E17D501001305C58F49
:1041F00097B00100E780E09D294597B00100E78076
:1042000020A2930730F817070020230FF71A97070B
:10421000002083D7A71117070020A307F71A170557
:1042200000201305651AA1838D4517070020230E72
:10423000F71897600000E780A09213450401D9BBEE
:1042400093F70502D1C797D501009385A5E517C55A
:1042500001001305656997B00100E780809717D5C5
:1042600001001305A58A97B00100E78080962945D3
:1042700097B00100E780C09A930740F81707002025
:104280002304F7149707002083D787081707002017
:10429000A30CF712A183170700202308F712854704
:1042A00017070020A303F7129707002023920706A1
:1042B00097500000E780E0C7170500201305C510E0
:1042C000914597600000E780A0891345040299B3E7
:1042D00093F70504FDC397D501009385A5DC17C5A9
:1042E00001001305656097B00100E780808E17D547
:1042F00001001305258397B00100E780808D2945D3
:1043000097B00100E780C0919707002083C7C70BD3
:104310001307700A6386E7061307800A638CE708B1
:104320001307600A6393E704930760F817070020F8
:10433000230CF7089707002083D76706170700208C
:10434000A304F708A183170700202300F708854777
:1043500017070020A30FF706B14517050020130526
:10436000A50697500000E780A07F97500000E780E7
:1043700040BC13450404970700202392070259B953
:10438000930770F8170700202300F7049707002011
:1043900083D7E70017070020A308F702A1831707B8
:1043A00000202304F702854717070020A300F70227
:1043B000994565B7930780F8F1B793F7050801456C
:1043C000E38A07C497D501009385C5CD17C50100C1
:1043D0001305855197A00100E780A07F17C5010054
:1043E0001305C57597A00100E780A07E294597B009
:1043F0000100E780E0829307A0F81707002023055B
:10440000F7FC9707002083D727FB17070020A30D91
:10441000F7FAA183170700202309F7FA8547170742
:104420000020A304F7FA97070020239707F8975076
:104430000000E78000B0170500201305E5F891455E
:1044400097500000E780C07113450408E1B64111A0
:1044500022C497D501009385A5C02A8417C5010001
:104460001305854806C697A00100E78080764C407A
:1044700017D50100130505E197A00100E7806075DD
:10448000294597A00100E780A0790347040093071E
:10449000F00F631FF70297D50100938565BC17C520
:1044A00001001305654497A00100E78080724C402D
:1044B00017D50100130505DE97A00100E7806071A4
:1044C0002244B2402945410117A30100670043750A
:1044D000B240224441018280B1C1411122C417C5BA
:1044E0000100130565402E8497D50100938545B2E0
:1044F00006C697A00100E780C06DA28517D5010010
:10450000130585E497A00100E780A06C2244B24027
:104510002945410117A30100670083708280411182
:1045200022C426C22E84AA8497D50100938505AFA4
:1045300017C501001305453B06C697A00100E7809B
:10454000406917D501001305E5E097A00100E78059
:104550004068294597A00100E780806C97D501004D
:104560009385C5AB97070020239297DA17C5010002
:1045700013058537854497070020239787D8970729
:104580000020239497D897170020239E873A97A05E
:104590000100E78000649715002083D5C53A17D540
:1045A00001001305A5DB97A00100E7808062294583
:1045B00097A00100E780C0669717002023829730FC
:1045C00097200000E780C0BC228597500000E7805C
:1045D000C028054597500000E780806197F7FF1FCE
:1045E000938747DBDC4703D70700C167FD176312DA
:1045F000F7022244B7E70400B240924403A38705C0
:1046000017F5FF1F0345854F1306000A8545410135
:104610000283B2402244924441018280011122CCA3
:1046200037E404005C5C06CE26CA354697D5010007
:104630009385C5B417E50100130505A4829711E918
:1046400017C501001305053097A00100E7804070F1
:1046500001A097F7FF1F9387274B3EC4B7F50700CC
:10466000856793870780814617F6FF1F1306464923
:10467000E10519453EC697E0FF1FE78080147C44A2
:10468000194697F5FF1F9385A547170500201305C9
:1046900025CA8297340017F6FF1F1306664697D582
:1046A00001009385650117D5010013056502977018
:1046B0000000E78020B8AA8421C197D50100938526
:1046C000659D17C501001305252297A00100E7800D
:1046D0004050A68517D50100130545AB97A00100F2
:1046E000E780204F294597A00100E7806053F24002
:1046F0006244D2440561828097E00000E780601A3E
:1047000017D501001305859F97600000E78040AC36
:1047100097A00000E780A06E97600100E78020D39B
:1047200017F5FF1F130585C397600100E780C0BB25
:1047300017D501001305859D97600100E780A0D380
:10474000AA8497600000E780801297100100E7803C
:1047500000AB97800100E780204497700000E7805D
:10476000C06A97700000E780808897300100E7807A
:10477000606C97D501009385E59117C5010013057D
:10478000A51699C897A00100E780A044A68517D573
:1047900001001305E5A199B797A00100E7806043E8
:1047A00017D50100130505A397A00100E78060421B
:1047B000294597A00100E780A04697300100E780D7
:1047C000404897F00000E7800067630F05108545BB
:1047D0003705040097300000E78060AF97D50100EF
:1047E0009385458B17C501001305051097A001009F
:1047F000E780203E17D501001305459F97A00100D3
:10480000E780203D294597A00100E780604197F7A8
:10481000FF1F9387E7A783D70700171700202314EC
:10482000F712854717170020230CF7089720000080
:10483000E78080B597200000E7808095171500205D
:104840000355651097500000E7802001970700206E
:1048500083C7D7C6ADEBA303010083274417130614
:104860007100854513055030829797D501009385D7
:10487000658217C501001305250797A00100E78091
:10488000403517D501001305A59897A00100E780D2
:104890004034294597A00100E780803897C5010082
:1048A0009385457F17C501001305050497A00100F6
:1048B000E780203217D501001305859B97A00100E2
:1048C000E780203105B597C501009385A57C17C504
:1048D00001001305650197A00100E780802F17D51F
:1048E00001001305659655B797C501009385857A34
:1048F00017C50100130545FF97A00100E780602D53
:1049000017D50100130585A697A00100E780602C4C
:10491000294597A00100E780A0300145975000008D
:10492000E780002DA5BF411122C437E4040083278E
:10493000041A06C6829797500000E78020FB832761
:10494000040817F5FFFF1305055B829797F7FF1F14
:104950002386A71A17F5FF1F1305C5A3975000005C
:10496000E780C08F2244B240410117030000670076
:1049700023CBB1CD29CD411126C2B7E40400FC44BC
:1049800006C622C441462A84170500201305C5A186
:10499000829717050020130525A197200000E780C6
:1049A000C09797100000E780A07E9707002023990A
:1049B000879E224403A38405B240924417F5FF1F4B
:1049C0000345C5131306000A89454101028382800D
:1049D000B7E70400FC471171A2DDCAD986DFA6DB68
:1049E000CED72E8432892E86AA851705002013057E
:1049F000A59D8297170700201307079D834707008F
:104A0000930680029387E70793F7F70FE3ECF6101E
:104A1000BA898A0717C70100130747F6BA979C435C
:104A2000BA9782878D4797C501009385E56817C5BA
:104A30000100130565EB630FF40097A00100E78008
:104A4000401917C501001305E52597A00100E7806F
:104A50004018BDA497A00100E780A01717C501006A
:104A60001305C52597A00100E780A016294597A04A
:104A70000100E780E01A930720F81146970500200F
:104A8000938585944A8517070020230FF79297078F
:104A90000020A38C079297F0FFFFE780202E2A8446
:104AA0001DC997C501009385256117C50100130530
:104AB000A5E397A00100E780C011A28517C50100FA
:104AC0001305852397A00100E780A010294597A032
:104AD0000100E780E01497C501009385E55D17C5E7
:104AE0000100130565E097A00100E780800E17C55F
:104AF00001001305A52197A00100E780800D29453D
:104B000097A00100E780C0114165930730FA054680
:104B1000970500209385458B7D15170700202305F9
:104B2000F78A97F0FFFFE78060252A841DC997C5A3
:104B300001009385655817C501001305E5DA97A0B4
:104B40000100E7800009A28517C501001305C51AF9
:104B500097A00100E780E007294597A00100E780C2
:104B6000200CB7E70400BC4F0566130606C8A14534
:104B700017F5FF1F034585F88297FE506E54DE54EB
:104B80004E59BE591161828091476303F40297C563
:104B900001009385655217C501001305E5D497A060
:104BA0000100E780000317C501001305651971BDF9
:104BB000B7E70400FC4F914517F5FF1F034505F4C7
:104BC000829797C501009385254F17C501001305EE
:104BD000A5D197A00100E780C0FF17C5010013050C
:104BE000E51797A00100E780C0FE294597A00100C6
:104BF000E780000397400000E780A033914535A48B
:104C000085476303F40297C501009385E54A17C5FC
:104C10000100130565CD97A00100E78080FB17C553
:104C200001001305251515B597F7FF1F2390277170
:104C3000B7E704000566BC4F130606C8C1450DBFA3
:104C40008D476303F40297C501009385E54617C5B8
:104C50000100130565C997A00100E78080F717C51B
:104C600001001305E512D5B3930740F8114697F5F7
:104C7000FF1F938565754A8517F7FF1F2306F77495
:104C800097F7FF1FA383077497F0FFFFE780000FDC
:104C90002A84E30405EE97C501009385E54117C515
:104CA0000100130565C497A00100E78080F2A2858A
:104CB00017C501001305450497A00100E78060F1C6
:104CC000294597A00100E780A0F545BD9147E31C69
:104CD000F4F6B7E70400FC4F9305000217F5FF1F39
:104CE0000345C5E1829797C501009385E53C17C54B
:104CF0000100130565BF97A00100E78080ED17C58F
:104D000001001305650AF1BD894763E3870297C572
:104D100001009385653A17C501001305E5BC97A00E
:104D20000100E78000EB17C501001305250931BB21
:104D300097F4FF1F83C4646997F7FF1F83C7D76881
:104D400097C5010093854537A20417C501001305D7
:104D5000A5B9DD8C97A00100E780A0E7A28517C563
:104D600001001305E50697A00100E78080E6C20474
:104D7000294597A00100E780A0EAC1849305D4FFEC
:104D800093960401C1824A8693F5F50F17F5FF1F2C
:104D90001305B56397200000E7802057E35F90DCA0
:104DA000930750F817F7FF1F2300F76283C73900F6
:104DB000228697F5FF1F9385256185074A8517F79A
:104DC000FF1FA304F76097F0FFFFE78020FB2A8412
:104DD000E30505DA97C501009385052E17C5010087
:104DE000130585B097A00100E780A0DEA28517C556
:104DF000010013056554C9B5894763E3870297C568
:104E000001009385652B17C501001305E5AD97A03B
:104E10000100E78000DC17C50100130525FD35B151
:104E200097400000E780E010A28517F5FF1F1305EB
:104E3000A55997500000E780A0D281B38D47630346
:104E4000F40297C501009385252717C501001305B6
:104E5000A5A997A00100E780C0D717C501001305D9
:104E6000A5FAE5B6B76602000146B775020005452A
:104E700097E0FF1FE780E094930760F817F7FF1FA4
:104E80002304F75497F7FF1FA381075493070006E5
:104E900017F7FF1F230CF752894717F7FF1FA307C8
:104EA000F75297F7FF1F2384075297F7FF1FA3803E
:104EB0000752C14717F7FF1F230CF750930720F93C
:104EC00017F7FF1FA306F750314697F7FF1FA3827E
:104ED000A75097F5FF1F9385254F4A8597F7FF1F2A
:104EE0002389074E97F0FFFFE78040E92A84E30615
:104EF00005C897C501009385251C17C5010013053A
:104F0000A59E97A00100E780C0CCA28517C501002F
:104F1000130505F155B3B1476303F40297C50100CA
:104F20009385851917C501001305059C97A00100FD
:104F3000E78020CA17C50100130545F039B6B7E769
:104F40000400FC4F9305000417F5FF1F034505BB44
:104F5000829797400000E780C0FDB145F9B59147C1
:104F600063E3870297C501009385051517C5010006
:104F70001305859797A00100E780A0C517C501001C
:104F8000130585EDD9B497F4FF1F83C4244497F724
:104F9000FF1F83C79743A204DD8C8E04B7770200FE
:104FA0006D14BE942286A68517C50100130505EC75
:104FB00097A00100E780E0C1B7E70400FC47228624
:104FC00097F5FF1F9385954028008297931604015B
:104FD000C1823000A685094597D0FF1FE780607E1B
:104FE0002A8409C917C50100130505EA97A0010025
:104FF000E78000D6930770F8194697F5FF1F938551
:10500000A53C4A8517F7FF1F2300F73C97F7FF1FC2
:10501000A38E873A97F0FFFFE78040D62A84E30EFD
:1050200005B497C501009385250917C5010013052F
:10503000A58B97A00100E780C0B9A28517C5010024
:10504000130585E595B99947630BF41297C50100DF
:105050009385850617C501001305058997A00100F2
:10506000E78020B717C50100130585E4F9BA914719
:1050700063E3870297C501009385050417C5010006
:105080001305858697A00100E780A0B417C501002D
:10509000130585E35DBA97F4FF1F83C4243397F7A4
:1050A000FF1F83C79732A204DD8C8E04B7770200FE
:1050B0006D14BE942286A68517C50100130505E26E
:1050C00097A00100E780E0B0B7E70400FC47228624
:1050D00097F5FF1F9385952F28008297931604015B
:1050E000C1823000A6850D4597D0FF1FE780606D17
:1050F0002A8409C917C50100130505E097A001001E
:10510000E78000C5930780F8194697F5FF1F938540
:10511000A52B4A8517F7FF1F2308F72A97F7FF1FCC
:10512000A386872A97F0FFFFE78040C52A84E3061D
:1051300005A497C50100938525F817B5010013054F
:10514000A57A97A00100E780C0A8A28517C5010035
:105150001305C5DB95B699476303F40297C50100B3
:10516000938585F517B501001305057897A0010013
:10517000E78020A617C501001305C5DAF9B0B7E727
:105180000400FC4F9305000417F5FF1F0345059726
:10519000829797400000E780C0D9994579B18D4743
:1051A0006303F40297C50100938505F117B501006B
:1051B0001305857397A00100E780A0A117C5010022
:1051C0001305C5D759B017C50100130525D897A0F9
:1051D0000100E780E0B71305C01297D0FF1FE780FA
:1051E0004016014597E0FFFFE780E0D60D45971098
:1051F0000000E780E0A3294597D0FF1FE7806014F7
:1052000097D0FF1FE780C0048DBA99476303F4026B
:1052100097C50100938545EA17B501001305C56CD4
:1052200097A00100E780E09A17C501001305C5D2D9
:1052300029B817F7FF1F0347771997F7FF1F83C791
:10524000E71822075D8F9166BA96C2061166C18281
:105250001306F6EF8D476365D60297E7FF1F938726
:1052600067139C4B17F6FF1F034636169386C7003D
:105270002DC203D6070069CA8907E39CD7FE894778
:105280001307A0F8114697F5FF1F9385E5134A858C
:1052900097F6FF1F238AE61217F7FF1FA307F712DF
:1052A00097F0FFFFE78080AD2A84E308058C97C55F
:1052B0000100938565E017B501001305E56297A02D
:1052C0000100E7800091A28517C50100130505CAFA
:1052D000E5B203D60700630EE60A8907E39BF6FEF4
:1052E0008D4779BF91476304F40297C50100938508
:1052F000A5DC17B501001305255F97A00100E78025
:10530000408D17C501001305E5C76FF00FF4B7E72F
:105310000400FC4F9305000817E5FF1F0345057EB9
:105320008297C9B897C50100938505D917B50100C3
:105330001305855B97A00100E780A08917C50100D0
:105340001305C5C56FF06FF02390E70017E5FF1F49
:105350001305450497300100E78020B497C501008C
:10536000938585D517B501001305055897A0010051
:10537000E780208617C50100130545C397A00100EB
:10538000E7802085294597A00100E7806089814753
:10539000C5BD2390070017E5FF1F1305A5FF973034
:1053A0000100E78080AF97C501009385E5D017B570
:1053B00001001305655397A00100E780808117C5A0
:1053C0000100130525C05DBF411122C406C626C2D7
:1053D0004AC0834705002A84A1C397C5010093856D
:1053E00065C917B501001305255097900100E780A6
:1053F000407E4C4017C50100130545FA9790010007
:10540000E780207D2244B24092440249294541016F
:1054100017A301006700C3805841B707CF009387E7
:10542000777D631CF7080445638504120359C500A2
:10543000630109120354E50097C50100938585C3F4
:1054400017B501001305454A97900100E780607881
:1054500003C60400A286CA8517C50100130585F599
:1054600097900100E780E076294597900100E7805A
:10547000207B4A86A685228597200000E780E0C42D
:1054800083C7140003C70400A207D98F13978700AE
:10549000A183D98FC2073167C1831307C755638AB8
:1054A000E70A22862244B240CA85268502499244F0
:1054B000410117F3FFFF6700E351B707CC00938763
:1054C000777D6310F70697C501009385A5BA17B5D8
:1054D00001001305654197900100E780806F1C442F
:1054E0008355C4008356E40003C6070017C50100B6
:1054F000130545EC97900100E780A06D2945979032
:105500000100E780E0710356C4000C440355E40039
:105510002244B2409244024941011723000067002F
:10552000C3BAB707CE009387777D6304F70297C5A8
:105530000100938525B417B501001305E53A97904E
:105540000100E78000694C4017C501001305C5DB69
:1055500075B5B24022449244024941018280B7E7C6
:105560000400FC4741112E8606C622C426C24AC04A
:105570002E842A89AA8517F5FF1F1305E5E4829773
:1055800097C50100938505B517B501001305C5350D
:1055900097900100E780E06397F5FF1F83C5C5E2A0
:1055A00017B501001305055B97900100E780606265
:1055B000294597900100E780A06697F4FF1F938428
:1055C000A4E083C7040041479387070693F7F70FCA
:1055D000636AF75C17B70100130787448A07BA9715
:1055E0009C43BA9782879D476307F40297C50100E1
:1055F000938545AE17B501001305052F979001005F
:10560000E780205D17B5010013054555979001000F
:10561000E780205CADAC97F7FF1F83C7F7DADDCBDF
:1056200017F7FF1F034777DA97F7FF1F83C7E7D9FD
:1056300022075D8F97F7FF1F83C747D9C2075D8F8A
:1056400097F7FF1F83C797D8E207D98F17F7FF1F78
:10565000232AF7D483C7640097C50100938585A7E3
:1056600017B501001305452817F7FF1F230BF7D2C5
:1056700097900100E780E05597F7FF1F938787D247
:105680008C4317F6FF1F0346C6D117B5010013055B
:10569000A54E97900100E780C053294597900100DF
:1056A000E780005897F7FF1FA38007D22244B2403B
:1056B00092440249930700F817F7FF1F2306F7D01B
:1056C0009D4517F5FF1F130525D041011743000025
:1056D0006700034997600000E780200097F7FF1FED
:1056E0002385A7CE9357850017F7FF1FA30FF7CC8D
:1056F000935705012A8417F7FF1F2309F7CC935707
:105700008501014517F7FF1FA302F7CC9760000042
:10571000E78060FD97F7FF1F238BA7CA97C501009D
:105720009385459B17B501001305051C9790010053
:10573000E780204A17F6FF1F034666C9A28517B502
:1057400001001305E544B1B7CD476303F40297C5E3
:1057500001009385259817B501001305E51897906A
:105760000100E780004717B501001305E54379BD47
:1057700037E404007C44414697F5FF1F9385D5C468
:1057800017F5FF1F130545C2829717F5FF1F130575
:10579000A5C197100000E78040B897100000E7808F
:1057A000209F97F7FF1F83C747C317F7FF1F0347C4
:1057B000B7C2A20703238405D98F17F7FF1F231150
:1057C000F7BE1306000A89452244B24092440249BA
:1057D00017E5FF1F03458532410102838D476303AF
:1057E000F40297C501009385E58E17B501001305F6
:1057F000A50F97900100E780C03D17B50100130584
:10580000654A29B517F4FF1F034424BC97F7FF1F0F
:1058100083C797BB97C501009385C58B220417B535
:1058200001001305650C5D8C97900100E780603ADC
:10583000A28517B501001305A53897900100E780F0
:105840004039294597900100E780803D0D4697F546
:10585000FF1F938565B7228597E0FFFFE780005221
:10586000AA8421C197C501009385C58617B501009B
:105870001305850797900100E780A035A68517B529
:1058800001001305253597900100E78080342244FC
:10589000B240924402492945410117930100670033
:1058A000233897F7FF1F239387A8B7E704001166F3
:1058B00003A38705130606E8914539B78D476303AF
:1058C000F40297C501009385E58017B50100130523
:1058D000A50197900100E780C02F17B501001305BF
:1058E000254B2DB317F4FF1F034424AE97F7FF1F7A
:1058F00083C797AD97B501009385C57D220417B581
:105900000100130565FE5D8C97900100E780602C17
:10591000A28517B501001305252D97900100E7809A
:10592000402B294597900100E780802F0D4697F581
:10593000FF1F938565A9228597E0FFFFE78000445C
:10594000AA841DC197B501009385C57817B50100DC
:10595000130585F997900100E780A027A68517B564
:1059600001001305A52905B797F7FF1F2392879A12
:10597000B7E70400116603A38705130606E893053D
:10598000000299B5894763E3870297B501009385C3
:10599000657417B50100130525F597900100E780A0
:1059A000402317B50100130565418DB197F4FF1F22
:1059B00083C4A4A197F7FF1F83C717A197B5010060
:1059C00093854571A20417B501001305E5F1DD8C3F
:1059D00097900100E780E01FA68517B50100130529
:1059E000652397900100E780C01E2945979001002C
:1059F000E7800023228697F5FF1F9385E59C268587
:105A000097E0FFFFE78080372A84630E051A97B579
:105A100001009385256C17B501001305E5EC9790FF
:105A20000100E780001BA28517B501001305C51F03
:105A300099BD854763F98718834519002244B24010
:105A400092440249B335B00097F7FF1F238AB78EFF
:105A500017B501001305851E41011793010067006A
:105A60004317A2852244B24092444A85024941012B
:105A7000170300006700032299476303F40297B5F8
:105A800001009385256517B501001305E5E597909D
:105A90000100E780001417B501001305E54BBDB602
:105AA00017F4FF1F0344649297F7FF1F83C7D79132
:105AB00097B5010093850562220417B5010013050F
:105AC000A5E25D8C97900100E780A010A28517B534
:105AD00001001305251897900100E780800F2945E4
:105AE00097900100E780C013194697F5FF1F938533
:105AF000A58D228597E0FFFFE7804028AA841DC17D
:105B000097B501009385055D17B501001305C5DD47
:105B100097900100E780E00BA68517B501001305FB
:105B2000651495B397F7FF1F23988788B7E704009C
:105B3000116603A38705130606E89305000869B1FB
:105B4000854797B501009385E55817B50100130502
:105B5000A5D9630BF40097900100E780800717B583
:105B60000100130565115DB497900100E7806006A0
:105B700017B501001305C51197900100E780600576
:105B8000294597900100E780A0092244B240924441
:105B9000024997F7FF1F2395078041011763000013
:105BA000670023A497B501009385C55217B501007E
:105BB000130585D397900100E780A00117B5010078
:105BC0001305C53DA1B4B2402244924402494101AB
:105BD0008280411106C622C497E0FFFFE780001AC9
:105BE0009377F50FA1C32A8497B5010093850550DB
:105BF00017B50100130545CF97900100E78060FDC0
:105C00009375F40F17B50100130505739790010004
:105C1000E78020FC2244B24029454101179301004E
:105C200067000300B240224441018280411122C436
:105C300091462A8417F6FF1F130646879D652D455A
:105C400006C697D0FF1FE780C0B7B7F7070003C7A6
:105C50000701A5476313F70001A093060010014652
:105C60009D65254597D0FF1FE780A0B597F7FF1FDB
:105C7000238E87822244B240914617F6FF1F1306F7
:105C8000E6829D652945410117D3FF1F670063B375
:105C90005171CAD137E904008327C904A2D52E86E1
:105CA00086D7A6D32E84AA8517E5FF1F1305C571D5
:105CB000829797E7FF1F83C727711307700A6387CF
:105CC000E710636CF7001307600A6384E704BE50B3
:105CD0002E549E540E596D6182801307800A63888A
:105CE000E7161307900AE394E7FE8D476309F41C57
:105CF00097B501009385857717B501001305C5BEDB
:105D000097900100E780E0EC17B50100130545739B
:105D100025A08D47630CF40297B5010093850575A6
:105D200017B50100130545BC97900100E78060EAB4
:105D300017B501001305056A97900100E78060E937
:105D4000294597900100E780A0ED51B7854717B529
:105D500001001305E56917E7FF1F2303F75E97901E
:105D60000100E780E0FEB7750200B7660200014659
:105D7000054597D0FF1FE780C0A4930760F817E799
:105D8000FF1F2303F76497E7FF1FA38007649307B0
:105D9000002617E7FF1F232BF762E577938707217C
:105DA00017E7FF1F2316F762B14597E7FF1F23820E
:105DB000076297E7FF1FA38EA76017E5FF1F130574
:105DC000A56097400000E780A0D911B7914763E331
:105DD000870297B501009385656917B50100130522
:105DE000A5B097900100E780C0DE17B5010013054C
:105DF000256299B797E4FF1F83C4445D97E7FF1FAF
:105E000083C7B75CA204DD8C8327C9046D14228686
:105E100097E5FF1F9385955B280082978E04931664
:105E20000401B7750200C1823000A695094597D0DC
:105E3000FF1FE7800099930770F817E7FF1F2305FE
:105E4000F758994597E7FF1FA382A758BDB7914719
:105E500063E3870297B501009385456117B501009B
:105E6000130585A897900100E780A0D617B501001B
:105E70001305855BD1B597E4FF1F83C4245597E7CD
:105E8000FF1F83C79754A204DD8C8327C9046D14B8
:105E9000228697E5FF1F93857553280082978E040D
:105EA00093160401B7750200C1823000A6950D4516
:105EB00097D0FF1FE780E090930780F8BDBF17B52C
:105EC00001001305255997900100E78060E813054C
:105ED000C01297C0FF1FE780C046014597D0FFFF63
:105EE000E78060070D4597000000E78060D42945F2
:105EF00097C0FF1FE780E04497C0FF1FE780403551
:105F0000F9B38280011126CA06CE22CC0344550083
:105F100083474500AA8422045D8C2EC617B5010074
:105F200013058557A28597900100E78080CA2285D6
:105F300062443246F240A685D24405611703000050
:105F4000670063C9011122CC2A8417B5010013052B
:105F5000A55306CE2EC697900100E78060DF22850C
:105F60006244B245F24005611713000067008325C3
:105F70008D4763FBB70A011126CA06CE22CC034423
:105F8000350097E4FF1F83C4745397B501009385D0
:105F9000E551B337800017E7FF1FA301F75209C48B
:105FA00097B501009385455117B50100130545517B
:105FB00097900100E780E0C197E7FF1F83C7175064
:105FC0006386970097000000E780202797E7FF1F70
:105FD00083C7D74E8DC785472306F100B7E7040076
:105FE00083A747177000854513055030829717B572
:105FF00001001305E54D97900100E78060D5996792
:10600000938757EE2316F100680085479145A30753
:1060100081002307F10097400000E78060B4F24060
:106020006244D244056182808280894763F7B70861
:10603000011122CC06CE26CA8344250085472A8436
:10604000639DF404914763F5B70403454500834716
:10605000340022055D8D97D7FF1F239EA73497003C
:106060000000E780C03F9967938767EE2314F10033
:106070008347340023059100A305F10083474400C2
:10608000954528002306F10097400000E78040ADC9
:10609000F2406244D24405618280FDF8996793879B
:1060A00067EE2314F10097D7FF1F83D7C730A305EE
:1060B000F10023050100A183E1B7828001119967F6
:1060C00022CCD51717F4FF1F1304847F2314F1008B
:1060D0008347040026CA970400209384C4862305BE
:1060E000F10083D7040028009545A305F100A183A2
:1060F00006CE2306F10097400000E78060A603D695
:1061000004008345040017B501001305E53D979091
:106110000100E78000ACF2406244D2440561828015
:106120009D677971D9172316F10097F7FF1F83C771
:10613000277906D62307F100A9C3B7E70400FC4777
:10614000414697E5FF1F938525261305F1008297A9
:106150006800CD4597400000E78080A097F5FF1FBD
:1061600083C5057617B501001305053B979001001F
:10617000E78020A6B25045618280B7E70400BC47A3
:10618000414681451305F1008297D9B7B7670203ED
:106190006971938757AA3EC489679387273023166E
:1061A000F10097F7FF1F9387A77183C70700232488
:1061B0008112A30701002307F10097F7FF1F9387C0
:1061C000877883D7070037E40400232611122318A9
:1061D000F10097D7FF1F9387071E83D7070041461B
:1061E00048082319F1007C4497E5FF1F9385C51BE0
:1061F0008297F145280097000000E7804022231293
:10620000A1027C442C002810794682973C44130557
:1062100061041306900D8145829730109305700F2D
:10622000014597D0FFFFE78060388320C112032427
:10623000811255618280B7C7A55A01119387C73370
:106240003EC497E7FF1F83C777273EC6B7F707000F
:1062500003C7070106CE22CCA5476313F70001A0B0
:106260001164930504F0930600100146254597C07C
:10627000FF1FE78000553000930504F0A146294533
:1062800097C0FF1FE780E05397E5FF1F83C51523E5
:1062900017B501001305053997900100E780609359
:1062A000F24062440561828001119165A14630008F
:1062B000938505F02D4506CE97C0FF1FE7806050FF
:1062C0002247B7C7A55A9387C7336314F702B2456D
:1062D00017B5010013054528B335B00097E7FF1F38
:1062E000A38EB71C97900100E780A08EF240056155
:1062F0008280814517B501001305452897E7FF1FE8
:10630000A38E071A97900100E780A08C97000000E9
:10631000E780A0F2E1BFB7C7A55A79719387F73537
:106320003EC6B7E70400FC47AA8506D622D44146FC
:1063300008088297B7F7070003C70701A54763134B
:10634000F70001A01164930504E8930600100146CC
:10635000254597C0FF1FE780C0467000930504E8FD
:10636000D146294597C0FF1FE780A04517B501001A
:106370001305052F97900100E780809DB2502254AD
:106380004561828079719165D1467000938505E8F9
:106390002D4506D697C0FF1FE780A0423247B7C7FA
:1063A000A55A9387F73517B5010013052525631006
:1063B000F702B7E70400FC4717E5FF1F1305C5FE0A
:1063C00041460C08829717B50100130525219790C7
:1063D0000100E780E097B25045618280B7F707007F
:1063E00003C70701A5476313F70001A09165411199
:1063F000930600100146938505E8254506C697C01B
:10640000FF1FE780003CB24017B5010013050513DC
:106410004101179301006700A393C1676976814624
:10642000FD1705061397060141836364B7003E8597
:1064300082803307D50003470700B98F214713F83F
:106440001700858363050800B18FC207C1837D17DC
:106450001377F70F6DF78506F1B7B7C7A55A011186
:106460009387E7343EC42AC6B7F7070003C707017E
:1064700006CE22CC26CAA5476313F70001A091647B
:106480002A84938504EE930600100146254597C0A3
:10649000FF1FE78000333000A146938504EE2945B5
:1064A00097C0FF1FE780E031A28517B501001305F3
:1064B000651997800100E780C07197000000E780B0
:1064C00020CDF2406244D244056182800111916581
:1064D000A1463000938505EE2D4506CE97C0FF1FDF
:1064E000E780202E2247B7C7A55A9387E734631861
:1064F000F702B24517B501001305450A97D7FF1FEC
:10650000239BB7EAC205C18197800100E780606CD8
:1065100097000000E780C0C7F24005618280D14744
:10652000D14517B501001305650917D7FF1F2314BF
:10653000F7E897800100E780C06917D5FF1F035572
:1065400085E797000000E78080F1F9B7411126C286
:1065500006C622C493F71500AE848DCBAD673717FE
:1065600000409387A7AA1CC3B7E70400BC4F1306DB
:106570000019854517D5FF1F0345C5E3829713C54D
:106580001400B240224492444101828093F72500D6
:106590006385071097F5FF1F83C5C53A854793C4E8
:1065A000240063E5B70499CD97E7FF1F83C707F180
:1065B00095C3854517F5FF1F1305C53097300000BB
:1065C000E780005A1395040197F7FF1F238C0736C5
:1065D000418145BF4165054697F5FF1F9385852E8F
:1065E0007D1597F0FFFFE780005FE9BF17F4FF1FFD
:1065F0000344442D97F7FF1F83C7D72C22045D8CDB
:10660000AD679387B755630FF40463EA8702A96700
:106610009387A755630AF406C20597E7FF1F83C750
:10662000E7E9C1819DE741652E867D1597F5FF1F3E
:106630009385452997F0FFFFE780E05925A8B167CA
:106640009387C7556308F402B5679387D755E31559
:10665000F4FC17F5FF1F1305E52697300000E780CF
:10666000205009A817F5FF1F1305C5259700000046
:10667000E7808089A28517B5010013056500978022
:106680000100E78000553DBF17F5FF1F1305852367
:1066900097000000E780408BF1BF93F7450001456C
:1066A000E38107EE17B501001305C5FE97800100D1
:1066B000E780006A97300000E780A05E13C54400C1
:1066C000C9B5411122C437E404005C5C06C63546F6
:1066D00097B50100938585AA17C501001305C599D3
:1066E000829711E917B50100130585FB978001001A
:1066F000E780006601A08327041C82972A84054551
:1067000097C00000E780401997700100E780609E05
:1067100097600100E780607397B00000E780C02AAF
:106720002285B2402244410182801567B71700409C
:106730001307575598C3D8439D66558FD8C3D84380
:10674000FD76758FD8C3D8431367F70FD8C3356765
:106750001307C7CC98C3828041111305800406C675
:1067600022C426C297C0FF1FE780609485457D55EF
:1067700097C0FFFFE780606585457D5597C0FFFFA7
:10678000E780006F371400408327840A8D45130586
:10679000002093E707202324F40A97C0FFFFE78037
:1067A000C062B7E4040097D0FFFFE780C095C858E7
:1067B00097800100E780C05917C501001305C58BFC
:1067C00097800100E780C0588327840C85454145A8
:1067D00093E707082324F40C97C0FFFFE780406984
:1067E0008D451305000897C0FFFFE780606897D0CC
:1067F000FFFFE7800083014597D0FFFFE780E0853A
:1068000085450545894717F7FF1F230FF71297D0D6
:10681000FFFFE780208637070004B7E700E023A0EA
:10682000E71097D0FFFFE780C01697D0FFFFE78003
:10683000802A97000000E78000E997000000E780C9
:10684000E0A697000000E780A0C897E0FFFFE78080
:10685000C00D97100000E78040A797000000E78078
:10686000602D97100000E780C0A183A704081705DA
:1068700000001305E5CD829797D7FF1F238CA7B2A1
:10688000BC4C130600648545829797000000E780A2
:1068900000EA97C0FF1FE780A0B501458280B7F7E7
:1068A000070003C70701A547AE866316F700939755
:1068B000450191C301A0AA850146254517C3FF1FC5
:1068C000670023F04111B2862E86AA852D4506C6A3
:1068D00097C0FF1FE780E0EEB24001454101828092
:1068E0009307000463E8C7021D71A2CC2A8408083C
:1068F00086CE32C697800100E7804022B24610085B
:10690000A285294597C0FF1FE780A0EBF6406644AB
:10691000256182803955828097F7FF1FA38407087D
:1069200097F7FF1F2380071E97F7FF1F238C07068B
:10693000B7E70400FC5F411106C682978967938719
:1069400007F4B2403E9597F7FF1F23ABA704410120
:106950008280930600022547830705006385D700E0
:106960006383E70082800505C5BF17F5FF1F034558
:1069700005030DE5411122C417F4FF1F130444025F
:106980001C4006C681CBB7E70400FC5F82971C4021
:106990001D8D7D81B2402244410182800545828067
:1069A0008145B307B5008387070091E789C917239D
:1069B0000000670003F18505C205C181DDB7828053
:1069C000AA871375F50F130705FD1377F70FA54673
:1069D00063E5E600138507FD82801307F5F9137759
:1069E000F70FE54663E6E600011593178501E18799
:1069F0001387F7FB1377F70F95467D5563E4E600A1
:106A0000138597FC828035C5011126CA4AC84EC637
:106A100052C406CE22CCAE8997000000E780A0F3D6
:106A20002A898144414A0305090097000000E78054
:106A300060F92A840305190097000000E78080F8B8
:106A400063470402634505021204B3879900498C29
:106A50002380870085040909E39744FD0545F2403A
:106A60006244D2444249B249224A056182800145CA
:106A7000FDB7014582808147E5483387F50003076C
:106A8000070019E305458280B306F500038606007A
:106A90009376F60F1388F6F91378F80F63E608017A
:106AA00081161396860161869376F70F1388F6F99F
:106AB0001378F80F63E60801138706FE6207618703
:106AC0006316C7008507C207C18345BF01458280A1
:106AD000011122CC2A842E8526CA4AC84EC606CE6B
:106AE0002E8997800100E780003793140501C1804B
:106AF0009309D0038307040099E301450DA0CA85DB
:106B0000228597000000E78040F70DC1B30794008D
:106B100083870700639C3701138514002295F24098
:106B20006244D2444249B249056182800504D9B722
:106B300097F7FF1FA38807E697F7FF1F238407FC3B
:106B400097F7FF1F238007E697F7FF1F239807E4B7
:106B500097F7FF1F238507E497F7FF1F23A207E49A
:106B600097F7FF1F83C717FA99EF411106C69720C1
:106B70000000E780A0D2B240854717F7FF1FA303AC
:106B8000F7F8410182808280011106CE22CC26CA0C
:106B90004AC84EC697200000E780C0D105E197F7AC
:106BA000FF1F238E07DE97F7FF1F23AB07DEF240A0
:106BB0006244D2444249B249056182809700000094
:106BC000E780E0DA6DF597F4FF1F9384E4DD1309A5
:106BD00040078D4997F6FF1F83C6C6DCE9DA17F731
:106BE000FF1F034737DCB30727033384F400035543
:106BF000240083550400636FB5000507337737031E
:106C0000FD1697F7FF1F238FD7D897F7FF1FA38B8A
:106C1000E7D8C9B7898D91073E95C205C1812695F0
:106C200097200000E78000D359D1835724003E9578
:106C30002311A40045B763070548638505487171B2
:106C400056CBC16A26D34AD14ECF52CD5AC95EC760
:106C500062C506D722D566C36AC12E8AAA890149B0
:106C6000B54B17FBFF1F130B6BCEF91A97D4FF1F01
:106C70009384847317BC0100130C8CB7931709011C
:106C8000C18363E04703BA502A549A540A59FA4917
:106C90006A4ADA4A4A4BBA4B2A4C9A4C0A4D4D6121
:106CA0008280B3872901038707006307770DA94610
:106CB00097F7FF1F83D787CE6313D73AD5CFDA97DD
:106CC00017F5FF1F130585C82380070097000000F4
:106CD000E78060C897B50100938545A32A84970093
:106CE0000000E78080D949C51305640097000000C3
:106CF000E78060C62A8497000000E78020C297B52D
:106D00000100938525A1228597000000E780E0D649
:106D100015CD8307240013F7F7FD01C725476397B7
:106D2000E7021308300289470D4797B601009386A2
:106D3000A69E17B601001306E69E930500080A8575
:106D400097800100E78000020A8539A897B5010005
:106D50009385C59F228597000000E78000D219CD5A
:106D600017B501001305059F97000000E78080C359
:106D700097F7FF1F239407C2050909B797B50100CC
:106D8000938505A2228597000000E78000CF79C592
:106D900083073400130700026385E7002547639FDC
:106DA000E70A1305340097000000E780C0BA97B5E2
:106DB00001009385259F2A8497000000E780E0CB9F
:106DC0000DC19307300209478D4617B6010013061F
:106DD000A69D930500080A8597800100E78080F84A
:106DE000A5B797B501009385A59D22859700000062
:106DF000E780A0C80DC517F7FF1F034767AC97F6DC
:106E0000FF1F83D646B417B601001306E69B930511
:106E100000080A8597800100E780C0F435B797B570
:106E200001009385A59C228597000000E780E0C4BF
:106E30000DC181474147B386970083C60600639E14
:106E400006228507E399E7FE17B50100130585AF14
:106E500021BF17B501001305259A39B797B5010071
:106E60009385859B228597000000E78000C163031E
:106E7000051E83073400130700026385E7002547DA
:106E8000639AE71C1305340097000000E780A0AC6C
:106E900097B50100938585982A8497000000E780C4
:106EA000C0BD2DC19305D003228597800100E780E6
:106EB000C0F711C9830615000547938706FD93F7B0
:106EC000F70F6377F70017B501001305A59569BDA6
:106ED00093071003639FF60097F7FF1F2381E7AC2A
:106EE00097000000E78080A317B501001305059601
:106EF000A5BD97F7FF1F238407AA97F7FF1F23A1BC
:106F000007AADDB797B501009385458E22859700C6
:106F10000000E78080B631C99305D00322859780B1
:106F20000100E78080F011E517B501001305859396
:106F300025BD8A85050597000000E78000AD6DD569
:106F4000B7E70400FC4741468A8526858297268557
:106F500097F0FFFFE780603C97F0FFFFE78040235A
:106F600017B501001305459201B597B5010093854A
:106F70002585228597000000E78020B079C597B568
:106F800001009385A591228597000000E78080B4D9
:106F90002A8D97B5010093856585228597000000AD
:106FA000E78040B3AA8C63080D046A8502C097008D
:106FB0000000E780409A01468A852A8D978001006B
:106FC000E780200182472A846307FD029307F5FFCB
:106FD00063E3FA0263960C0281474147B386970048
:106FE00083C60600B1E68507E39AE7FE17B5010000
:106FF0001305059795BB17B501001305A58AADB319
:107000008A85668597000000E78020A011E517B506
:1070100001001305658B89BBB7E70400FC47268593
:1070200041468A858297268597F0FFFFE780E02E0C
:10703000131504014181A68597E0FFFFE780A09327
:1070400017B501001305858A05B317B501001305AF
:10705000658B19BB17B501001305C58C31B3938639
:1070600017001306F004E365D6D0DA9717F6FF1F72
:107070002316D6922380E70001B397B501009385CC
:10708000658D0A8597800100E780C0DB814C130481
:10709000B100414DB387940103C607002285E28504
:1070A000850C97800100E78060D30904E394ACFF6E
:1070B00097A50100938505E4228597800100E7806C
:1070C00060D859B18280E5CD854763FAC70E83C782
:1070D000150003C70500A207D98F13978700A18366
:1070E000D98FC2073167C1831307C7556399E70C6E
:1070F00097F7FF1F83D727856383A70C797122D465
:1071000026D206D64AD04ECE3284AE842AC6970006
:107110000000E780C08535ED93070007B24563E1C5
:10712000870817F7FF1F0347E787894763EAE706E2
:1071300097F9FF1F83C9099D93074007B389F90297
:10714000B7E70400FC4717F9FF1F1309E9852286FA
:10715000A685138549004A95829797F7FF1F83C735
:10716000679A0D478507B3F7E7024E992310890008
:107170002311090017F7FF1F2306F79897F7FF1F42
:107180009387478283C70700850717F7FF1F230BE5
:10719000F780B250225492540259F24945618280DC
:1071A00022862254B25092540259F24917A5010086
:1071B0001305457D456117830100670083A1828027
:1071C000011106CE22CC26CA01C5D54763EFB70010
:1071D00017A501001305057D97800100E78040B7E2
:1071E000F2406244D2440561828003470500930760
:1071F000500A2A846318F700034715009307A00577
:107200006307F70017A501001305457BF1B7034796
:1072100035009307100A630EF70059476386E500AF
:10722000034745006305F70217A501001305457ADA
:1072300065B7D1449147D1465D476393D400594720
:1072400063FAE50017A501001305057A71B7D54467
:107250009547D5B737E704007847B305F4000A85AA
:1072600041460297269483471400034504008A850B
:10727000A2075D8D97D0FFFFE780E06F95B74111C2
:107280000D658D4506C697C0FFFFE78060BEB71746
:1072900000408D6623A6D70C17F5FF1F1305C58682
:1072A0001387C70C9387870C1CC15CC585668967EB
:1072B0005CC958C114C518C9B7E70400B24003A39C
:1072C000871E4101028382808280411126C2AE84E2
:1072D0008D4522C406C62A8497C0FFFFE78040B9C7
:1072E000B717004099C803A5C70C418D23A6A70C6A
:1072F000B240224492444101828003A5870C418D13
:1073000023A4A70CF5B78347050003471500A20780
:10731000D98FC2076177C18713072720639AE700D7
:10732000834525003705040017030000670023FA92
:10733000828017E6FF1F1306E67E8147B28613039D
:10734000F00FA9483308F6000348080013F7F70FB9
:107350006307A80C630668008507E39517FF2947B4
:10736000B387E6002380A70097E7FF1F9387477C3A
:107370005DA8411113D765001347170006C693F6A1
:107380003500058B954791CA054699476387C60026
:1073900009469D476383C600A14713F6450033366F
:1073A000C00093F68503050685C2A145638BB6042C
:1073B000E145638AB604930580026388B6049305A9
:1073C00080036393B600914697F5FF1F2387F59CD2
:1073D00097F5FF1F2382C59C97F5FF1FA38ED59AB3
:1073E000BE8517A501001305256497700100E7808D
:1073F000407EB240854717F7FF1FA300F79A41016F
:1074000082808546D1B78946C1B78D4675BF17A51D
:1074100001001305E563177301006700837B17E71D
:10742000FF1F1307E770BA972380B700E147E30215
:10743000F5F493077002E30CF5FC82802A87238021
:107440000500814717E5FF1F1305C56D1308F00FF1
:107450002946B306F50083C606006396E60297E662
:10746000FF1F9386E66CB69783C707000545238008
:10747000F5009947636EF7029D4763FDE700E1471A
:10748000630DF7008280638506018507E393C7FCDF
:107490000145C5B7238005008280B737004003C788
:1074A000370083C7050093F70704D98F2380F500C1
:1074B0008280797126D24AD097F4FF1F83C4C49783
:1074C00017F9FF1F1309899606D622D44ECE52CC47
:1074D00056CA5AC8B307990083C7070093F7F70F36
:1074E000A5C79387140093F7F70F0D476361F70C57
:1074F00017F7FF1F2302F79497F7FF1F93878793D0
:10750000A69783C707001307100293F7F703638F4B
:10751000E7266363F70A054463808720E389076CE5
:1075200009476389E71413070002E38EE756B7E7BC
:1075300000E03707400023A0E71801000100CA94CB
:107540002380040023A0E710B787004003C767002B
:10755000058BE30F077697F6FF1F83C6068E054758
:10756000E39AE67429472381E70209472383E70268
:107570002385E70297F7FF1FA382078297F7FF1F74
:10758000A38D078AB7870040A381070017F7FF1F65
:10759000A308078005472383E700B2502254925482
:1075A0000259F249624AD24A424B4561828097F7BA
:1075B000FF1F2383078889B7130730026386E70A12
:1075C00063E6E71413074002638AE7081307000322
:1075D000E39FE7F497F7FF1F93878785A69703C775
:1075E0000700A1471377F70FE31AF71A17EAFF1FEF
:1075F000130ACA5483476A0097E6FF1F2386F6786A
:1076000097E7FF1F83C7F75391C7FD5797E6FF1F03
:10761000238CF67697E5FF1F83C5555297E7FF1F2A
:10762000A384B77697E7FF1F83C7475193F90708ED
:107630009306000493F707066393D7509307A009B6
:10764000638DF51863EAB7149307F005638AF54C68
:10765000930750096388F52C0144BDABFD5717E72C
:10766000FF1F2302F772E1B5FD5717E7FF1F230B3A
:10767000F77075BD17A501001305054F9770010040
:10768000E780006D97E7FF1F9387877AA69703C46B
:107690000700814917EAFF1F130ACA621374F40F27
:1076A00097AA0100938ACA4C63C789042945977039
:1076B0000100E780E056854717E7FF1FA302F76048
:1076C00017E7FF1F230F875E17E7FF1F2308F76CDD
:1076D00037E700E0B70640002320D718010001007B
:1076E000378600408347A60293F7370F2305F6023B
:1076F0002320D7102DBDB3073A0183C50700568557
:10770000850997700100E780C04C79BF854717E76E
:10771000FF1F2307F75A21BD17A501001305C54414
:1077200097700100E780C06297E7FF1F938747705B
:10773000A69703C40700814917EAFF1F130A4A4CA2
:107740001374F40F97AA0100938A8A4263C58902D1
:10775000294597700100E780A04C854717E7FF1F78
:10776000A30EF74817E7FF1F230B874817E7FF1FF4
:107770002306F7626DBBB3073A0183C50700568540
:10778000850997700100E780C044C9B7854717E7AE
:10779000FF1F2305F74661BB9307400A638DF5344D
:1077A0009307200B6388F5369307100AE396F5EAF2
:1077B00083072A00014463D1074297E7FF1F83C76D
:1077C000173893F63700638E061A0546638EC62275
:1077D00009466399C61A1D4775A217E5FF1F0345A1
:1077E0000536C94717EAFF1F034A7A3597E5FF1F99
:1077F00083C5053517E4FF1F034494346319F5105E
:10780000CD476316FA1093077008639CF5021307BF
:10781000300FB7170E006308E4001307900DB7B7D9
:1078200004006314E40817E7FF1F2325F756BE85FD
:1078300017A501001305453497700100E7806039F2
:1078400021BD93078008639DF50033048040B7771E
:1078500046001374F40F938787CDB3D78702E1B73F
:1078600093079008639AF50033048040916713747E
:10787000F40F9387C766D5B79307A008639BF500FD
:1078800033048040B7173D001374F40F93870790BB
:10789000E9B79307B008639AF50033048040916715
:1078A0001374F40F938797D04DBF93F5F5078D4769
:1078B000639BF50033048040B7975B001374F40FAB
:1078C000938707D859BF8947639BF50033048040ED
:1078D000B7770B001374F40F9387071BBDBF854761
:1078E000639AF50033048040DD671374F40F9387C7
:1078F00067E3A5B789E9330480408D671374F40FFB
:10790000938777DC99BFF1679387072029BF97009A
:107910000000E78040A2A285528597000000E78022
:1079200080A11DBB9305610017E5FF1F03452521BD
:1079300017E4FF1F0344B42097000000E78040B025
:1079400093057100228597000000E78060AF3C003E
:1079500017E7FF1F232AF74C834761002304F10038
:1079600083477100A304F100894717E7FF1F230D28
:10797000F7408357810017E7FF1F2311F71C0944C5
:10798000A1AC154793F64700B336D00093F78703B1
:10799000850685C32146638BC7066146638AC70691
:1079A000130680026388C706130680036393C7002B
:1079B000914717E6FF1F2301D63E97E6FF1FA38DD1
:1079C000F63C97E7FF1F238AE73C17E7FF1F0347B3
:1079D00027179376070497E7FF1F83C777168DEE67
:1079E0001377770C93067008630CD7021377F707A9
:1079F0008D46631ED70AB307F040B7955B0093F737
:107A0000F70F938505D881A81947ADBF854755B7AE
:107A1000894745B78D4771BF930670086311D70238
:107A20001307300FB7150E006389E7021307900D97
:107A3000B7B504006383E7021307700845BF9306D8
:107A4000800C6311D702B307F040B775460093F777
:107A5000F70F938585CDB3D5F50297E7FF1F23ABCD
:107A6000B732F9B39306900C631AD700B307F0400E
:107A7000916593F7F70F9385C566F1BF9306A00C48
:107A8000631BD700B307F040B7153D0093F7F70F1E
:107A900093850590C9B79306B00CE319D7F4B307E3
:107AA000F040916593F7F70F938595D06DB78946B0
:107AB000631BD700B307F040B7750B0093F7F70FC0
:107AC0009385051B49BF8546631AD700B307F0406D
:107AD000DD6593F7F70F938565E3B5BF09EBB30752
:107AE000F0408D6593F7F70F938575DCADB7F165C1
:107AF000938505209DB783472A00C18B99C7854789
:107B000017E7FF1F2305F72881BE97E7FF1F238094
:107B1000072899B6854717E7FF1FA300F7282DBE52
:107B20003C0017E7FF1F2321F730094793070003A5
:107B30002314F10097E6FF1F2388E6242DBD639AE6
:107B40000758A94763ECB74417A70100130707EBD1
:107B50008A05BA959C41BA97828717E4FF1F0344B0
:107B600014FE094A630C440F636C8A088547630955
:107B7000F40A9307F00F17E7FF1F0347E72063F6A8
:107B8000E70017E7FF1F2301F72017EAFF1F034A4B
:107B9000AA1F930700041374FA0F63F44701130438
:107BA000000497E7FF1F9387272883AA07002286F0
:107BB00017E5FF1F130585F8D685330A8A40A29A78
:107BC00097700100E78080F597E7FF1F238E471B22
:107BD00097E7FF1F23AA572597E7FF1F83C7D71AE9
:107BE0001547639AE762B7E700E03707400023A034
:107BF000E71801000100B7860040238086028DA5AA
:107C00008D47630CF40A9947E315F4F697A7010032
:107C1000938747E517E7FF1F2328F720A947A1BF50
:107C200017E7FF1F0347672197E7FF1F9387C717D2
:107C3000494697A501009385E5EB6306870097A564
:107C40000100938525E73E8597700100E78000EDF0
:107C500017E7FF1F232AA71CC94731BF97E6FF1F5D
:107C600083C6A61D054797E7FF1F9387E713639415
:107C7000E6023E851306700297A50100938505E58F
:107C800097700100E78080E917E7FF1F232EA718F0
:107C900093077002CDB53E851306300497A5010009
:107CA000938505DD97700100E78040E717E7FF1F28
:107CB000232CA716930730047DBD97E5FF1F83C5CE
:107CC00005E817A50100130565EC97700100E78032
:107CD00040F0854A17EBFF1F034B2B1697E5FF1F5C
:107CE00083C5E5E517A50100130545EA63185B0B9D
:107CF00097700100E780E0ED97E7FF1F83C727E457
:107D0000B5CBE368F4E617A401001304E4E2638C46
:107D1000670117A401001304A4E26386470117A4B6
:107D20000100130464E3228597700100E780A0122C
:107D30001375F50F93071500860717E7FF1F230537
:107D4000F7068D4717E7FF1FA300F70697E7FF1F0A
:107D5000938787050147BE861376F70F890763650A
:107D6000A60297E7FF1F23A1D70C97E7FF1F83C742
:107D7000A70311B597A70100938707D517E7FF1F42
:107D80002324F70A9147C5BB3306E40003460600E7
:107D9000A380070005072380C7007DBF97700100FF
:107DA000E78020E397E7FF1F83C767D9E1D7E36246
:107DB000F4DC17A40100130424D5638C570117A425
:107DC00001001304E4D46386470117A401001304DF
:107DD000A4D5228597700100E780E0071375F50FA1
:107DE00093071500860717E7FF1F230FF7FA8D4744
:107DF00017E7FF1FA30AF7FA97E7FF1F9387C7FA52
:107E00000147BE861376F70F8907E37CA6F4330695
:107E1000E40003460600A380070005072380C7008F
:107E2000D5B797E5FF1F83C585D117A501001305B9
:107E3000A5D697700100E780C0D997E7FF1F83C7D9
:107E400077F693E7470017E7FF1FA30DF7F4834783
:107E50002A0017E7FF1FA305F7F46FF0EFFF17A540
:107E600001001305A5D497700100E78060EE97E745
:107E7000FF1F9387E7F283C7070017E7FF1F230F52
:107E8000F7CA17E4FF1F034424F033348000A9B37A
:107E900017A501001305C5D297700100E78040EBDC
:107EA00097E7FF1F83C717F093E7070117E7FF1F47
:107EB000A30AF7EE83472A0017E7FF1F2302F7EE16
:107EC0006FF08FF917A501001305C5D09770010059
:107ED000E78000E803470A007D8B51EFB787004039
:107EE00003C767021377C70B136727002383E702D3
:107EF00003C7A7021377C70B136727002385E70281
:107F000003C7E7021377C70B136727002387E7022E
:107F100003C727031377C70B136727002389E702DB
:107F2000854717E7FF1F230BF7CC17E7FF1F230930
:107F3000F7D817E7FF1F2307F7E417E7FF1F23040E
:107F4000F7E497E7FF1FA38B07CA97E7FF1FA389F3
:107F500007D697E7FF1FA38707E297E7FF1FA384D2
:107F600007E297E7FF1FA38B07E297E7FF1FA386B0
:107F700007EC6FF06FEE89476312F70297E7FF1F78
:107F800083C707BC9146638CD70863E0F604638E11
:107F9000E70C6369F70A05476380E70EFD5717E7AB
:107FA000FF1FA303F7DE37074000B7E700E023A079
:107FB000E71801000100B78600401306F0FC23819A
:107FC000C60223A0E7106FF08FD613072008638244
:107FD000E7086362F70213071008E391E7FC3787AD
:107FE00000408347670293F7C70B93E727002303FB
:107FF000F7026FF06FE6130730086389E702130793
:108000004008E39DE7F8378700408347270393F74D
:10801000C70B93E727002309F7026FF0EFE33787D9
:1080200000408347270393F73707F5B737870040AA
:108030008347E70293F7C70B93E727002307F7026D
:108040006FF08FE1378700408347E70293F73707E8
:10805000F5B7378700408347A70293F7C70B93E72D
:1080600027002305F7026FF02FDF37870040834793
:10807000A70293F73707F5B73787004083476702B2
:1080800093F73707ADB717A501001305A5B597708E
:108090000100E780E0CB97E7FF1F238107AAD5B354
:1080A00017A50100130505B597700100E78040CAC8
:1080B00097E7FF1F239407A897E7FF1F9387C7CC75
:1080C00003C40700894763F3870009441374F40F5E
:1080D00021B613070002E393E7EC6399090A638F63
:1080E000F500930720026381F50817A50100130529
:1080F000E5B397700100E780C0AD4DB517A501004D
:10810000130505B097700100E78080C4014417ABE8
:108110000100130B2BB0A14AB3078A0083C50700E7
:108120005A85050497700100E780A0AAE31654FF62
:1081300017950100130505E297700100E78040C123
:1081400017E4FF1F0344C49F11E497E7FF1FA389AF
:10815000079C59B48947E313F4E4854717E7FF1FE9
:10816000A300F79C6FF04FCF17E6FF1F0346369D25
:1081700097E5FF1F83C5A59C17A50100130505AA58
:1081800097700100E780E0A46FF00FCD638FF504D6
:1081900093071002E39BF5F497E5FF1F83C5459A0B
:1081A00017A50100130585A997700100E78060A25B
:1081B00097E7FF1F23AA47C797E7FF1F938787BD4E
:1081C000944383D7470017E7FF1F034707BD17E610
:1081D000FF1F2325D6961D4497E6FF1F2392F69690
:1081E00097E7FF1F238FE794C5BA97E5FF1F83C565
:1081F000259517A501001305E5A597700100E780F7
:10820000409D97E7FF1FA38D079097E7FF1F2397D8
:1082100007926FF0CFF62547E387E79C19476391F4
:10822000E702B786004023808602B7E700E0370701
:10823000400023A0E71801000100130600FC41B331
:108240001307100A6391E702B78600402380860275
:10825000B7E700E03707400023A0E718010001005E
:10826000130680FCA9BB1307A009E38FE7FC1307E3
:10827000400AE38BE7FC13072002E386E7960547F5
:10828000E383E796B7E700E03707400023A0E7184D
:10829000E391099601000100B78600402380860221
:1082A000130620FC29BB17E7FF1F0347F7AD630840
:1082B000F71E63E7E7029547630EF70E99476308D9
:1082C000F704B786004023800602B7E700E03707CF
:1082D000400023A0E718010001001306A0FCC5B16F
:1082E0009307F005630AF700930750096306F70048
:1082F00093071002E317F7FCB7E700E037074000E9
:1083000023A0E71801000100B786004051BF97E99C
:10831000FF1F83C969A793070004CE8A63F437015E
:10832000930A000497E7FF1F938707B003AA07008B
:1083300013F4FA0F2286D28517E5FF1F1305058077
:1083400097600100E780807DB3878940529417E7EA
:10835000FF1F230BF7A297E7FF1F23A787AC638EAE
:108360000902B787004023805703B7E600E03706CD
:10837000400023A0C6180100010003C727021347CD
:1083800007042381E70203C727021377C70F23815E
:10839000E70223A0C6106FF08F99B78600402380B4
:1083A0000602B7E700E03707400023A0E718010006
:1083B0000100FDB5378700408347370097E6FF1F70
:1083C00083C6169E93F70708D58FA301F700B7065B
:1083D0004000B7E700E023A0D71801000100130612
:1083E000A0FC2301C70223A0D7106FF04F9497E79A
:1083F000FF1F9387E7A3A69783C7070093F7F70F9D
:10840000D9CF97E7FF1F83C747A3D1EB17E7FF1F1C
:1084100003479797930700026313F70897D7FF1F47
:108420009387C77103AB070097DAFF1F83CA4A71AE
:1084300017DAFF1F034ADA7097D9FF1F83C96970E3
:10844000D2875687CE865A8697D5FF1F83C5556D2E
:1084500017A501001305858197600100E78060770B
:1084600097E7FF1F23A8679397E7FF1F238657937C
:1084700097E7FF1FA382479397E7FF1F238F37914B
:1084800097D7FF1F238E8768B7E700E037074000C4
:1084900023A0E71801000100B7860040D1B3B7E779
:1084A00000E03707400023A0E71801000100B7866D
:1084B000004025B529472381E70209472383E702C6
:1084C0002385E7022387E7022389E7026FF08F8A7B
:1084D00003C76700118B6302078C83C75700918B1A
:1084E000B5CF17E7FF1F0347479585476313F70687
:1084F00097E7FF1FA383E78A97D7FF1F23800770A3
:1085000097D7FF1F238E077A97E7FF1F238C0786D5
:1085100097E7FF1F2389078697D7FF1FA380076E62
:1085200097D7FF1FA38E077897E7FF1FA38C0784B9
:1085300097E7FF1FA389078497E7FF1FA38007869C
:1085400097E7FF1FA38B078EB787004011476FF097
:108550008F8417D7FF1F2305F75C79BF854717D78F
:10856000FF1F230DF76817D7FF1F230BF77417E7BB
:10857000FF1F2309F78017E7FF1F2306F78069BF56
:10858000854717D7FF1F230BF76617D7FF1F230950
:10859000F77217D7FF1F2307F77E17D7FF1F230494
:1085A000F77E17D7FF1FA30B076417D7FF1FA30979
:1085B000077017D7FF1FA307077C97D7FF1FA38458
:1085C000077C8280411106C697000000E78080FB8F
:1085D000B787004023800700130740FC2386E7008D
:1085E0001307C004A386E70017D7FF1F130707551B
:1085F0002398E70017D7FF1F13074758239AE70070
:1086000017D7FF1F1307C763239CE70017D7FF1F68
:108610001307476F239EE70029472381E702094795
:108620002383E7022385E7022387E7022389E70202
:10863000A3810700930600F8A380D7009306900259
:108640002380D700FD562383D7002381E700B70698
:10865000400037E700E02320D71003C71700136757
:108660001700A380E700B24097D7FF1F239A077235
:1086700041018280411106C697000000E78080F02A
:10868000B787004023800700130700FC2386E7001C
:108690003147A386E70017D7FF1F1307274A239800
:1086A000E70017D7FF1F1307674D239AE70017D777
:1086B000FF1F1307E758239CE70029472381E702A0
:1086C00009472383E7022385E702A3810700930676
:1086D00000F8A380D700930690022380D700FD56B0
:1086E0002383D7002381E700B706400037E700E087
:1086F0002320D71003C7170013671700A380E700D4
:10870000B24097D7FF1F239D076841018280F16720
:108710009387072017D7FF1F232EF766854717D7A4
:10872000FF1F231BF766A14717D7FF1F2307F76615
:1087300097D7FF1FA383076697D7FF1F238007667E
:1087400097D7FF1FA38E073C97D7FF1F238A073CAD
:10875000814717D5FF1F1305E53CFD5517D6FF1FB1
:108760001306063D2947B306F5002380B600B3067D
:10877000F600238006008507E397E7FE97D7FF1FE3
:108780002386076A97D7FF1FA382076A97D7FF1F21
:10879000238F076897D7FF1FA389075E97D7FF1F0F
:1087A000A387075E97D7FF1F2382075E97D7FF1F18
:1087B000238D075C97D7FF1F238C075C97D7FF1F7C
:1087C000A386075C97D7FF1F2383075C97D7FF1FFC
:1087D000A38F0764828017D7FF1F0347076685476B
:1087E0006316F70017030000670003E91703000092
:1087F000670083DD411122C406C617D7FF1F034758
:10880000C76385472E8613F4F50FAA856317F7040F
:1088100017D5FF1F1305C54697600100E78000309C
:1088200097D7FF1F238E0748B7870040238487020E
:10883000B7E600E03706400023A0C618010001009B
:1088400003C7A7021377C70F2385E702B24022446C
:1088500023A0C61001454101828017D5FF1F1305D3
:10886000E53597600100E780602B97D7FF1F2387CE
:108870000738B787004023828702B7E600E0370653
:10888000400023A0C6180100010003C76702137748
:10889000C70F2383E7025DBF411106C697000000A2
:1088A000E78020E7B2404101170300006700E3F2D0
:1088B00017D5FF1F0345C54E3335A000828041C93F
:1088C000D9C597D7FF1F83C7A74DD1C3011122CCAC
:1088D0004AC84EC656C25AC006CE26CA52C42E89AF
:1088E000AA890144930A0004371B03006377240319
:1088F000B3078940C207C183BE8463F4FA009304BE
:108900000004C204C180130A1BD497D7FF1F83C77A
:10891000E72E9DE37D1A631C0A00F2406244D244B4
:108920004249B249224A924A024B0561828097F03D
:10893000FFFFE78040B8D1BF338589002694A68524
:10894000420497000000E78020EB418045B7828019
:10895000411106C622C429C12E8495C997D7FF1F8D
:1089600083C7074495CB97D7FF1F83C727298DC798
:1089700013070004AE876374B700930700041394D1
:1089800007014180A28597000000E780E0E622858C
:10899000B2402244410182800144D5BF411106C644
:1089A00097F0FFFFE78020B197D7FF1F83C71725F8
:1089B000A1CB97D5FF1F83C5852489C917D5FF1F74
:1089C0001305052497E0FFFFE780202797D7FF1FB7
:1089D000A386072297D7FF1F2382073C37E700E0D3
:1089E000B70640002320D718010001003786004059
:1089F0008347660293F7370F2303F6022320D7102D
:108A0000B2404101828097D7FF1F9387A746184243
:108A10009C4383D645000345070083C5C700035622
:108A200046006396A50083D5E700638DD50201114A
:108A300006CE2386A7002397D700B705CF00DC4BCF
:108A40009385757D05077D162EC2230001003AC46B
:108A50002316C1002317D10099C30A858297F240DB
:108A6000056182808280DC4DDC4B81CFB7E704005A
:108A7000904503A38705914517D5FF1F0345C53FC3
:108A8000028382806D713C083EC6B707E500232251
:108A900091103EC8AA843C083285232611103ECA94
:108AA00023248110232021112E8997300000E78094
:108AB000A05C2A84979501009385C51E1785010047
:108AC000130585E297600100E780A010A285179545
:108AD00001001305A52D97600100E780800F29454F
:108AE00097600100E780C013B705CB009385757DC3
:108AF000680097100000E780C065A2856800973085
:108B00000000E780C049014781467000CA8526857C
:108B100097200000E780408905CD2A8497950100C1
:108B20009385451817850100130505DC9760010042
:108B3000E780200AA285179501001305E5279760B5
:108B40000100E7800009294597600100E780400D9A
:108B50008320C110032481108324411003290110B4
:108B60005161828097D7FF1F9387C73018429C437B
:108B7000797122D406D60348070083C807012A84E6
:108B800083D64500035546006396080183D8270124
:108B9000638DD8022388070105072399D70037087A
:108BA000CC00DC4B1308787D3ACC1307F5FF42CAA2
:108BB00023080100231EE100231FD10099C70808E4
:108BC00032C62EC482973246A24522859700000005
:108BD000E78080EBB2502254456182806D713C0881
:108BE0003EC0B707E5003EC23C083EC42326111034
:108BF0002324811023229110231701002318010040
:108C000023190100231A0100231B010097A7FF1F4E
:108C100083D7C77C99E3C167FD172316F10097A797
:108C2000FF1F83D7C77B91EB97D7FF1F93878724BD
:108C30009C439C43DC4783D7070017A4FF1F130402
:108C4000E479584C2317F10083574400484B23180C
:108C5000F10031E1979501009385C50B178501005F
:108C6000130585C897600100E780A0F617950100FD
:108C70001305850B97600100E780A0F529459760F3
:108C80000100E780E0F98320C110032481108324D0
:108C900041105161828097A7FF1F83C7977489EBAA
:108CA000B7E70400BC5782975C4C23AA0700E1BFDA
:108CB000FD1797A6FF1FA386F67203560701834789
:108CC00004014C470A85230BF10097300000E78030
:108CD000202A97D7FF1F9387E7199C4301478146B6
:108CE00088430A866C0097100000E780E06BAA8436
:108CF00029C1979501009385E501178501001305AA
:108D0000A5BE97600100E780C0ECA685179501001D
:108D10001305450297600100E780A0EB29459760A5
:108D20000100E780E0EF584CB7E70400BC57484B20
:108D30009DBF97A7FF1F83C7D76AF5D7B7E7040082
:108D4000BC4F1044854517D5FF1F0345E512829798
:108D50001DBF5C4EDC4BB9CFB1CD411122C417858C
:108D60000100130565B82E84979501009385C5F819
:108D700006C697600100E780C0E5A285179501004F
:108D8000130505FE97600100E780A0E42945976080
:108D90000100E780E0E8B7E704002244B24003A303
:108DA000870517D5FF1F0345250D1306400691457E
:108DB000410102838280411122C417A4FF1F1304C2
:108DC000A45F1C4C06C689C7DC4399C34C488297F4
:108DD000584CB7E70400BC57484B82975C4CB240F4
:108DE000224423AA07004101828017A7FF1F13070F
:108DF000A75E834707009306F00B850793F7F70FED
:108E000063E9F60097A6FF1F2388F65C0345070079
:108E10008280930700F8FDB78357450063860710EB
:108E200001114AC817A9FF1F1309495B52C4032A3D
:108E3000C90106CE22CC03274A0126CA4EC656C215
:108E4000F15735E31307D00DFD57636EC704B7E93B
:108E5000040083A709072A8413058600420541817F
:108E6000B284AE8A8297232AAA000325C9015C49ED
:108E7000A9E797950100938525E61785010013055D
:108E8000A5A697600100E780C0D4179501001305DF
:108E900065F597600100E780C0D329459760010020
:108EA000E78000D8DD57F2406244D2444249B249DB
:108EB000224A924A3E850561828093874400B70525
:108EC000CF002319F5009385757D310597100000BB
:108ED000E78020280325C9018345640031059730C8
:108EE0000000E780C00B0325C9012686D685310521
:108EF00097300000E780C0077146A2854A859760D9
:108F00000100E780A0C1504419CA83A7890585459F
:108F100017D5FF1F034545F68297814769B797002C
:108F20000000E780E0CBD5BFFD573E858280411130
:108F300026C297A4FF1F9384644AD84C22C437E406
:108F400004003C54484B06C68297DC4C0323C405FE
:108F50002244B240924423AA070017D5FF1F0345BD
:108F6000A5F1854541010283411126C297D4FF1F17
:108F7000938444F09C4006C622C44AC0D5C3DC4357
:108F8000C5C35CC12300B5002A8497950100938571
:108F9000E5CF178501001305259597600100E7804F
:108FA00040C3294597600100E78080C79C4023A407
:108FB000070023A2070097A7FF1F9387E73FDC4F17
:108FC000DC4B91C7295597000000E78000DF97A789
:108FD000FF1F9387A740DC4FDC4B89C79700000039
:108FE000E78020F537E904008327C905894517D5AF
:108FF000FF1F034565E882978327C905914517D56B
:10900000FF1F034565E782979C4003A3470163095F
:10901000030022852244B240924402494101028366
:10902000B2402244924402494101828001113285BA
:1090300006CE22CC26CA2E8497300000E780C003DB
:10904000AA84979501009385A5C71785010013058C
:10905000A58997600100E780C0B703078400035625
:10906000640083554400A68617950100130545D179
:1090700097600100E780E0B5294597600100E7802F
:1090800020BA97A7FF1F83C78733639D97000145C9
:1090900097000000E78060D281450A8597000000B4
:1090A000E780C0ECF2406244D244056182806D7179
:1090B00023248110232611102322911093F74500B9
:1090C0002E84638707143C083EC0B707E5003EC204
:1090D0003C083EC423170100231801002319010096
:1090E000231A0100231B010097A7FF1F83D7C72C5A
:1090F00099E3C167FD172316F10097A7FF1F83D7D8
:10910000C72B91EB97D7FF1F9387C7D69C439C43F0
:10911000DC4783D7070017A7FF1F1307E72923178B
:10912000F100544F835747002318F100DC4AA1E7B0
:1091300097950100938505BD177501001305C57A44
:1091400097600100E780E0A8179501001305C5BDF1
:1091500097600100E780E0A7294597600100E7805C
:1091600020AC134544008320C110032481108324C4
:1091700041105161828097A7FF1F83C7572425554F
:10918000D9C3FD1717A6FF1FA30BF62203D60601AE
:1091900083470701CC460A85230BF1009730000076
:1091A000E78000DD97D7FF1F9387C7CC9C4317A7A5
:1091B000FF1F13076720979601009386E6B988433F
:1091C0000A866C0097100000E780001EAA8451D91F
:1091D00097950100938505B3177501001305C570B8
:1091E00097600100E780E09EA685179501001305B2
:1091F00065B497600100E780C09D29459760010034
:10920000E78000A2268597000000E78000BB91BFA1
:1092100093F725009DC7B7E70400BC474146814549
:1092200028088297255597000000E78000B9280894
:109230009305F00F97000000E78040D3134524000A
:109240001DB793F71500014599DF97000000E780EF
:1092500020991345140001BF5C4D411106C688C317
:1092600017D7FF1F2328F7C0B7E7040083A7070815
:10927000170500001305E5E38297B24097D7FF1F5B
:10928000238CA7BE01454101828001119307700F15
:109290002316F10006CE97D7FF1F83C777BF8DE750
:1092A000B7E7040083A7870D17A6FF1F034606161E
:1092B0006C0017D5FF1F0355E5BD82973335A0001D
:1092C00097D7FF1FA386A7BCF2400561828041119A
:1092D0009397050122C406C626C2C1872E8463D493
:1092E0000702B7E40400FC5417A5FF1F034505124D
:1092F000829719C1BC5482972165218DB2402244C6
:1093000092444101828093F715008DC7B7E70400AE
:1093100083A7471A17A6FF1F1306460E97D5FF1FF0
:10932000938545B617A5FF1F0345450E8297134544
:109330001400E9B793F7250099CFB7E70400BC4FB5
:1093400013060064894517A5FF1F0345250C829766
:109350001345240065B793F785009DC7B7E7040060
:1093600003A8871A1307401F97A7FF1F83C7070A81
:10937000814613064006994517D5FF1F035585B151
:109380000298134584009DBF93F745000145BDD762
:10939000B7E4040083A7041817D5FF1F035585AF52
:1093A0008297BC4C13060064914517A5FF1F034527
:1093B000E50582971345440091B797D7FF1F83D7E0
:1093C00067AD6398A70217D7FF1F2316B7AC17D74F
:1093D000FF1F2313C7AC17D7FF1F2310D7AC2E8650
:1093E00017950100130505B7BE85175301006700E7
:1093F000437E17950100130565B7176301006700E9
:10940000239503574500011106CE22CC97D7FF1FA5
:1094100083D747A817950100130545B56310F706D4
:10942000C167F91717D7FF1F2326F7A637E40400F3
:1094300097D7FF1F23A207A67C4C894517A5FF1FBE
:109440000345C5FC82977C4C914517A5FF1F03453A
:10945000E5FB829797B7FF1F83C7570685CB8547E4
:10946000A307F100832744171306F1008545130570
:109470005030829717950100130585A3976001006E
:10948000E780008DF24062440561828097C7FF1F2C
:1094900083C7074317950100130545A6E5F38547E4
:1094A000A307F100832744171306F1008545130530
:1094B00050308297179501001305C5A1C1B77D15DE
:1094C000954763E0A71C179701001307279B0A0520
:1094D0003A951C41011122CC06CE26CABA972E8499
:1094E0008287179501001305E5A897600100E780C2
:1094F00020861DAA03C7250099476311F7022E8510
:1095000097000000E78020F0834564001795010074
:10951000130545A797500100E780A06B97B7FF1F81
:10952000238E07F817950100130585A77DBF03C794
:10953000250095476319F702C16717D7FF1F035727
:109540006795F91703D5A5006309F702B7E704008B
:1095500083A7C717829717950100130565A5975034
:109560000100E780E07E854717B7FF1F2308F7F467
:1095700017950100130545A68DBF97D7FF1F239BA5
:10958000A79083D7E500B7E40400096617D7FF1F4B
:109590002313F79083D705011306069017A5FF1F25
:1095A0000345C5E617D7FF1F2318F78E83D725017C
:1095B000A14517D7FF1F2312F78EBC4C8297BC4CD6
:1095C00013060064914517A5FF1F034525E4829704
:1095D0000356E4008355A400179501001305859EEA
:1095E00097500100E780E05EBDBF179501001305AD
:1095F000659FE5BD83C525009147639CF5028547BE
:10960000179501001305859FA307F10097500100EE
:10961000E7800074B7E7040083A747171306F1003B
:109620008545130550308297F2406244D24405616B
:10963000828099476392F502228597000000E780B7
:1096400080DC83456400179501001305A5939750AE
:109650000100E7800058C9BF9547639FF500834725
:1096600014001795010013056599E39007E8179515
:1096700001001305659A95BD179501001305459ADC
:10968000F9B782806D7123248110232611102322C3
:109690009110328401CD8947630AF5028320C110FD
:1096A00003248110832441105161828017950100A9
:1096B0001305C597AE8497500100E7806069A285C5
:1096C000268597C0FFFFE780C0E9C9BFB7E7040060
:1096D000FC4728008297179501001305E5959750E0
:1096E0000100E780E0668347810039C41307000B5F
:1096F0006380E7021387A7051377F70F8D4663EDA5
:10970000E602A285280097C0FFFFE780A05879B73E
:109710008547E3F587F88345910017750100130528
:10972000E551B335B00097B7FF1F238BB7C09750F3
:109730000100E780004A9DB703479100A207D98F37
:1097400035671307D7556385E7086368F7022D6708
:109750001307B7556387E70631671307C755638A51
:10976000E70429671307A7556394E702A285280039
:1097700097C0FFFFE780407D15B739679306E7651F
:10978000638DD70663E9F6001307E7556380E706A4
:10979000A28528003DB73D679306F7556386D70637
:1097A0001307F766E396E7FE97D0FFFFE780809701
:1097B000F5B50146A285280097C0FFFFE780A07499
:1097C000F1BDA285280097C0FFFFE780E073F9B5DF
:1097D0008947E3F587EC9305E4FFC205C1811305D2
:1097E000A10097A0FFFFE780808B4DBDA2852800D8
:1097F00097C0FFFFE780007855B5A285280097D075
:10980000FFFFE780C08259BD97D0FFFFE780408B04
:1098100071B5411122C417A4FF1F130464C0AA86A6
:1098200017860100130606672285C14506C69750B4
:109830000100E78020530357440097A7FF1F938739
:1098400027BF2393E700035764002394E700B24047
:10985000224441018280011106CE22CC97000000F3
:10986000E78060FB37E404008327841417A6FF1FFA
:10987000130606BBD54501458297832784179305B8
:10988000F1001305503082978347F100A1C7A30769
:109890000100832744171306F10085451305503056
:1098A00082978327441717A6FF1F130666B8CD4576
:1098B0001305703082978547A307F100832744176B
:1098C0001306F1008545130550308297F24062443B
:1098D000056182808327441717A6FF1F130646B52C
:1098E000CD4513057030D5B7130101DE232C81203F
:1098F00037E4040083270408232E1120232A912013
:109900002328212123263121170500001305659CFA
:10991000829717A9FF1F130969AF99478544230050
:10992000A9002318F100978501009385A55F93078F
:10993000400617750100130525FB2314F1102304BD
:10994000910097C9FF1F9389090097500100E78094
:10995000402883D5090017850100130565549750E9
:109960000100E7800027294597500100E780402B40
:1099700003D50900856997000000E780C0E98327C7
:1099800044173000854513055030829783274417CC
:1099900017A6FF1F1306C6A9CD4513057030829781
:1099A0008327441717A6FF1F130686A6B545130580
:1099B00060308297832744171008894513051031BA
:1099C00082978327441730028945130520318297F7
:1099D00083274415938509C80D458297832744152D
:1099E000938509C811458297A30191002302910034
:1099F00023049100232401102308010083278416E7
:109A00003002914513057040829783278416130610
:109A10003100854513050040829783278416500046
:109A200085451305104082978327841610088545C5
:109A3000130520408297832784163000854513053F
:109A400050408297832704157D55829783274413BE
:109A50007D5582977D5597A0FFFFE78000AE832755
:109A6000440C829797A0FFFFE780408A83278414E5
:109A700017A6FF1F1306C69AD54501458297894749
:109A80001306700F814508082302F1009780FFFF3D
:109A9000E780E0658D471306700F81452802230893
:109AA000F1009780FFFFE780806491472304F11065
:109AB000977701009387C7D4984383C747003AC478
:109AC0002306F10097C0FFFFE780806C50008545BA
:109AD000054597A0FFFFE78060AD10089305700F64
:109AE000094597A0FFFFE78060AC30029305700F37
:109AF0000D4597A0FFFFE78060AB3000954511450D
:109B000097A0FFFFE78080AAC16717C7FF1F130751
:109B10006738F9171CC32322070017A5FF1F130579
:109B2000A58E97A0FFFFE78040A78327C41D17C518
:109B3000FF1F1305A53482973C480345090085455E
:109B400082978320C1210324812183244121032979
:109B500001218329C120130101228280C16717C816
:109B6000FF1F03582833F9176301F8083DCDB5CD21
:109B7000011126CAB7E4040083A7841222CC2E86E2
:109B80002315B10006CE2A8401478146ED45428562
:109B900082972AC611ED178501001305A539975044
:109BA0000100E780E01AF2406244D24405618280FD
:109BB000FC440356A100A28582972C0017C5FF1F05
:109BC0000355452D97A0FFFFE780E0A969DD1785C4
:109BD00001001305653797500100E780601783A7E0
:109BE000C412ED45280082977DBF8280011106CE08
:109BF00022CC2DC9854717A7FF1FA300F78297A77F
:109C0000FF1F238D078037E4040083278417930503
:109C1000F1001305503082978347F100A9CBA307C9
:109C20000100832744171306F100854513055030C2
:109C30008297832744171796FF1F1306667DB54545
:109C40001305603082978547A307F10083274417E7
:109C50001306F1008545130550308297F2406244A7
:109C6000056182809797FF1FA389077A49BF8327E1
:109C700044171796FF1F1306A679B54513056030E4
:109C8000E9BFC16717C5FF1F0355C520F917630753
:109C9000F500B7E7040003A3C71702838280011110
:109CA0008547A307010017C7FF1F2303F71EB7E768
:109CB000040083A7471706CE1306F1008545130558
:109CC00050308297F240056182801783FFFFE702E0
:109CD000633D2A8408452E89B28919C900C19715A8
:109CE00000009385A586610597300100E78080011B
:109CF00081447D5A97100000E780E03963C7A404CF
:109D0000814497100000E780003A63C8A40497C715
:109D1000FF1F9387A7189C43DC47B307F94091873F
:109D20002302F400638309048327C900B307F440C6
:109D30009587A302F4001C4C89C79C4799C32285D0
:109D400082971783FFFF670023395C441397140041
:109D50008504BA972390470171BF1C4813971400DC
:109D60008504BA972390070069BF832789000547B8
:109D7000B307F4409587A302F40083570400638E71
:109D8000E7028DC309476384E7040D47E395E7FACB
:109D9000978701009387077D1CCC978701009387E5
:109DA000677D11A897870100938747431CCC97874D
:109DB00001009387A7435CC8BDBF978701009387C5
:109DC000E72E1CCC978701009387472FEDB7978725
:109DD00001009387E77D1CCC978701009387477E1E
:109DE000D9BF95E51783FFFFE702632D00461844AE
:109DF0008347940075839D8B6317F70097100000CD
:109E0000E78060B448C41783FFFF6700832D82801A
:109E10001783FFFFE702032913893500C164420954
:109E20004111AA890144F11413590901054A2EC6AA
:109E300097100000E7802026B2456348A400014542
:109E400041011783FFFF6700232983A70900131728
:109E50001400BA9783D707006388B700639497000C
:109E600063742A010504E1B70545D9BF1783FFFFD5
:109E7000E7026322AA892E89328BB6843A8ABE8A87
:109E800097A00000E78020FB71C92685972000007D
:109E9000E78020098D4763E7A7007D551783FFFF03
:109EA0006700E32283DB440097100000E780A024D2
:109EB0002A8497100000E7804025930774003144FE
:109EC0003305850263CDA70297100000E780A0222A
:109ED00097100000E78020222A8497100000E78076
:109EE000C0229307740031443305850263C3A7047D
:109EF00097100000E78020209307450029A89710BD
:109F00000000E7808020330585021307F0179307D0
:109F1000C017E35FA7FA2D55E3C277F963040B027C
:109F2000D6865286A6854A8597200100E78020BA0A
:109F3000B5B797100000E780401D330585029307F1
:109F4000C5FFD1BF832749001385C90083D52700EA
:109F500097000000E78000EC61F581B769553DBFCF
:109F600097C7FF1F239EA7F297C7FF1F938707F38B
:109F7000904381470C463307F500420741836393C2
:109F8000B70082805446139847008507C2962390F5
:109F9000E600D5B797C7FF1F938747F09C4303C5DB
:109FA0008700828017C5FF1F035585EF82801783C6
:109FB000FFFFE702C310C1671387D7FF630BE502FA
:109FC000636AA700F1176300F50201451783FFFFDD
:109FD000670023111387E7FF6302E502FD171D8D5C
:109FE00013351500E5B797500000E780C0267D15B2
:109FF000C5BF97500000E78040FBD5BF97500000D9
:10A00000E78060F9EDB71783FFFFE702430B4111CB
:10A01000AA8401442EC697100000E780C008B2450C
:10A020006348A400014541011783FFFF6700630BEC
:10A030009C48131514003E9583570500E385B7FE31
:10A040000504C9BF03485500814693F7F60F63E541
:10A05000070181473E858280584593975600BA97FD
:10A0600003D727006316B70003D70700E304C7FE32
:10A070008506E1BF8346450001479377F70F63E408
:10A08000D700814711A81C45131657000507B29742
:10A0900003D60700E313B6FE3E8582801783FFFFD9
:10A0A000E702430093170501C18797CAFF1F938AF0
:10A0B000EADE635BF00883A70A00C0479C470357AA
:10A0C0000400198D420541816368F5000144228531
:10A0D0001783FFFF6700430012052A94CDBFDC47BA
:10A0E00013944900014A3E94834744006341FA02B5
:10A0F000014A834754006349FA028509C20993D98A
:10A10000090183A70A009847E3EBE9FCC1B71C44A7
:10A1100013195A00A6853E994A8597000000E780EA
:10A12000C0EE05E1050AC9B75C4413195A00A685BB
:10A130003E994A8597000000E78020ED19E1050A65
:10A140004DBFE30C09FA61B7AA8481495DBF17834B
:10A15000FFFFE702C3F61C452A8481E79307C50089
:10A160001CC51C44231204001CC09307F00F63EDB0
:10A17000B70093F5F50F228597200000E78020E2D5
:10A180001783FFFF6700E3F593940501C167C18062
:10A1900063F9F500A685228597200000E78040E559
:10A1A000C5B7C18193F5F50F228597200000E780A0
:10A1B00000DFA685228597200000E78040E0C9B730
:10A1C00097C7FF1F938787CD884382801C4599C717
:10A1D00097C7FF1F23A4A7CC014582807D558280AD
:10A1E00097C7FF1F938787CB98438347450048470E
:10A1F00092073E9582801783FFFFE70243EC61716F
:10A2000000451C183EC6B70780013EC81C183ECA50
:10A210008357440002CE02D002CC231EF1008347B4
:10A2200084002A8902D22301F1023C083ED402D6DE
:10A2300097000000E78000FB835705002316F1021A
:10A2400097500000E78060C42307A1025C400355DB
:10A250006400F18313F717008347F102520551811F
:10A26000F99BD98FA307F10297100100E780807551
:10A2700039CDAA840355050097A00000E78080BC73
:10A2800083D704002AD26800231CF10083D724005E
:10A29000231DF1001C4803D647008C439720000083
:10A2A000E78000CD8347B400CA86178601001306F5
:10A2B00066D98117A305F4006C00481097200100AF
:10A2C000E780E0805D611783FFFF670083E1215530
:10A2D000D5BF1C45B1CF03C5A700894613576500FC
:10A2E000630BD7028D46630ED70285466300D70203
:10A2F000130740063305E50203C7B700418B15CBB2
:10A3000083C7B700BD8B3355F54082801375F503C5
:10A310001307803EC5B709671375F5031307077167
:10A32000D1BF372709001375F5031307077CD9B789
:10A33000014582801783FFFFE70263D803A98500E8
:10A34000630C09048347B900AE8493F7070E85C3F5
:10A3500003459900930520030D810505B305B5025A
:10A360008844610597300100E780E0A935A02E857B
:10A3700097000000E78020F62A8419CD970000009E
:10A38000E780605C8325C900B307B54063FA8700A6
:10A390002E94B305A440E9F51783FFFF670063D44B
:10A3A00085457DBF1783FFFFE70263D12A8403D56C
:10A3B0000500011132C636C43AC22EC002CA02CC10
:10A3C00002CE97A00000E780E0A782452ACA228536
:10A3D0002ECC97000000E780E0E003570500231E25
:10A3E000E10097500000E78040AAA246324692471B
:10A3F000230FA10036874C08B286228501469700BC
:10A400000000E780E0A605611783FFFF670063CDCA
:10A410001783FFFFE702A3CA61711C183EC6B70786
:10A4200080013EC81C183ECA3C0800453ED4AA84A0
:10A4300002CC02CE02D002D202D697000000E78002
:10A4400060DA8357050035592316F1029750000052
:10A45000E780A0A32307A10209C48357440081EB2E
:10A4600021594A855D611783FFFF670083C7035544
:10A4700064005205518197100100E780A0542A8999
:10A4800065D18347B40093F7070E99C7130584017C
:10A4900097300100E780609983574400231EF10044
:10A4A000834784002301F1025C4003550900D983EE
:10A4B00013F7070883471102231CA10093F7F7073E
:10A4C000D98FA300F10283572900231DF1005C40BE
:10A4D000F18313F717008347F102F99BD98FA30784
:10A4E000F10297A00000E780E0952AD235D9834792
:10A4F00094006800139757008347B400FD8BD98FF1
:10A50000A305F4001C4803D647008C4397200000A5
:10A51000E78000A6A687178701001307A7B274007B
:10A5200005464C10268597000000E78060942A8934
:10A530000DD98347B400A685FD8BA305F4009700D1
:10A540000000E78060DF31BF1783FFFFE70223B71A
:10A55000832485FE2A844111268597000000E78028
:10A5600080D7834734FF93F7070E8DCB2AC6268505
:10A5700097000000E78060C809CD834734FFB245EB
:10A58000FD8BA309F4FE91C5228597300100E78079
:10A59000808741011783FFFF6700A3B47DD983271C
:10A5A000C4FF2685829775F5834734FF93F7070E1E
:10A5B00091C7228597300100E7802087032584FE1C
:10A5C00097000000E78000E5E9B71783FFFFE70287
:10A5D00003AC9C4141112A8903C7070089472E8497
:10A5E000935667006380F6040D466388C60493079C
:10A5F000F0076304F7022E8597200000E780C0A7CC
:10A60000AA848149C16B130C490097C7FF1F938728
:10A61000E7889C43984763E4E90441011783FFFFFF
:10A620006700A3AA03D745008547E3F8E7FE2E8518
:10A6300097200000E780A0A9E1B703D74500E3FE1B
:10A64000E7FC2E8597200000E78000A3AA842285DE
:10A6500097200000E78060A4C204C98C5DB7DC4786
:10A660000355A900139A49003E9A93170501C18723
:10A67000635DF00083570A006397A70263E77403E2
:10A680008327CA00034D5A002DA0A1672167A98F17
:10A690001307F7EFE374F7FE6397090097000000D4
:10A6A000E780209161FD85098DB783278A00034DDE
:10A6B0004A00835DA90003576900216A138BC70014
:10A6C0003AC6814A33CA4D01631E5D0197B7FF1F29
:10A6D0009387477D9C43E1DBA28662868145268580
:10A6E0008297D1B7A1679387F7EF930C4BFF63F283
:10A6F0004703B2455A8597F0FFFFE780A0710DC16F
:10A7000003278B00104709CE10436382C402310730
:10A71000D5BFEE85668597000000E780008F71F950
:10A7200093861A0093FAF60F130B0B0271BF835630
:10A7300044005C43E3E9F6F622853AC69710000030
:10A74000E780807DA1679387D7042A8A035D440050
:10A75000324763E897008347D90093E707F8A306D9
:10A76000F9001C4766852286E2858297C167084406
:10A77000FD17337AFA00529508C02312A40125B7B9
:10A7800097B7FF1F938787719843814715C3144775
:10A79000814763FFD500939745004C47BE9519C983
:10A7A00003C7550081476375E600DC451606B2977E
:10A7B0003E85828003C745008147E37BE6FE16069F
:10A7C0009C45F5B71783FFFFE702C38DAA892E8A40
:10A7D000814497BAFF1F938A6A6C83A70A0098473F
:10A7E00063E6E4001783FFFF6700038FDC471394E1
:10A7F000440001493E9413BB140083474400634B5B
:10A80000F900014913BB140083475400634FF9005A
:10A810008504E1B70844931759005287DA86014648
:10A82000A2853E9582990509C9BF484493175900EE
:10A830005287DA860546A2853E9582990509E9B7D1
:10A840001783FFFFE702A387814517F5FFFF130575
:10A85000054897B7FF1F2395076497000000E7801E
:10A86000A0F61783FFFF6700C38797B7FF1F938783
:10A87000E7629C4395C31783FFFFE702438481454A
:10A8800017F5FFFF1305A54497000000E780C0F30C
:10A890001783FFFF6700E38482801783FFFFE702CF
:10A8A000638037E404008327841241112315E100FB
:10A8B000AE893289368A3A8681460147ED45AA84B7
:10A8C00082972AC621C90356A100D285974001006C
:10A8D000E780C0248327C413CE8526858297058907
:10A8E00005C98327440D2314210101462C00268528
:10A8F00082972A8401C9B7E7040083A7C712ED45F0
:10A9000028008297228541011773FFFF6700C37CEF
:10A910004944D5B76554FDB75C41FD175CC18280E1
:10A920001773FFFFE702A379B7E70400FC5F829784
:10A9300095473305F50281450D811773FFFF6700C9
:10A94000437A1773FFFFE7028377B7E70400FC5FE2
:10A95000829795473305F5020D811773FFFF670056
:10A9600043781773FFFFE7028375B7E7040083A7F7
:10A97000870B0355050082971773FFFF6700637607
:10A980001773FFFFE702A373035505003287AE86F6
:10A990001796FF1F0356E6AF97B5FF1F9385C55067
:10A9A00097000000E780A0EF1773FFFF6700637355
:10A9B0001773FFFFE702A370B7E7040083A7C71769
:10A9C00082971773FFFF6700C3711773FFFFE702DA
:10A9D000036FB7E7040083A7871397B5FF1F93851D
:10A9E000A54C829701451773FFFF6700836F1773AC
:10A9F000FFFFE702C36CB7E7040083A7C71F8145C9
:10AA00001795FF1F0355E5A482971773FFFF670093
:10AA1000436D1773FFFFE702836AB7E7040083A75C
:10AA2000871397B5FF1F93852549829701451773B3
:10AA3000FFFF6700036B1773FFFFE7024368B7E789
:10AA4000040083A7C71F81451795FF1F035565A6FF
:10AA500082971773FFFF6700C3681773FFFFE70252
:10AA600003662E8597800000E780E0AF97800000A6
:10AA7000E780E0EC1773FFFF6700A3661773FFFF23
:10AA8000E702E36397800000E780E0F61773FFFFBB
:10AA9000670023655C49E1175CC95CC583572501E4
:10AAA000A1072319F50083570501A1072318F50015
:10AAB0008280F1473305F50297B7FF1F9387C7419F
:10AAC0009C433E9582808D476315F60803D7460068
:10AAD000854763F0E7081773FFFFE702435E36859B
:10AAE00036842E8997100000E780005929C98357C2
:10AAF000440093140501C18063E3970422859710F5
:10AB00000000E7806057FD14231294009307A00211
:10AB10006300F5029307B0026307F5029307900202
:10AB2000631FF500228597000100E780C08501A81A
:10AB30000146CA85228597A00000E78060B01773A0
:10AB4000FFFF6700035A228597100000E780C003CB
:10AB5000FDB7828097B6FF1F938646389C42014519
:10AB600099CF9843D44217B6FF1F2329E636639640
:10AB7000D70097B6FF1F23A5E6361385C7FE828050
:10AB80001773FFFFE702A35397000000E780A04B75
:10AB9000714433058502914597900000E78020E9D4
:10ABA00011E565551773FFFF6700A35397B7FF1FA4
:10ABB00023A2A73297000000E780E0483305850212
:10ABC000914597900000E78080E661DD97B7FF1F11
:10ABD00023A4A73097000000E780E04697B7FF1F47
:10ABE0002394A72E97000000E780E04597B7FF1F4A
:10ABF000239DA72C977701009387074A17B7FF1F5C
:10AC00002328F72C97070000938707E917B7FF1F42
:10AC1000232EF72A014579B71773FFFFE702234A6E
:10AC2000AA8517B5FF1F1305252A97100000E78096
:10AC3000C05B1773FFFF6700C34A1773FFFFE7028C
:10AC4000034897000000E78060FD97100000E78050
:10AC5000405B97B7FF1F938767289C4391CF13876B
:10AC6000C7FE19CB83D5C7FF17B5FF1F130585276F
:10AC700097200100E78020191773FFFF67006346E4
:10AC80001773FFFFE702A34397000000E780C0ECC3
:10AC900009CD834785002A8493F7070499EB035570
:10ACA000E50097000000E78080F91773FFFF670059
:10ACB00043438347C5009304450117B9FF1F130998
:10ACC000E92185E3832709005CC997B7FF1F23A704
:10ACD000972083274900F1FB97B7FF1F23A29720F6
:10ACE000E9B7FD172306F500610597800000E780AE
:10ACF000C0D68307840063CB07048347840093E7AF
:10AD000007F82304F400B7E704009C5F829742052C
:10AD1000A94741813375F5028347840093F707FC07
:10AD2000C98F2304F4008347D4003E951C402318A8
:10AD3000A40089CF984319CB8347C4005040814574
:10AD400085073305F50242054181029783270900F3
:10AD50005CC897B7FF1F23A397188327490089E78B
:10AD600097B7FF1F23AE97168347C4009DDF835517
:10AD7000040117B5FF1F1305E51697200100E780B2
:10AD8000800825B71773FFFFE702633397B7FF1FEC
:10AD90009387873A9C4701448583858B85E3AE84FE
:10ADA000B2853A8697100000E780804B2A8419C547
:10ADB00097100000E780C041829408CC2285177369
:10ADC000FFFF670003321773FFFFE702A32D411156
:10ADD0002E8932C6AA8997000000E780C031324729
:10ADE00013060502CA86970500009385C5CC17B5E2
:10ADF000FF1F1305650D97000000E780E0F82A8427
:10AE000025C99304C50097000000E780E04119467A
:10AE1000AA85268597100000E78080158545268540
:10AE200097100000E7806011177501001305852455
:10AE30004E9583450500268597100000E780201673
:10AE40005C4831468145A1075CC85CC48357240136
:10AE5000E1172319F40083570401E1172318F400C4
:10AE60001C4C3E859770FFFFE7806028A3042501F6
:10AE7000228541011773FFFF670003261773FFFF49
:10AE8000E702E3234111AA842EC632C497100000C2
:10AE9000E7806036004DB2452246834784000CC0EF
:10AEA00050C093F7F70393E707042304F400231833
:10AEB0000400268597100000E780803183479400C6
:10AEC000A9462317A40013D7370005073307D70275
:10AED0009D8B85072306F400A306E40083C70401C5
:10AEE000D8488507230FF7FE17B7FF1F130707FF83
:10AEF0005843232A04009307440129E317B7FF1F8F
:10AF00002320F7FE17B7FF1F232AF7FC17B4FF1FF4
:10AF1000130444FD228597200100E78000E11C44D2
:10AF2000858B5D8D19E58145228597200100E7809D
:10AF300080ED41011773FFFF6700A31A1CC317B709
:10AF4000FF1F232FF7F8D9B71773FFFFE702231767
:10AF500097050000938565B7014597000000E780DD
:10AF600000B001451773FFFF6700A3171773FFFFBA
:10AF7000E702E31497000000E78080B01773FFFF3B
:10AF8000670023168347C500A5E31773FFFFE70299
:10AF900003132A840355E50097000000E78000C8EA
:10AFA00021C18347840093F7F7FB2304F4001C407E
:10AFB00091C7DC4381C74C40014582979700000050
:10AFC000E78080B917B5FF1F1305C5F19720010071
:10AFD000E780A0E50355E40097000000E78020C665
:10AFE0001773FFFF6700E30F82801773FFFFE7020D
:10AFF000030D97B7FF1F938767EE970500009385B2
:10B0000065C817B5FF1F1305E5ED23A0070023A2B0
:10B01000070097200100E780E0CE1773FFFF67006D
:10B02000430C1C4D91CFDC4381CF1773FFFFE70228
:10B0300003098345070082971773FFFF6700630AC0
:10B04000828097B7FF1F938727EC9C4303C50700B7
:10B05000828097B7FF1F938727EB9C4303C5170098
:10B06000828097B7FF1F938727EA9C4303C5270079
:10B07000828097B7FF1F938727E99C4303C547004A
:10B08000828097B7FF1F938727E89C4303C537004B
:10B09000828097B7FF1F938727E79C4303C557001C
:10B0A000828097B7FF1F938727E69C4303C56700FD
:10B0B000828097B7FF1F938727E59C4303C57700DE
:10B0C000828097B7FF1F938727E49C4303C58700BF
:10B0D000828097B7FF1F938727E39C4303C59700A0
:10B0E000828097B7FF1F938727E29C4303C5A70081
:10B0F000828097B7FF1F938727E19C4303C5B70062
:10B1000011E11D45828097B7FF1F9387E7DF9C43BE
:10B1100003C5C700828097B7FF1F9387E7DE9C4374
:10B1200003C5D700828097B7FF1F9387E7DD9C4355
:10B1300003C5E700828097B7FF1F9387E7DC9C4336
:10B1400003D50701828097B7FF1F9387E7DB9C43F6
:10B1500003C52701828097B7FF1F9387E7DA9C43D7
:10B1600003D54701828097B7FF1F9387E7D99C4398
:10B1700003D56701828097B7FF1F9387E7D89C4369
:10B1800003D58701828097B7FF1F9387E7D79C433A
:10B1900003C5A701828097B7FF1F9387E7D69C431B
:10B1A00003C5B701828097B7FF1F9387E7D59C43FC
:10B1B00003C5C701828097B7FF1F9387E7D49C43DD
:10B1C00003C5D701828097B7FF1F9387E7D39C43BE
:10B1D0008857828097B7FF1F938707D39C4303D577
:10B1E000C702828097B7FF1F938707D29C4303D57E
:10B1F000E70219E11305800C828097B7FF1F938740
:10B20000A7D09C4303C50703828097B7FF1F93878E
:10B21000A7CF9C43C85B828097B7FF1F938747CE19
:10B220008843828097B7FF1F9387C7CD884382806A
:10B2300019E17D558280F5DE984265DFFDD917B7AB
:10B24000FF1F130767EF1847AA877155058B631D0A
:10B25000072403C507001547E37DA7FC03C7370094
:10B260001305F0057D171377F70FE364E5FC03C3BF
:10B270005700E30003FC83C86700E38C08FA03C7A8
:10B280007700494579171377F70FE364E5FA03C7A9
:10B29000A70011481305F7FF1375F50FE36BA8F826
:10B2A00003CE97000D481305FEFF1375F50FE362FB
:10B2B000A8F803C8B7006309080065181378F80FE9
:10B2C0001305600DE36705F703C5C70079487915D5
:10B2D0001375F50FE36FA8F403C8D7000D457D186B
:10B2E0001378F80FE36705F503D80701930E4017AD
:10B2F0005118420813580801E3ED0EF303C8E700A4
:10B300007D181378F80FE36605F303C827017D184D
:10B310001378F80FE36F05F103C88700C54E751861
:10B320001378F80FE3E70EF103D86701856E938E6B
:10B33000BEE06D18420813580801E3EC0EEF03D885
:10B3400047016D18420813580801E3E40EEF03D8D3
:10B3500087017918420813580801E36C05ED03C80A
:10B36000A7017D181378F80FE36505ED03C5B70154
:10B370001D487D151375F50FE36DA8EA03C5D701C8
:10B38000714879151375F50FE365A8EA03D5E70150
:10B390001308E00F7D1542054181E36CA8E803C561
:10B3A0000702494879151375F50FE364A8E8C853F7
:10B3B00001C937C834005915130858BFE36BA8E614
:10B3C00003A8870237C53400130555BF5918E36237
:10B3D00005E717B5FF1F2327C5B203C6050117B53B
:10B3E000FF1F2323F5B20545E375C5E403D8250106
:10B3F000D04933760603E31E06E203C61501E30ACD
:10B4000006E217B6FF1F232DB6AE83C527000146FF
:10B410006387A50003C61700F1453306B60283C74C
:10B4200007039305C00272971A071307C70516038F
:10B430001A9796084697B387B70241553E973297B9
:10B44000420741836362E8061773FFFFE70223C7E1
:10B45000368597800000E780A06897000100E780AC
:10B4600020482A8497A00000E780805A2A9497F009
:10B470000000E78060262A9497900000E780A08172
:10B480002A9497F0FFFFE780E06F2A94974000002E
:10B49000E78060932A9497700000E780A09C229533
:10B4A0001773FFFF6700E3C382801773FFFFE70294
:10B4B00003C14111A307A10097A00000E780A0C528
:10B4C0009305F100170500001305E5B597F0FFFFA0
:10B4D000E780802F014541011773FFFF670063C0BC
:10B4E0001773FFFFE70223BB17B4FF1F1304C4C485
:10B4F0000328840079599368180097B4FF1F23A18B
:10B5000014C51378180063100802BA84BE89368BFC
:10B51000328A2E89AA8A97F0FFFFE780E0A77D157F
:10B52000269519E531594A851773FFFF670023BA3D
:10B5300097F0FFFFE78040A67D152695A167E353AE
:10B54000F5FE97B7FF1F9387E7F598433E8C814B35
:10B5500001CB014597F00000E7802044933B1500A4
:10B560004A85DA865686D28597900000E780C04DDE
:10B570002A8911CD1C44F99B17B7FF1F2322F7BC62
:10B5800083270C00CDD3E3800BFA829769BF268511
:10B5900097B7FF1F23A407BA97F0FFFFE780809CAF
:10B5A0004146CE8517B5FF1F130585C297300100B0
:10B5B000E780C05697D00000E78040990325040B30
:10B5C00097D00000E780009D054597D00000E780F8
:10B5D00000A4054597000000E78060EDA9B797B784
:10B5E000FF1F938767B59C47858BEDC71773FFFFD8
:10B5F000E702E3AC17B5FF1F1305C5BB97B7FF1FE5
:10B6000023AC07B297B7FF1F23AA07B297B7FF1F54
:10B6100023A807B297200100E780208197500000FF
:10B62000E780E0F597100100E780A04C971001003B
:10B63000E780A05297B7FF1F938787AE9C4391C7BF
:10B64000054597800000E780402097B7FF1F93874C
:10B65000E7969C4399C741657D1597700000E78088
:10B6600040A297F00000E780E03D97D00000E7801F
:10B67000808F97B7FF1F9387E7C09C4313971701ED
:10B680006356070097F00000E78000AD97B7FF1FF3
:10B6900023A007B497B7FF1F23AE07B297B7FF1FCA
:10B6A00023AC07B297B7FF1F23AA07B29700000089
:10B6B000E780008C97000000E780007297F0FFFFA2
:10B6C000E780401897F00000E78040D61773FFFF2F
:10B6D000670023A1828097B7FF1F9387E7A5884360
:10B6E00082801773FFFFE702839D97800000E78049
:10B6F000607597800000E780C0771773FFFF6700D1
:10B70000439E1773FFFFE702E3992A849304140210
:10B7100001112E85B289A685214636C63A89973011
:10B720000100E780403D0DE9B24638082686CE8507
:10B730001305940497500000E780604121462C08CF
:10B740004A8597300100E780003B133515000561FD
:10B750001773FFFF670043980145D5BF1773FFFFBD
:10B76000E702E3959305450617A5FF1F1305057A24
:10B7700097100100E78020691773FFFF6700639649
:10B780001773FFFFE702A39341112EC697F0FFFF47
:10B79000E780601BB24588C141011773FFFF670056
:10B7A00043941773FFFFE702E38FAA842E849780E8
:10B7B0000000E780006CAA8985452285970000007B
:10B7C000E780E07D83C7E4011389940899E3138936
:10B7D0000403CE85228597000000E780407C214647
:10B7E00093051902228597000000E780607897B7DB
:10B7F000FF1F938767948C43228597100000E78092
:10B80000C082214693858402228597000000E7804C
:10B8100020761773FFFF6700238C1773FFFFE70283
:10B820008387397197F00000E780E0B49305400604
:10B8300061E997800000E78000606302051497A724
:10B84000FF1F83C7676E13B7170097A6FF1F238DCF
:10B85000E66C014499CFC16417B9FF1F1309C98D64
:10B860009309400EFD1497000000E780C0866342F4
:10B87000A40A97F0FFFFE780000D4169B72909008E
:10B88000096AFD7A2A8B81447D199389F97B130A11
:10B890000A71938A8AC797000000E780C08363D744
:10B8A000A4041304400EB387840217B7FF1F1307C5
:10B8B000A7880324070B3E948357C4016382270B98
:10B8C00018403307EB4063EAE900834744008507EB
:10B8D000B3874703D6976365F70801468145094555
:10B8E00097F0FFFFE780604EAA8B29E597400000A4
:10B8F000E780808385476317F50689659385057121
:10B9000017A5FF1F1305856097100100E780A04F62
:10B9100095A0B30734030327090BBA9703D7C701D0
:10B920006308970003C75700A38207002382E7003C
:10B93000050415BF9305C500228597000000E78028
:10B9400080E65E852286976501009385E57397F012
:10B95000FFFFE780E0525E8597100000E780608A75
:10B96000850415BF97A7FF1F9387077D9C478D838D
:10B97000858BC1F721611763FFFF6700437501469F
:10B980008545094502D002D202D402D697F0FFFFC6
:10B99000E780A043AA8479DD97F00000E780E09C6F
:10B9A0001389C4002A8481454A8597000000E780F6
:10B9B000005F0C4041464A8597000000E780405BED
:10B9C000832944006385090C4E8502D802DA02DC23
:10B9D00002DE97300100E78000482ACE14100546A9
:10B9E0002C0808184ECC97500000E780E00A137529
:10B9F000F50F51ED8355840093E525004A859700A6
:10BA00000000E780E05E11460C104A8597000000B8
:10BA1000E780005601469765010093856567268596
:10BA200097F0FFFFE780C045268597000000E7807C
:10BA3000407D5C40A1D3014685450D4597F0FFFF51
:10BA4000E780A038AA841DD548401389C4009730E8
:10BA50000100E78040402AC64A8597000000E78041
:10BA6000404C3246636FC5004C404A859700000049
:10BA7000E780005001468145268597F0FFFFE7806B
:10BA80002040268597000000E780A077E5B5835524
:10BA90008400ADB71763FFFFE702636297A7FF1F3C
:10BAA000938787699C471DC193E7870017A5FF1FF0
:10BAB0001305C54517A7FF1F2324F768971001003A
:10BAC000E78040321763FFFF6700A361DD9B17A784
:10BAD000FF1F2327F76697300000E780E0647DF1C1
:10BAE00017A5FF1F1305854297100100E780E0337B
:10BAF000D1BF1763FFFFE702035A4169AA892E8A63
:10BB0000B28A368BBA8B814417ACFF1F130CCC6200
:10BB1000930C400E7D1997F0FFFFE780C05B63C474
:10BB2000A40001443DA03384940383270C0B3E946E
:10BB30008357C401638627055A87D6865286CE85E9
:10BB40001305040397000000E780E0BB01C92380D0
:10BB50000B0022851763FFFF670063578347F401DB
:10BB600085C35A87D6865286CE85130594089700DA
:10BB70000000E78040B909C585472380FB00D1BF9D
:10BB8000850451BF835745006380071E1763FFFF7D
:10BB9000E702435101112A8497000000E780C04D5D
:10BBA00009C985476309F50605611763FFFF67004B
:10BBB000A35297E00000E780007C7DF583574400A6
:10BBC0004947ED9BE392E7FEC145228597000000BF
:10BBD000E7804033AA84228597000000E780204F49
:10BBE0000357440002CE91472A89631AF700228541
:10BBF00097000000E780A0513C082ACC3ECE97E099
:10BC00000000E78080765C55C5D374084A86A68517
:10BC10000545829751BF03574400D147E3F6E7F843
:10BC2000032A0400C169014997AAFF1F938ACA50D9
:10BC3000130B400EFD1997F0FFFFE780C049634FDB
:10BC4000A90E2285032A040097000000E780C04265
:10BC5000A1452A89228597000000E780A02AAA84AE
:10BC6000228597000000E780804A14402A86AA892E
:10BC700078082685CA8597000000E780C0E7AA8477
:10BC800005D503C7F40189476315F7008347C10150
:10BC900081DF5546D2851385640097300100E78027
:10BCA000E0E7014597800000E780C01901C583D710
:10BCB000C401A5E797A7FF1F938707489C479355A3
:10BCC0001900858913D73700058B01CF8983858BB0
:10BCD0006399B70001452EC697000000E780C0DBDE
:10BCE000B2454E8597800000E780601F0346C10182
:10BCF0002A8493751900268597900000E780E03923
:10BD000035C1268597800000E780E018268511C0A0
:10BD1000014597800000E780004C97300000E780E5
:10BD2000A0408547E312F5E883C754001307F00FDE
:10BD3000E38CE7E68507A382F400BDB5B30469038D
:10BD400083A70A0BBE9483D7C401638B3701554682
:10BD5000D2851385640097300100E780C0D955DD96
:10BD60000509D1BD5DD86DB782801763FFFFE7027B
:10BD7000633397800000E780000C05C1C164014473
:10BD800017A9FF1F1309493B9309400EFD1497F0B3
:10BD9000FFFFE7804034634EA40017A5FF1F130583
:10BDA000E51697100100E780E0031763FFFF6700C7
:10BDB000A332330534038327090B3E958357C5010E
:10BDC000638897002312050097800000E780A00C8D
:10BDD000050475BF97A7FF1F938707369C478D8380
:10BDE000858B8DE31763FFFFE702632D17A5FF1F08
:10BDF0001305C51197100100E78020031763FFFFAB
:10BE00006700232E82801763FFFFE702432B97050D
:10BE100000009385C5A017A5FF1F1305250F9710D8
:10BE20000100E78020EE1763FFFF6700832B176395
:10BE3000FFFFE702C3288841B7E70400BC5B0505A4
:10BE400042054181829709C585472300F500050514
:10BE50001763FFFF6700E32883C7F5FF2E8585077B
:10BE6000A38FF5FE828083C7F5FFFD1793F7F70FC9
:10BE7000A38FF5FE99EF1763FFFFE7024324B7E7AF
:10BE80000400BC571385F5FF82971763FFFF670017
:10BE9000432582801C41035745008D8FBA951CC1F4
:10BEA0002312B5003E85828093D78500A2051441F8
:10BEB000DD8D835745001387E6FF18C189072312DC
:10BEC000F50013D685004111238FB6FEA38FC6FE61
:10BED0004101828018419307F7FF1CC18357450039
:10BEE00085072312F500A30FB7FE82808357450014
:10BEF0008D8F2312F5001C41BE950CC12E858280CA
:10BF0000AA8703D7470008410D8FAA952392E7001F
:10BF10008CC38280184108453305A740828083572F
:10BF20004500035765001D8F1C4108453385A74018
:10BF30003305A74082801763FFFFE70243184111D2
:10BF40002EC62A8497000000E780A0FDB2456373E7
:10BF5000B50001A0835744000840BE952312B400E9
:10BF60003E9541011763FFFF6700A3171763FFFFAB
:10BF7000E702E31441112E84B28532C69700000017
:10BF8000E780A0FB3246A28597300100E78000B928
:10BF900041011763FFFF6700C3141763FFFFE70248
:10BFA00003122E84854597000000E78000F92300E6
:10BFB00085001763FFFF6700C3121763FFFFE702E7
:10BFC000031041112317B100894597000000E78055
:10BFD000C0F68347E1002300F5008347F100A3008A
:10BFE000F50041011763FFFF6700A30F1763FFFF11
:10BFF000E702E30C93D78500A2054111DD8D2317DD
:10C00000B100894597000000E78020F38347E100F5
:10C010002300F5008347F100A300F50041011763F9
:10C02000FFFF6700030C1763FFFFE7024309139745
:10C03000850193D78501C166938606F0D98F13D702
:10C040008500758FD98FA2053707FF00F98D411143
:10C05000DD8D2EC6914597000000E78000EE6C0054
:10C06000114697300100E78060AB41011763FFFF85
:10C07000670023071763FFFFE70263041C41854540
:10C0800003C4070097000000E78080E6228517635D
:10C09000FFFF670003051763FFFFE70243021C4130
:10C0A0004111894503C7070083C717002307E10033
:10C0B000A307F10097000000E78080E30355E1004B
:10C0C00041011763FFFF6700C3011763FFFFE7022A
:10C0D00003FF1C414111894503C7070083C71700AF
:10C0E0002307E100A307F10097000000E78040E08C
:10C0F0008357E100410113D58700A2075D8D4205FA
:10C1000041811763FFFF6700C3FD1763FFFFE7026D
:10C1100003FB0C4141112A8411466800973001004D
:10C12000E780C09F9145228597000000E78040DCB2
:10C13000B247C166938606F01397870113D587012E
:10C14000598D13D78700758F598DA2073707FF00C8
:10C15000F98F5D8D41011763FFFF670083F81C4570
:10C16000BE950CC18280AE87944391E6584101EFA1
:10C170000CC15CC1828003C7570013671700A382FC
:10C18000E700B687D5B70CC3EDB7AA87084119CD2C
:10C190001841D44398C36313D500D8C32A870346F4
:10C1A00057009376160081E623200700828094438F
:10C1B00081CA8C4203A847008CC363930601CCC399
:10C1C000799A14C3A302C7003687D1BF1C45DC4748
:10C1D0001D8DB777DBB6938777DB09853305F502CD
:10C1E000420541818280F147B385F50248452E958D
:10C1F00082808347450085072302F500828017630C
:10C20000FFFFE702C3EB2A8409E41763FFFF67001F
:10C2100043ED83474400F5DBFD1793F7F70F230247
:10C22000F400E5F71C4403D7270005072391E70036
:10C23000DC4399C3228582974C4889CD83475400BB
:10C24000898B99E71C4422859C479C439C47829795
:10C25000232A04000040232004007DB71763FFFF5A
:10C26000E702E3E58357250041112EC681EB014427
:10C27000228541011763FFFF6700A3E6035705000E
:10C280008147F146E305F7FEB385D70240458507B0
:10C290002E948345440008C4F5F5B247AA8481E78B
:10C2A000232A040009A81C456C0022859C439C435A
:10C2B000829748C84DDD85472312F400B2472320FA
:10C2C0000400231804002319F4005C485CC483D7DD
:10C2D0002400FD172391F40061BF1763FFFFE702FD
:10C2E00003DE97A7FF1F938767C4884323260500B3
:10C2F00023240500410597100100E78000B3176370
:10C30000FFFF670003DE1763FFFFE70243DB17A4AD
:10C31000FF1F1304A4C11C40411199CF9C47230067
:10C32000B5002AC65CC197000000E78040FB1C40B6
:10C33000DC4399C33245829741011763FFFF6700D1
:10C3400043DA0347450029E3584DAA877D551DCFA1
:10C350001763FFFFE702A3D61CC3DC4797A6FF1FA6
:10C3600023A6E6BCF156130507012390D7009705D5
:10C3700000009385050297100100E780A098014511
:10C380001763FFFF6700E3D57D55828082801763C6
:10C39000FFFFE702C3D20111614681452800976083
:10C3A000FFFFE780C0D497A7FF1F938727B89C4360
:10C3B00028009305F00FDC473EC697000000E78099
:10C3C000C0F405611763FFFF6700A3D197A7FF1FA4
:10C3D0009387C7B59C43D847A1679387C702631E5D
:10C3E000F70A397106DE22DC26DA80004AD84ED6FA
:10C3F00052D456D23285B28497000000E780C0C77D
:10C40000AA89268597000000E78020C92318A4FC8C
:10C41000268597000000E78040C82319A4FC2685E4
:10C4200097000000E78060C783D744000A8A231A78
:10C43000A4FC858393F7F70F230EF4FC8607BD0752
:10C4400093F7073F3301F1408A8A01498347C4FDCE
:10C450006367F902CE85130584FC232C54FD9700F5
:10C460000000E78080EA5281130104FCF25062541C
:10C47000D2544259B259225A925A21618280268559
:10C4800097000000E78060C193171900D69705094F
:10C490002390A7001379F90F55BF828097A7FF1F3C
:10C4A0009387C7A89C43D847A1679387A702631ABD
:10C4B000F70A397106DE22DC26DA80004AD84ED629
:10C4C00052D456D23285B28497000000E780C0BAB9
:10C4D000AA89268597000000E78020BCFD57231815
:10C4E000A4FC26852319F4FC97000000E780E0BA3D
:10C4F00083D744000A8A231AA4FC858393F7F70F95
:10C50000230EF4FC8607BD0793F7073F3301F14084
:10C510008A8A01498347C4FD6367F902CE85130502
:10C5200084FC232C54FD97000000E78000DE52813C
:10C53000130104FCF2506254D2544259B259225AA7
:10C54000925A21618280268597000000E780E0B43E
:10C5500093171900D69705092390A7001379F90FAF
:10C5600055BF828097A7FF1F9387479C9C43D8475E
:10C57000A16789076310F70A397106DE22DC26DA23
:10C5800080004AD84ED652D456D23285328997008E
:10C590000000E78060AEAA894A8597000000E78026
:10C5A000C0AF835749000A8A2318A4FC858393F7F8
:10C5B000F70F230CF4FC8607BD0793F7073F330101
:10C5C000F1408A8A8144834784FD63E7F402CE8583
:10C5D000130584FC232A54FD97000000E780E0D275
:10C5E0005281130104FCF2506254D2544259B259A0
:10C5F000225A925A216182804A8597000000E78082
:10C60000C0A993971400D69785042390A70093F4AC
:10C61000F40F55BF828097A7FF1F938727919C43F4
:10C62000D847A1679387E704631EF70A397106DECE
:10C6300022DC26DA80004AD84ED652D456D2328531
:10C64000B28497000000E78020A3AA89268597007E
:10C650000000E78080A42318A4FC26859700000032
:10C66000E780A0A3231AA4FC268597000000E7809A
:10C67000C0A283D744000A8A2319A4FC858393F7B8
:10C68000F70F230EF4FC8607BD0793F7073F33012E
:10C69000F1408A8A01498347C4FD6367F902CE8568
:10C6A000130584FC232C54FD97000000E780E0C5AF
:10C6B0005281130104FCF2506254D2544259B259CF
:10C6C000225A925A21618280268597000000E780D5
:10C6D000C09C93171900D69705092390A7001379DA
:10C6E000F90F55BF828097A7FF1F938727849C432C
:10C6F000D847A1679387C704631AF70A397106DE22
:10C7000022DC26DA80004AD84ED652D456D2328560
:10C71000B28497000000E7802096AA8926859700BA
:10C720000000E7808097FD572318A4FC2685231A74
:10C73000F4FC97000000E780409683D744000A8A03
:10C740002319A4FC858393F7F70F230EF4FC8607C7
:10C75000BD0793F7073F3301F1408A8A01498347B8
:10C76000C4FD6367F902CE85130584FC232C54FDB8
:10C7700097000000E78060B95281130104FCF25079
:10C780006254D2544259B259225A925A216182803B
:10C79000268597000000E780409093171900D697F0
:10C7A00005092390A7001379F90F55BF8280979749
:10C7B000FF1F9387A7779C43D847A167DD076317BF
:10C7C000F7041763FFFFE702838F797132853284A4
:10C7D00097000000E780408A2AC622859700000063
:10C7E000E780A08B2311A102228597000000E7803B
:10C7F000A088B2452300A102280897000000E78026
:10C80000C0B045611763FFFF6700A38D82809797D3
:10C81000FF1F9387A7719C43D847A167938787041D
:10C820006317F7041763FFFFE702638979713285A5
:10C83000328497000000E78020842AC62285970072
:10C840000000E78080852311A10222859700000067
:10C85000E7808082B2452300A102280897000000EB
:10C86000E780A0AA45611763FFFF67008387828086
:10C870009797FF1F9387876B9C43D847A167938740
:10C88000A7046312F7021763FFFFE7024383011156
:10C890002800814597000000E78020A70561176305
:10C8A000FFFF6700038482809797FF1F93870768C5
:10C8B0009C43D847A167938757026319F702175320
:10C8C000FFFFE702C37F0111328597F0FFFFE7808A
:10C8D000A07A2308A1008145280097000000E78086
:10C8E000C0A205611753FFFF6700A37F828097975F
:10C8F000FF1F9387A7639C43D847A1679387E702ED
:10C90000631BF7041753FFFFE702637B01113285B6
:10C91000328497F0FFFFE7804078AA84228597F061
:10C92000FFFFE7808077854709E9228597F0FFFFC1
:10C93000E78080744205B337A000280081452318A2
:10C9400091003ECA97000000E780209C05611753C4
:10C95000FFFF6700037982809797FF1F9387075D2A
:10C960009C43D84799476313F7081753FFFFE70223
:10C97000037579713285328497F0FFFFE780C06FCD
:10C980002AC6228597F0FFFFE78020712310A102BD
:10C99000228597F0FFFFE780206E2301A102228508
:10C9A00097F0FFFFE780406DA301A102228597F079
:10C9B000FFFFE780606C2302A102228597F0FFFF52
:10C9C000E780806B2313A102228597F0FFFFE780A9
:10C9D000A06AB2452314A102280897000000E7804E
:10C9E000C09245611753FFFF6700A36F828097973E
:10C9F000FF1F9387A7539C43D847A1679387C7031B
:10CA00006313F7081753FFFFE702636B79713285F1
:10CA1000328497F0FFFFE78020662AC6228597F0D0
:10CA2000FFFFE78080672310A102228597F0FFFFB8
:10CA3000E780A0662311A102228597F0FFFFE7801F
:10CA4000A0632302A102228597F0FFFFE780C06266
:10CA5000A302A102228597F0FFFFE780E061230394
:10CA6000A102228597F0FFFFE7800061B245A30392
:10CA7000A102280897000000E7802089456117532C
:10CA8000FFFF6700036682801753FFFFE7022363FF
:10CA900001112A8497F0FFFFE780005EAA842285B7
:10CAA00097F0FFFFE780605F228597F0FFFFE78048
:10CAB000C05E035744008D4763F7E700228597F077
:10CAC000FFFFE780805D228597F0FFFFE780E05C55
:10CAD0002800A68597000000E78020830561175392
:10CAE000FFFF670003609797FF1F938727449C43CE
:10CAF000D847A167FD07631FF7001753FFFFE70241
:10CB0000035C328597000000E78040F81753FFFF71
:10CB10006700235D82809797FF1F938727419C437F
:10CB2000D847A167E5076315F7081753FFFFE7022A
:10CB3000035979713285328497F0FFFFE780C05343
:10CB40002AC6228597F0FFFFE7802055228597F0BF
:10CB5000FFFFE78080542310A102228597F0FFFF9A
:10CB6000E780A053520551812311A102228523029F
:10CB7000010297F0FFFFE7802050A302A102228567
:10CB800097F0FFFFE780404F2303A102228597F033
:10CB9000FFFFE780604EB245A303A102280897F08B
:10CBA000FFFFE780807645611753FFFF67006353FF
:10CBB00082809797FF1F938767379C43D847A16769
:10CBC0009387E703631FF7001753FFFFE702234F25
:10CBD000328597000000E78060EB1753FFFF670086
:10CBE000435082809797FF1F938747349C43D847D1
:10CBF000A16793874704631EF7021753FFFFE702FD
:10CC0000034C79713285328497F0FFFFE780C0468C
:10CC10002AC6228597F0FFFFE7802048B245280802
:10CC200097F0FFFFE780606E45611753FFFF6700D5
:10CC3000434B82809797FF1F9387472F9C43D8478A
:10CC4000A167938787026310F7041753FFFFE7027A
:10CC5000034779713285328497F0FFFFE780C04146
:10CC60002AC6228597F0FFFFE7800041B2452300E6
:10CC7000A102280897F0FFFFE7802069456117535C
:10CC8000FFFF6700034682801753FFFFE70223433D
:10CC9000011197F0FFFFE780203EAA85280097F05A
:10CCA000FFFFE780806605611753FFFF670063435E
:10CCB0009797FF1F938787279C43D847A167D10782
:10CCC000631FF7001753FFFFE702633F32859700AA
:10CCD0000000E780A0FB1753FFFF670083408280BE
:10CCE0009797FF1F938787249C43D847A167C50761
:10CCF000631FF7001753FFFFE702633C328597007D
:10CD00000000E780A0F81753FFFF6700833D828093
:10CD10009797FF1F938787219C43D847A167B9073F
:10CD2000631FF7001753FFFFE7026339328597004F
:10CD30000000E780A0F51753FFFF6700833A828069
:10CD40009797FF1F9387871E9C43D847A167AD071E
:10CD5000631FF7001753FFFFE70263363285970022
:10CD60000000E780A0F21753FFFF6700833782803F
:10CD70009797FF1F9387871B9C43D8478947631862
:10CD8000F7021753FFFFE70283330111328532C8E0
:10CD900097F0FFFFE780402EAA85280097F0FFFF5D
:10CDA000E780A05605611753FFFF67008333828039
:10CDB0009797FF1F938787179C43D847A1678D07D5
:10CDC0006311F7041753FFFFE702632F0111328548
:10CDD000328497F0FFFFE780202A13066100AA84BF
:10CDE0004C00228597300000E780C0232800A685EC
:10CDF00097F0FFFFE780605105611753FFFF670061
:10CE0000432E82809797FF1F938787129C4381CF81
:10CE1000DC4391CB1753FFFFE702632A8297175336
:10CE2000FFFF6700032C82801753FFFFE7022329CF
:10CE300079713C08AE843ED2A165B7070A002A8406
:10CE40003ED448103C08DD053ED636C432C63AC250
:10CE500097D0FFFFE780E02F12474810BA8597F080
:10CE6000FFFFE780C01332464810B28597F0FFFFFE
:10CE7000E780E014A2464810B68597F0FFFFE780F0
:10CE80000012501001478146A685228597D0FFFFEA
:10CE9000E780805145611753FFFF670083241753D4
:10CEA000FFFFE702C32101117C000329C501AE8405
:10CEB0003ECAA165B70707002A843ECC48087C001B
:10CEC000C5053ECE97D0FFFFE780A0288345D90057
:10CED000480897F0FFFFE780800C50080147814623
:10CEE000A685228597D0FFFFE780004C0561175388
:10CEF000FFFF6700031F1753FFFFE702431C83C7B1
:10CF0000950093F7F707A384F50097000000E780EA
:10CF100040F91753FFFF6700C31C1753FFFFE702D9
:10CF2000031A79713C08AE843ED2A165B7070900A7
:10CF30002A843ED448103C08938545043ED632C628
:10CF400036C497D0FFFFE780C020A2464810B685C0
:10CF500097F0FFFFE780A00432464810B28597F0B3
:10CF6000FFFFE780C005501001478146A685228556
:10CF700097D0FFFFE780404345611753FFFF6700ED
:10CF800043161753FFFFE702831383C79500411130
:10CF90002A8493F7F707A384F50032852EC697F00D
:10CFA000FFFFE780800F85672AC46370F5029770E2
:10CFB0000000E78020E92246B24509ED114781468D
:10CFC000228597000000E78060E641011753FFFFCC
:10CFD0006700231101478346F501DDB71753FFFFB3
:10CFE000E702430C01113C003ECAB7070A003ECCE1
:10CFF0003C003ECE83C79500AA89328593F7F70798
:10D00000A384F5002E8497F0FFFFE7800009856771
:10D01000637DF504A165AA8493858504480897D0AB
:10D02000FFFFE7800013268597700000E78080E10E
:10D030002A8929E19145480897F0FFFFE78020F60B
:10D04000A685480897F0FFFFE78060F7CA85480883
:10D0500097F0FFFFE780A0F4014781465008A285C2
:10D060004E8597D0FFFFE780203405611753FFFFFF
:10D07000670083068145480897F0FFFFE78020F2AC
:10D080000349090275BF1753FFFFE702A301797136
:10D090001C103ECAB7070F003ECC404D1C10AA849E
:10D0A000AE894808994532C636893ECE97D0FFFFF3
:10D0B000E780200A32464808B28597F0FFFFE780F4
:10D0C00000EE630C0902A545480897F0FFFFE780D2
:10D0D000C0E62546CA8597200100E78020A45008B5
:10D0E00001478146CE85268597D0FFFFE780C02B7C
:10D0F00045611753FFFF670023FE8355C4024808AC
:10D1000097F0FFFFE780A0EB0355E402814505C5DA
:10D11000854785456301F502C167FD179305F00F4B
:10D12000630BF5007D1597700000E780208E930556
:10D13000150093F5F50F480897F0FFFFE78020E60C
:10D1400083450403480897F0FFFFE78040E58345E7
:10D150001403480897F0FFFFE78060E48355240339
:10D16000480897F0FFFFE78080E5835544034808AF
:10D1700097F0FFFFE780A0E49DB71753FFFFE7029A
:10D1800003F483C795008146014693F7F707A3840C
:10D19000F50097000000E78040EF1753FFFF67009E
:10D1A00043F41753FFFFE70283F179713E841C10AB
:10D1B0003ECA2E89B7070F00A1653ECCFD051C10A5
:10D1C000AA84480842C03AC23ECE36C432C697D07E
:10D1D000FFFFE78000F832464808B28597F0FFFF6E
:10D1E000E780E0DBA2464808B68597F0FFFFE780BE
:10D1F00000DD12474808BA8597F0FFFFE78020DC82
:10D200000248630C08029145480897F0FFFFE78049
:10D21000C0D21146A28597200100E78020905008D7
:10D2200001478146CA85268597D0FFFFE780C01752
:10D2300045611753FFFF6700C3EA8945480897F027
:10D24000FFFFE78080CF834704002300F50083477A
:10D250001400A300F500E1B71753FFFFE70283E4D2
:10D2600083C7950001112A8A93F7F707A384F50075
:10D270003285AE8432C697F0FFFFE78000E2324687
:10D280002A89328597F0FFFFE78000DF85676373A7
:10D29000F902AA894A8597700000E780A0BA2A841B
:10D2A00019ED114781464A86A685528597000000F0
:10D2B000E780C0B705611753FFFF6700E3E193877D
:10D2C000E9FF93F7F70F0547E366F7FE8347F5019C
:10D2D00095EB8947E380F9FE8346F40152850147C7
:10D2E0004A86A68597000000E78040B4A167D90769
:10D2F00048083ECC230A010002CE97000000E780D8
:10D30000A0B04DBF639EE7008947639EF900930775
:10D310001020231FF50097700000E780C0B76DBF95
:10D320000947E39BE7FA8D47E398F9FA228597705E
:10D330000000E78080DF9797FF1F938767DE9C439D
:10D3400099E79797FF1F938767C79C4399C703D5B2
:10D35000040097800000E780A0CE231F04002285F0
:10D360005DBF1753FFFFE70283D501113C003ECAA2
:10D37000B7070B003ECC3C003ECE83C795002A8900
:10D38000328593F7F707A384F500AE8497F0FFFF8B
:10D39000E780A0D093170501C187635AF006A16505
:10D3A0002A849385E502480897D0FFFFE78060DA7A
:10D3B000A285480897F0FFFFE78060C09797FF1F9E
:10D3C0009387C7BF9C43A9EB01449375F40F4808AA
:10D3D00097F0FFFFE780A0BC9355844093F5F50FCD
:10D3E000480897F0FFFFE78080BB9355044193F511
:10D3F000F50F480897F0FFFFE78060BA01478146C4
:10D400005008A6854A8597D0FFFFE780E0F90561BF
:10D410001753FFFF6700E3CC416585460546A285AB
:10D420007D1597500000E78060BD59DD51059700DC
:10D430000100E780808F130440063344850271B7F2
:10D440001753FFFFE702A3C70111B70706003EC647
:10D4500083C7950021642A8993F7F707A384F50011
:10D46000AE8428009305A4040AC40AC897D0FFFF1D
:10D47000E78020CE300001478146A6854A8597D0B7
:10D48000FFFFE78060F297E0FFFFE780801513045D
:10D490009404480822CC230A010002CE9700000021
:10D4A000E780809605611753FFFF670083C317531A
:10D4B000FFFFE70223BFC1642A8901449799FF1F38
:10D4C000938989C7130A8002FD1497E0FFFFE78064
:10D4D00080C16347A40001451753FFFF6700C3BF26
:10D4E000B307440303A7C90ABA9703D70700630623
:10D4F000970083D72700638427010504F9B7054502
:10D50000E1BF1753FFFFE702E3B92A8A2E8999C1C9
:10D5100023A0050081498144979AFF1F938A8AA11D
:10D52000614B97E0FFFFE78040C263C7A4004E85D0
:10D530001753FFFF670043BA3384640383A70A00CD
:10D540003E948357040099E763040900232089006F
:10D550008504C1BF4146D2851305440097100100E0
:10D56000E780605975F5A289E5B71753FFFFE70219
:10D5700063B339717C083ED4B7070A003ED67C08F5
:10D580003ED883C795002A8A328593F7F707A3848C
:10D59000F5002E8932C697F0FFFFE78000B085675F
:10D5A0006373F5083246AA84328597F0FFFFE7805F
:10D5B000A0AC8547AA8963E8A706A1659385850481
:10D5C000281097D0FFFFE780C0B82685977000002D
:10D5D000E78040872A8429ED9145281097F0FFFFC6
:10D5E000E780E09BA685281097F0FFFFE780209D4D
:10D5F000CE85281097F0FFFFE780609A01478146AB
:10D600003010CA85528597D0FFFFE780E0D9A16727
:10D610009387770448183EDC230A010202DE97F064
:10D62000FFFFE780607E21611753FFFF6700C3AAF9
:10D630008145281097F0FFFFE7806096A6852810A7
:10D6400097F0FFFFE780A0979797FF1F938747E525
:10D650009C4381CB22856389090097D00000E78035
:10D6600040248345040271B797D00000E780C022B0
:10D67000CDBF1753FFFFE702E3A283C79500411117
:10D68000AA8993F7F707A384F5003285AE84328A1E
:10D6900097F0FFFFE78060A08567637FF5022A8926
:10D6A00097600000E780007A2A84914631C583475D
:10D6B000F50105476387E70291C70D476366F704E5
:10D6C000AD461DA89305050303250A0041469710A2
:10D6D0000100E78040420DE941011753FFFF670059
:10D6E000A39F9305950803250A0041469710010062
:10D6F000E7806040814669F54A86A6854E85970099
:10D700000000E780C081C9BF83250A001305940883
:10D7100097700000E780A02919C1C146F1BF979713
:10D72000FF1F9387E79F9C4399E79797FF1F938776
:10D73000E7889C4399C7228597800000E780208A6C
:10D7400069FD8547A30FF400228597B00000E780AC
:10D750006084228597600000E780E0734E858146F3
:10D760004A86A68597F0FFFFE780607BA1679387D5
:10D77000570448003EC42302010002C697F0FFFF91
:10D78000E780806891BF1753FFFFE702C39083C70C
:10D7900095004111AA8993F7F707A384F500328514
:10D7A0002E89B28A97F0FFFFE780208F8567637428
:10D7B000F50EAA8497600000E780C0682A840DED0A
:10D7C000416B014A979BFF1F938B0B97130C400EE5
:10D7D0007D1B19A833048A0383A70B0B3E94835740
:10D7E000C40163836705050A97E0FFFFE780A08E09
:10D7F000E342AAFE95460DA08357C50163969702A2
:10D800009305050303A50A00414697100100E78030
:10D81000802E994611E181462686CA854E8597F06D
:10D82000FFFFE780C06F85A883A50A0013050403E6
:10D8300097700000E780A017C14679FD2285231E5E
:10D84000940097A00000E780E074228597600000B4
:10D85000E78060649797FF1F938787C49C43A9C3A1
:10D8600023000402228597D00000E78040F04E8517
:10D8700081462686CA8597F0FFFFE780406AA16748
:10D880009387070448003EC42302010002C697F0B4
:10D89000FFFFE780605741011753FFFF67002383B5
:10D8A00089472300F402E1B7397106DE22DC4AD849
:10D8B000800052D456D25AD026DA4ED65ECE2E8A68
:10D8C00032892A8B97D0FFFFE780E07D060571053E
:10D8D00041998A8A3301A140232224FC231404FCA9
:10D8E00097D0FFFFE780207C83479A000605350527
:10D8F00093F7F7072315A4FCA304FA004A8523260F
:10D9000024FC97E0FFFFE780407993170501C1876A
:10D910006340F0025681130104FCF2506254D25469
:10D920004259B259225A925A025BF24B21618280CB
:10D93000AA844A8597E0FFFFE7802076AA894A8576
:10D9400097E0FFFFE7806075A1659385C5022A898E
:10D95000130544FC97C0FFFFE780A07F268597C092
:10D96000FFFFE780E073854511C94A86CE8597C0E1
:10D97000FFFFE780606DAA8B21E98945130544FC10
:10D9800097E0FFFFE780A061A685130544FC97E0C0
:10D99000FFFFE780C062CE85130544FC97E0FFFFE0
:10D9A000E780E061CA85130544FC97E0FFFFE7804C
:10D9B000006101478146130644FCD2855A8597D001
:10D9C000FFFFE780609EB9B78145130544FC97E0EF
:10D9D000FFFFE780C05CA685130544FC97E0FFFFCE
:10D9E000E780E05DCE85130544FC97E0FFFFE7800C
:10D9F000005DCA85130544FC97E0FFFFE780205CCB
:10DA0000814497D0FFFFE780006AE3D4A4FA83A79C
:10DA10000B0113971400BA9783D5070099C5130516
:10DA200044FC97E0FFFFE78080598504D9BF7971F6
:10DA300006D622D44AD000184ECE52CC56CA26D290
:10DA40005AC8AE893289AA8A97D0FFFFE780A065BD
:10DA50000605690541990A8A3301A140232A24FC5D
:10DA6000231C04FC97D0FFFFE780E06383C7990085
:10DA700006052D0593F7F707231DA4FCA384F900E1
:10DA80004A85232E24FC97E0FFFFE780006193176F
:10DA90000501C187634FF0005281130104FDB250AC
:10DAA000225492540259F249624AD24A424B456189
:10DAB0008280AA844A8597E0FFFFE780005EA16527
:10DAC0009385A5022A89130544FD97C0FFFFE780CF
:10DAD0004068268597C0FFFFE780805C854509C9BF
:10DAE000CA8597C0FFFFE78020592A8B29E1894525
:10DAF000130544FD97E0FFFFE780604AA685130504
:10DB000044FD97E0FFFFE780804BCA85130544FD85
:10DB100097E0FFFFE780A04A01478146130644FDD6
:10DB2000CE85568597D0FFFFE7800088B5B7814541
:10DB3000130544FD97E0FFFFE7806046A6851305C7
:10DB400044FD97E0FFFFE7808047CA85130544FD49
:10DB500097E0FFFFE780A046814497D0FFFFE78072
:10DB60008054E3DBA4FA83270B0113971400BA97C0
:10DB700083D5070099C5130544FD97E0FFFFE780B3
:10DB800000448504D9BF1743FFFFE702435383478F
:10DB90004500404DD5EFFD575DC4834694000947CD
:10DBA0006363D70A0346B400854663EEC60883065E
:10DBB000E40063CA06085C45F9562390D7009787AE
:10DBC000FF1F83C7673799E3A304E4009787FF1F0C
:10DBD0009387C73E9C4381E78947A306F400979744
:10DBE000FF1F9387E78B9C4381E789472306F40057
:10DBF0009705000093854506AA841305040197F054
:10DC00000000E7802010FD57231AF40281471CDC36
:10DC100001489787FF1F23AD87309787FF1F9387A2
:10DC20006731232E040304C0804397D0FFFFE780B1
:10DC3000C05161463306C502814522859740FFFFEA
:10DC4000E780E04A81473E851743FFFF670063494D
:10DC5000FD57D5BF1743FFFFE70263462A840355EC
:10DC6000450297600000E780E01D19E5231E0400CF
:10DC70001743FFFF6700E3468357E401F5DB930595
:10DC800004FF174501001305657A97E00000E7805F
:10DC9000E014F9BF1743FFFFE70263422E89A16535
:10DCA00041119385E5032A8436C432C6BE843AC244
:10DCB00097C0FFFFE780E04912472285BA8597E0C9
:10DCC000FFFFE780C02D32462285B28597E0FFFF37
:10DCD000E780E02EA2462285B68597E0FFFFE78029
:10DCE000002E630309029145228597E0FFFFE7803C
:10DCF000C0241146A68597100100E78020E241016B
:10DD00001743FFFF6700E33D8945228597E0FFFF4A
:10DD1000E780A02283C704002300F50083C7140016
:10DD2000A300F500E9BF1743FFFFE702433983C7AC
:10DD30009500444D054793F7F707A384F5001C426F
:10DD4000411183C707006367F7062E842A89B1C093
:10DD500003C7D400630FF7021787FF1F13070726B7
:10DD6000184305C3A386F40097A00000E780404A4B
:10DD700083C7D40099E741657D1597400000E7808F
:10DD8000403083D72403918B89C797E00000E78058
:10DD9000C0134A85A28597F0FFFFE7808010A16736
:10DDA000C10748003EC42302010002C697F0FFFFEE
:10DDB000E780800541011743FFFF67008332174367
:10DDC000FFFFE702C32F03D745008D47AA84411107
:10DDD0002E8432892E8563E3E70297E0FFFFE78018
:10DDE000C02BAA8523000900268597C0FFFFE78086
:10DDF000A02841011743FFFF6700A32E97E0FFFF14
:10DE0000E780A0292AC6228597E0FFFFE780E02867
:10DE1000B24585472A862300F900268597C0FFFF73
:10DE2000E7808022F9B7397106DE22DC26DA80002D
:10DE30004ED652D456D24AD85AD05ECEAE89B2848B
:10DE4000AA8A97D0FFFFE780002506051305250263
:10DE500041990A8A3301A140232224FC231404FCA3
:10DE600097D0FFFFE780202383C7990006054D0563
:10DE700093F7F7072315A4FCA384F900268523262E
:10DE800024FC97E0FFFFE780402193170501C1873D
:10DE90006340F0025281130104FCF2506254D254E8
:10DEA0004259B259225A925A025BF24B2161828046
:10DEB000AA8B03AB040097C0FFFFE780601E51E50B
:10DEC00083D7440001498544F11793B71700A30194
:10DED000F4FC834734FCA165C9C79385E5041305A9
:10DEE00044FC97C0FFFFE780C026A685130544FCCD
:10DEF00097E0FFFFE780A00ADE85130544FC97E06A
:10DF0000FFFFE780C00B834734FC114691E30946CD
:10DF1000DA85130544FC97E0FFFFE7806005814444
:10DF2000630A0900416B7D1B97D0FFFFE780A016B5
:10DF300063CCA40201478146130644FCCE85568576
:10DF400097C0FFFFE7804046B1B7A685130634FCB3
:10DF500097000000E780E0E6933415002A898604E4
:10DF60008DBF9385C504A5BF8327C90013971400EF
:10DF7000BA9783D5070063886501130544FC97E0D1
:10DF8000FFFFE780C003850445B71743FFFFE702A3
:10DF9000831079711C103EC4B7070F003EC61C10D9
:10DFA0003EC883C79500AA8A328593F7F707A384F2
:10DFB000F500AE89328497E0FFFFE780000E9317EB
:10DFC0000501C187635AF0062A8A228597E0FFFF80
:10DFD000E780A00C2A895285032B040097C0FFFF1D
:10DFE000E780000C39ED8357440081440544F11764
:10DFF00093B71700A303F10083457100DA872287E6
:10E00000CA865286280097000000E780E0C80147D2
:10E0100081463000CE85568597C0FFFFE780C03827
:10E02000A1679387D70348083ECC230A810026CEF8
:10E0300097F0FFFFE78040DD45611743FFFF670072
:10E040000309A2851306710097000000E78060D7DE
:10E05000AA84094455D13544E30055FB4A8597F01D
:10E06000FFFFE78000450D4441D9014497D0FFFFF1
:10E07000E7806002634DA400C16B0144FD1B97D093
:10E08000FFFFE7804001634EA4001544B5B7DC44B0
:10E0900013171400BA9783D7070063832703050477
:10E0A000F1B7D84493171400BA9703D70700631B3E
:10E0B000770123902701268597A00000E78080DB69
:10E0C00001441DBF050465BF1743FFFFE70283FD41
:10E0D00083C7950041112A8A93F7F707A384F500B7
:10E0E00032852E89328497E0FFFFE78000FB93178B
:10E0F0000501C1876353F006AA89228597E0FFFFD7
:10E10000E780A0F92311A1004E85832A040097C05F
:10E11000FFFFE780E0F839E5835744008544014478
:10E12000F11793B71700A300F1000348110003573C
:10E130002100D6875285CE862686CA8597F0FFFFB6
:10E14000E7806006A167F10748003EC42302910002
:10E1500022C697F0FFFFE78020CB41011743FFFF66
:10E16000670083F7A2851306110097000000E7807F
:10E1700040C52A84894455D98357210011678544B5
:10E18000BA97C2071167C1831307F7EFE36FF7F878
:10E190009787FF1F9387C7F89C4381CB854513055D
:10E1A000210097500000E7802075835521002285CB
:10E1B000814497C0FFFFE78040E525D92310050083
:10E1C000228597A00000E78040CD85B71743FFFF69
:10E1D000E70263EC83C7950041112A8B93F7F70799
:10E1E000A384F50032852E8A328497E0FFFFE78012
:10E1F000C0EA93170501C1876351F006AA8A2285F8
:10E2000097E0FFFFE78060E92A895685832B0400A9
:10E2100097C0FFFFE780C0E831E5835744008144A1
:10E220000544F11793B71700A301F100034831002B
:10E23000DE875A854A87D6862286D28597F0FFFFE9
:10E24000E78060F6A167ED0748003EC42302810025
:10E2500026C697F0FFFFE78020BB41011743FFFF71
:10E260006700E3E6A2851306310097000000E7800F
:10E2700040B5AA8409445DD99167CA97C20711675E
:10E28000C1831307F7EF0544E362F7FACA8597C025
:10E29000FFFFE78080D7014451F9814997D0FFFF04
:10E2A000E78060E063DBA900984893971900BA976C
:10E2B00003D7070005EF2390270197D0FFFFE780E2
:10E2C00080DE1544E384A9F6268597A00000E78048
:10E2D000C0BC9787FF1F9387A7E49C430144B9D72D
:10E2E0004A8597500000E780C05889B785097DB7F7
:10E2F0001743FFFFE70203DB79713E847C083EC8C9
:10E300002E8AB7071400A1653ECAE5057C08AA89D4
:10E31000080836C4428932C6BA8AC6843ECC97C041
:10E32000FFFFE78000E3CA85080897E0FFFFE7806A
:10E3300000C732460808B28597E0FFFFE78020C893
:10E34000A246630A09049D45080897E0FFFFE7809D
:10E35000C0BE1D4681459740FFFFE78040D96389D5
:10E360000A089145080897E0FFFFE78000BD1146C5
:10E37000A68597000100E780607A10080147814672
:10E38000D2854E8597C0FFFFE780000245611743A5
:10E39000FFFF670063D4B685080897E0FFFFE780BA
:10E3A00000C21C400808D8439355C701858912074D
:10E3B0005183B205D98D97E0FFFFE78040C01C4034
:10E3C000080883C5870097E0FFFFE78040BD1C4039
:10E3D000080883C5A70097E0FFFFE78040BC1C400A
:10E3E000080883C5970097E0FFFFE78040BB85BF23
:10E3F0008945080897E0FFFFE78020B483C7040041
:10E400002300F50083C71400A300F500BDB7174330
:10E41000FFFFE70223C983C795004111AA8993F73B
:10E42000F707A384F5003285AE84328497E0FFFFBE
:10E43000E780A0C693170501C187635DF0042A89B0
:10E44000032A040097C0FFFFE78080C519E98357BE
:10E4500044000548F11793B71700A307F100814660
:10E4600031A81306F100A28597000000E7806095AF
:10E470001DC51C459DC783D6470001480347F100D1
:10E4800093078500D2884A86A6854E8597000000AE
:10E49000E78040E641011743FFFF6700E3C30948F7
:10E4A0007DBF1D486DBF1743FFFFE702A3BF657126
:10E4B0005C083EC4B7077B013EC65C083EC883C704
:10E4C00095002A8A328593F7F707A384F500AE8971
:10E4D00097E0FFFFE78040BA8357E100E1C7894535
:10E4E000280097C0FFFFE780C0C68145280097E05D
:10E4F000FFFFE780C0AA97C0FFFFE780A0CC978707
:10E50000FF1F9387E7F99C431784FF1F0344C4A2AE
:10E51000AA843334800099C3136424009787FF1FB3
:10E520009387C7A99C4399C3136444009787FF1F2F
:10E53000938707BF9C4399C31364840083D5040069
:10E540002800014997E0FFFFE78060A783D52400FA
:10E55000280097E0FFFFE78080A683D544002800CD
:10E5600097E0FFFFE780A0A597D0FFFFE780A0AE70
:10E5700093150501C181280097E0FFFFE78020A4E3
:10E58000A285280097E0FFFFE78060A39C446360BA
:10E59000F902014781463000CE85528597C0FFFFC2
:10E5A000E78080E059611743FFFF6700E3B2DC4476
:10E5B0001314490028003E9497E0FFFFE78060961F
:10E5C000834744000347540089070607BA97860724
:10E5D000E36AF5FC835524002800814A97E0FFFF99
:10E5E000E780E09D83454400280097E0FFFFE78037
:10E5F000009B83455400280097E0FFFFE780209AA6
:10E600008347440063C9FA00814A8347540063C1C9
:10E61000FA020509A5BF1C4413975A002800BA97AF
:10E6200083D50700850A97E0FFFFE7804099C9BFBF
:10E63000032BC40093975A0028003E9B83552B0060
:10E64000850A97E0FFFFE780809783550B0028003D
:10E6500097E0FFFFE780A0964DBF1743FFFFE7025B
:10E6600003A65C4993E717005CC997A00000E78008
:10E6700020B61743FFFF6700C3A61743FFFFE7025B
:10E6800003A42E84814597F0FFFFE780C0E705C50E
:10E6900083570500FD172310F50009C48357250093
:10E6A0002310F40097000000E78060FB014517434A
:10E6B000FFFF670003A331457DD823100400C5BFC9
:10E6C0001743FFFFE702039E83C7950041112A8A83
:10E6D00093F7F707A384F50032852E89328497E0FB
:10E6E000FFFFE780809B93170501C1876356F00603
:10E6F000AA89C145228597E0FFFFE780A0802A8B89
:10E700004E85832A040097C0FFFFE780609931E9B6
:10E7100083574400231101000544F11793B71700F4
:10E72000A300F10081440348110003572100D6875C
:10E730005285CE862286CA8597F0FFFFE780A0A685
:10E74000A1679387170248003EC42302810026C6B2
:10E7500097E0FFFFE780406B41011743FFFF670031
:10E76000A39713061100A28597F0FFFFE78060656D
:10E77000AA8409E523110100094475B79305210016
:10E780005A8597000000E78080EF835721002A8494
:10E79000D9DB9787FF1F9387A7989C4381CB85453B
:10E7A0001305210097500000E780001583552100D4
:10E7B0002685314497C0FFFFE78020852DD52310A3
:10E7C0000500268597900000E780206D0144A1BFD9
:10E7D0001743FFFFE702A38E41112E896C00AA8424
:10E7E00002C697F0FFFFE78000D20DC10357050076
:10E7F00005072310E50097000000E78040E6814709
:10E800003E8541011743FFFF6700A38D32479547BF
:10E8100065DBCA85268597300000E780400DC1473B
:10E82000E34005FE3244854741462310F4008357F8
:10E830000900A685130544002311F4009700010088
:10E84000E780C02D228545BF1743FFFFE702838580
:10E8500083C795004111AA8A93F7F707A384F500AF
:10E860003285AE89328497E0FFFFE78000839317FB
:10E870000501C1876356F0062A8AC145228597D0D3
:10E88000FFFFE7802068AA845285032B040097C00D
:10E89000FFFFE780E08031E9835744002311010046
:10E8A0008544F11793B71700A300F1000144034812
:10E8B000110003572100DA875685D2862686CE8539
:10E8C00097F0FFFFE780208EA1679387070248003B
:10E8D0003EC42302910022C697E0FFFFE780C052AA
:10E8E00041011733FFFF6700237FA2851306110044
:10E8F00097F0FFFFE780E04C2A8409E5231101002F
:10E90000894475B726859305210097000000E780AC
:10E9100060ECAA8449FD83552100228597B0FFFF52
:10E92000E780A06E49F5014997C0FFFFE780A07717
:10E93000635DA900184893171900BA9703D7070019
:10E940000DEF035721002390E70097C0FFFFE780FA
:10E950008075630625039777FF1F9387677C9C4329
:10E9600099C70355210097500000E78080F0228569
:10E9700097900000E78060521DBF050975B7954468
:10E980003DB705C19307F00F630FF500C547630C52
:10E99000F5009307F5FF05453315F5004205418164
:10E9A00082800145828041657D158280B9E91733F7
:10E9B000FFFFE702C370034506033284970000009F
:10E9C000E78060FC9305803EB305B502C205C181B6
:10E9D00081CD0357E402854763F8E700130504017E
:10E9E00097E00000E78020428357E40241677D17EB
:10E9F0006385E700FD172317F4021733FFFF670055
:10EA0000436E82801733FFFFE702E368004283C74B
:10EA10009500444D0349140093F7F707A384F500CC
:10EA200083470400220911673369F900A167B347DE
:10EA3000F90041112A8BAE8A63ECE70E834724006C
:10EA40001307C00EB91793F7F70F6373F710034757
:10EA50003400C14763EEE70E834744001307E00725
:10EA600093C707086371F70C8349840083477400D8
:10EA7000A209B3E9F900856763F7F90A034A64005C
:10EA8000834754004E85220A336AFA0097500000EB
:10EA9000E780403B61C123962403834B3400137A03
:10EAA000FA00239A34032388740323994403938937
:10EAB0000401631C090023A60402239804024E8566
:10EAC00097E00000E78060363DA0034924004A85B6
:10EAD00097000000E78020EB2397A40283474400BF
:10EAE0004E85A388F402E38D0BFCE30B09FC97E051
:10EAF0000000E780202F97900000E7800073814698
:10EB00000146D6855A8597E0FFFFE7800058A16748
:10EB1000938797033EC423020100480002C697E092
:10EB2000FFFFE780602E41011733FFFF6700235A84
:10EB30008544A2862686D6855A8597E0FFFFE78022
:10EB4000C054A167938797033EC423029100F1B795
:10EB5000BD44C5B79144F1BF1733FFFFE7028354AB
:10EB600001111C08404D3EC2B7070F003EC41C08EF
:10EB70003EC62A89AE8997C0FFFFE780A0DA585CBD
:10EB80001C5C6346B70E6394E50063E2A70E338511
:10EB9000A740B3B7A700B305B7401306803E814630
:10EBA0009D8D97000100E78080B793140501C18017
:10EBB000A1659385C503480097B0FFFFE7806059C2
:10EBC0008145480097D0FFFFE780603D83550404EE
:10EBD000480097D0FFFFE780803E8355240448001B
:10EBE00097D0FFFFE780A03D814589CCC167FD1725
:10EBF0009305F00F6388F400268597500000E780A6
:10EC0000E0E0AA85480097D0FFFFE7804039035530
:10EC10004404814501CDC167FD179305F00F6307DB
:10EC2000F50097500000E78060DEAA85480097D085
:10EC3000FFFFE780C03683456404480097D0FFFF9C
:10EC4000E780E03583457404480097D0FFFFE780F4
:10EC50000035500001478146CE854A8597B0FFFFB9
:10EC6000E780807405611733FFFF6700E346814446
:10EC700081B71733FFFFE702834483C7950093F7FB
:10EC8000F707A384F50097000000E78020ED173315
:10EC9000FFFF670003451733FFFFE702A34083C769
:10ECA00095004111404D93F7F707A384F5002A8A98
:10ECB0003285B284AE8997D0FFFFE780003E2A8B71
:10ECC000268597D0FFFFE780403D2A89268597D08B
:10ECD000FFFFE780603A93170B0163CA0702E177F1
:10ECE000CA97C207C183116763E3E702930709105C
:10ECF000C207C1831307B00F637BF70093170901A5
:10ED0000C187AA8A634AF000C54763FE57014101E3
:10ED10001733FFFF6700433C97B0FFFFE780C02831
:10ED2000E31725FFD5B763080B0263060902814488
:10ED300063890A02B7077F002310640523112405A5
:10ED40007CC0568597000000E780E0C39304803EB6
:10ED5000B304950239A0B7077F00232004047CC0C8
:10ED600081440355240497E00000E780A0A3A1C4D8
:10ED700097C0FFFFE78000BB269593D7F441333758
:10ED80009500AE97BA9708DC5CDCCE85528597007B
:10ED90000000E780A0DC99E023220404A1679387A8
:10EDA000B70348003EC42302010002C697E0FFFFFC
:10EDB000E7808005A9BF814701481CDC232E04039E
:10EDC000E9B71733FFFFE702832F97C0FFFFE78004
:10EDD000C037E1473305F502914597500000E780C1
:10EDE00000C5E55711C59777FF1F23A5A7148147D5
:10EDF0003E851733FFFF6700C32E85471777FF1F38
:10EE0000230CF71282801733FFFFE702432B97771B
:10EE1000FF1F9387E71180433DC08357040463902D
:10EE2000A70683572404639CB7043689B28497C02D
:10EE3000FFFFE78020AF5C5C63C3B7046395B70056
:10EE40001C5C63EEA7028347640463F3F400A687A7
:10EE50002303F4048347740463F39700A687A30392
:10EE6000F4048357440441677D176385E7008507F1
:10EE70002312F4043C4481C7CA8526858297173340
:10EE8000FFFF670003269777FF1F9387670A9C435E
:10EE9000014599C303C5870082801733FFFFE7024E
:10EEA00003220111B70707003EC683C79500584DDE
:10EEB0000AC493F7F7070AC8A384F5002A89AE8429
:10EEC00011CB1C4283C707002304F7009790000072
:10EED000E7800034216493055402280097B0FFFFB7
:10EEE000E780202797000000E78020FAAA85280005
:10EEF00097D0FFFFE780A00A300001478146A68532
:10EF00004A8597B0FFFFE780204A1304440248086F
:10EF100022CC230A010002CE97E0FFFFE780C0EE7B
:10EF200005611733FFFF6700C31B1733FFFFE702BD
:10EF3000031901117C003ECAB70707003ECC7C00D4
:10EF40003ECE83C795002E84AA8493F7F707A38447
:10EF5000F500A16593855502480897B0FFFFE7804B
:10EF6000401F97000000E78040F2AA85480897D02C
:10EF7000FFFFE780C002500801478146A285268531
:10EF800097B0FFFFE780404205611733FFFF67003E
:10EF900043159777FF1F9387A7F99C43094599C3AA
:10EFA00003C5970082809777FF1F938767F89C437C
:10EFB000094599C303C5D70082809777FF1F9387C0
:10EFC00027F79C43014599C303C5A70082801733E7
:10EFD000FFFFE702230D0111B70708003EC683C7F4
:10EFE0009500404D0AC493F7F7070AC8A384F500BB
:10EFF0002A89AE8429C41442854703C7060063E00A
:10F00000E70A83479400094681496380C702B30732
:10F01000F740A304E400B339F00083C716002305CA
:10F02000F40097900000E780A01E03572403058B8F
:10F0300019C76386090097D00000E78000E92164C2
:10F0400093058402280097B0FFFFE78080109700A7
:10F050000000E78040F4AA85280097D0FFFFE780F2
:10F0600000F497000000E78080F5AA85280097D07B
:10F07000FFFFE780C0F2014781463000A6854A8540
:10F0800097B0FFFFE780403213047402480822CC97
:10F09000230A010002CE97E0FFFFE780E0D605617A
:10F0A0001733FFFF670043031733FFFFE702230116
:10F0B00001117C003ECAB70708003ECC7C003ECE62
:10F0C00083C795002E84AA8493F7F707A384F500DD
:10F0D000A16593858502480897B0FFFFE780600728
:10F0E00097000000E78020EBAA85480897D0FFFF33
:10F0F000E780E0EA97000000E78060ECAA85480816
:10F1000097D0FFFFE780A0E9500801478146A2851C
:10F11000268597B0FFFFE780202905611733FFFFA1
:10F12000670023FC9777FF1F938787E09C43014587
:10F1300099C303C5B70082801733FFFFE70223F8A6
:10F140000111B70707003EC683C79500404D0AC4AA
:10F1500093F7F7070AC8A384F5002A89AE8405C887
:10F160001C42054783C707006368F7060347B400DE
:10F17000630FF700A305F40097900000E7804009B3
:10F180008347B400B9CF97D0FFFFE78040BE21642A
:10F190009305B400280097B0FFFFE78080FB97003D
:10F1A0000000E78060F8AA85280097D0FFFFE7807D
:10F1B00000DF014781463000A6854A8597B0FFFFF2
:10F1C000E780801E2904480822CC230A010002CED1
:10F1D00097E0FFFFE78040C305611733FFFF67003B
:10F1E00043F097D0FFFFE78020BF55B71733FFFFED
:10F1F000E702E3EC01117C003ECAB70707003ECCF2
:10F200007C003ECE83C795002E84AA8493F7F7072F
:10F21000A384F500A165AD05480897B0FFFFE7801E
:10F2200040F397000000E78020F0AA85480897D0B7
:10F23000FFFFE780C0D6500801478146A28526859A
:10F2400097B0FFFFE780401605611733FFFF6700A7
:10F2500043E99777FF1F9387A7CD9C43094599C33F
:10F2600003C5C70082801733FFFFE70243E50111A2
:10F270007C00AE843ECAA165B70707002A843ECC55
:10F28000D1057C0048083ECE97B0FFFFE78060ECD8
:10F2900097000000E78020FCAA85480897D0FFFF70
:10F2A000E780E0CF500801478146A685228597B0C8
:10F2B000FFFFE780600F05611733FFFF670063E220
:10F2C0001733FFFFE702A3DF83C7950093F7F70724
:10F2D000A384F50097000000E78020F91733FFFFB3
:10F2E000670023E01733FFFFE702C3DB83C7950006
:10F2F0000329C501411193F7F707A384F5001C42C8
:10F3000083C90700854763E637079777FF1F938711
:10F3100027199C432E84AA8485CF97000000E7809C
:10F3200080F389476306F502630409028347C90035
:10F33000638037032306390197900000E78040ED92
:10F3400083572903898B89C797D00000E780E0B7EE
:10F350002685A28597000000E78020F1A167CD07F0
:10F3600048003EC42302010002C697E0FFFFE78089
:10F37000A0A941011733FFFF670003D69777FF1F4E
:10F38000938707BB9C431D4599C303C5E700828053
:10F390001733FFFFE702A3D20111B70707003EC6EC
:10F3A00083C79500584D0AC493F7F7070AC8A3848A
:10F3B000F5002A89AE8415C71C4283C707009396BF
:10F3C0008701E18663C4060685466381D7068346C6
:10F3D000E7006388F6002307F70097900000E780B6
:10F3E00020E321649305E400280097B0FFFFE78045
:10F3F00040D697000000E780A0F8AA85280097D0A3
:10F40000FFFFE780C0B9014781463000A6854A85E5
:10F4100097B0FFFFE78040F93504480822CC230A63
:10F42000010002CE97E0FFFFE780009E05611733E1
:10F43000FFFF670003CB1733FFFFE70243C801114B
:10F440007C003ECAB70707003ECC7C003ECE83C797
:10F4500095002E84AA8493F7F707A384F500A1658D
:10F46000B905480897B0FFFFE780A0CE97000000DD
:10F47000E78000F1AA85480897D0FFFFE78020B217
:10F48000500801478146A285268597B0FFFFE78097
:10F49000A0F105611733FFFF6700A3C41733FFFF17
:10F4A000E70243C0AA8401441779FF1F130989A802
:10F4B000E14997C0FFFFE78040C96344A4000145CC
:10F4C00019A833053403832709003E958357250087
:10F4D0006397970011051733FFFF6700E3BF05042B
:10F4E000C9BF032E8500630A0E121773FF1F130393
:10F4F00023C303230300631503002943639006120B
:10F5000003234E01631503001D436399071017334E
:10F51000FFFFE70243B8C689428A3E89BA8AB684A9
:10F52000328BAE8B2A84B5E103554E0019E50143B9
:10F530001A851733FFFF670083B9A167A98F116789
:10F5400063FBE70097000000E78080F5814597F0B6
:10F55000FFFFE780C0120844B70700E05841F98F69
:10F5600018455CC1B707001FF98F1CC55C4991C7DE
:10F57000610597E00000E780408BE38A09FA228565
:10F5800097900000E78060C65DB7328597C00000A5
:10F59000E78040430D4349DD1C44116703D5470014
:10F5A000A167A98F63FBE70097000000E78040EFA9
:10F5B000814597F0FFFFE780800C032384009316BA
:10F5C0004B01D1828347B300035663008588FD8BCE
:10F5D000A305F300FD777D8E558EFD76FD16B204F2
:10F5E000F18E83274301C58E231273012313D300A9
:10F5F0002304530123052301A3044301BDDF228516
:10F6000097B0FFFFE78020CDAA850844B5D16105FA
:10F6100097D00000E780207F8DB71D431A85828038
:10F620001733FFFFE70203A80569AA84AE89328A6F
:10F630000144FD5A7D1997C0FFFFE780C0A56347CD
:10F64000A40001451733FFFF670003A9D8449317AF
:10F650001400BA9703D70700631F3703239057019D
:10F6600063070A00268597900000E780A0809C44ED
:10F670009DC383D76700B3F72701639E3701D28804
:10F68000014881470147814601468145268597000B
:10F690000000E78040E5050479BF1733FFFFE7026C
:10F6A00063A079711C103EC4B7070F003EC61C1042
:10F6B0003EC883C79500AA8A328593F7F707A384CB
:10F6C000F5002E89328497D0FFFFE780009D9317C5
:10F6D0000501C187635AF006AA89228597D0FFFFEA
:10F6E000E780A09B2A8A4E85032B040097B0FFFF7A
:10F6F000E780009B39ED8357440081440544F117AE
:10F7000093B71700A303F10083457100DA872287BE
:10F71000D2864E86280097E0FFFFE780E05701473A
:10F7200081463000CA85568597B0FFFFE780C0C785
:10F73000A1679387F70348083ECC230A810026CEB1
:10F7400097D0FFFFE780406C45611733FFFF6700EC
:10F75000A398A2851306710097E0FFFFE78060661B
:10F76000AA84094455D1528597E0FFFFE78060D411
:10F770000D4459D90546D285268597000000E780BB
:10F7800060EA2A8451B71733FFFFE702439383559A
:10F7900007000346270041112A842E8532C62EC455
:10F7A00097E0FFFFE780E0D001C93246A2452285FD
:10F7B00097000000E78000E741011733FFFF670073
:10F7C00043921733FFFFE702038D83C79500411172
:10F7D000AA8A93F7F707A384F5003285AE893284AD
:10F7E00097D0FFFFE780608B93170501C1876357B0
:10F7F000F00AC1452A8A228597C0FFFFE780807002
:10F800002A8D228597D0FFFFE78020892A892285CB
:10F8100097D0FFFFE7804086930705F893F7F70F2F
:10F820001307E007AA8B637BF706228597D0FFFFBB
:10F83000E78080842A8C228597D0FFFFE780C083F1
:10F84000AA8C5285032B040097B0FFFFE780408508
:10F8500039E983574400231101008144F11793B71C
:10F860001700A300F100054403471100835621004F
:10F87000938784005685DA8822885286CE8597F051
:10F88000FFFFE78020A7A167E90748003EC42302E5
:10F89000810026C697D0FFFFE7800057410117334C
:10F8A000FFFF6700C38213061100A28597E0FFFFE8
:10F8B000E7802051AA8409E52311010009446DB7AE
:10F8C000930521006A8597F0FFFFE780A0F02A8466
:10F8D00041FD835521009356C900131649018548FF
:10F8E0006688E2875E87858A5182268597000000B8
:10F8F000E78060BF2A848DBF1723FFFFE702A3794B
:10F9000083C7950041112A8B93F7F707A384F5006D
:10F910003285AE89328497C0FFFFE7800078931765
:10F920000501C1876352F00A2A8A228597C0FFFF2A
:10F93000E780A076AA8A228597C0FFFFE780E0755E
:10F940002A89228597C0FFFFE7800073930705F897
:10F9500093F7F70F1307E0072A8C6377F7062285E2
:10F9600097C0FFFFE7804071AA8C228597C0FFFFF8
:10F97000E78080702A8D5285832B040097A0FFFFBB
:10F98000E780007239E58357440085440144F1174C
:10F9900093B71700A301F1000347310093078400D8
:10F9A0005A85DE882688D6865286CE8597F0FFFF58
:10F9B000E78040948D4748003EC42302910022C650
:10F9C00097D0FFFFE780404441011723FFFF670006
:10F9D0000370A2851306310097E0FFFFE780603EC9
:10F9E0002A84894455D99356C9001316490185487C
:10F9F0006A88E6876287858A5182D68597000000EB
:10FA0000E78060AEAA8449BF1723FFFFE70283693E
:10FA10002A8981440144617A916A176BFF1F130B95
:10FA20002B7097B0FFFFE780006863C7A4002285B2
:10FA30001723FFFF6700436A832709009399140087
:10FA4000CE9703D50700330745014207418363641E
:10FA5000570305C103270B0019C785453E8597400D
:10FA60000000E78060E9832709000504CE97239012
:10FA7000070085047DB797000000E78060A2832718
:10FA800009000504CE972390070065D5814597F0BE
:10FA9000FFFFE780C0BEF1BF1723FFFFE7028360CF
:10FAA00083C7950041112A8A93F7F707A384F500CD
:10FAB00032852E89328497C0FFFFE780005E93175E
:10FAC0000501C187635AF004AA89832A040097A01C
:10FAD000FFFFE780E05C31E5835744008544014443
:10FAE000F11793B71700A301F10003483100D6873F
:10FAF00052850147CE862686CA8597D0FFFFE780CC
:10FB0000806AA167F50748003EC42302910022C61F
:10FB100097D0FFFFE780402F41011723FFFF6700C9
:10FB2000A35BA2851306310097E0FFFFE780602901
:10FB30002A8489445DD99767FF1F9387675E9C433A
:10FB400081CF044997B0FFFFE780E055AA8526855D
:10FB500097400000E78040DA130504019700000099
:10FB6000E780C0EA228597800000E7800033814467
:10FB7000ADBF1723FFFFE702035283C79500411172
:10FB8000AA8A93F7F707A384F5003285AE893284F9
:10FB90002311010097C0FFFFE78020509317050154
:10FBA000C1876354F0062A8AC145228597C0FFFFAA
:10FBB000E7804035AA8B5285032B040097A0FFFFF6
:10FBC000E780004E21E98357440085440144F11742
:10FBD00093B71700A300F100034811000357210059
:10FBE000DA875685D2862686CE8597D0FFFFE780B6
:10FBF000805BA1679387270248003EC423029100DF
:10FC000022C697D0FFFFE780202041011723FFFF86
:10FC10006700E34BA2851306110097E0FFFFE78022
:10FC2000401A2A8489444DD99767FF1F9387474F0D
:10FC300098433E8901CF044997B0FFFFE780A04673
:10FC4000AA85268597400000E78000CB13050401B4
:10FC500097000000E78080DB97B0FFFFE780A044BB
:10FC600095443DD9930521005E8597F0FFFFE7801D
:10FC700060B6AA8435F11C480357210022852390E1
:10FC8000E70097800000E780402183270900A9D77B
:10FC90000355210097400000E780A0BD35BF172322
:10FCA000FFFFE702433F83C795004111AA8A93F7FC
:10FCB000F707A384F5003285AE89328497C0FFFF31
:10FCC000E780A03D93170501C1876351F0062A8A9A
:10FCD000228597C0FFFFE780403C2A895285032B8D
:10FCE000040097A0FFFFE780A03B31E58357440065
:10FCF00085440144F11793B71700A301F1000348AD
:10FD00003100DA8756854A87D2862686CE8597D0F7
:10FD1000FFFFE7804049A167F90748003EC423027E
:10FD2000910022C697D0FFFFE780000E4101172304
:10FD3000FFFF6700C339A2851306310097E0FFFF7C
:10FD4000E78020082A8489445DD99167CA97C20751
:10FD50001167C1831307F7EF8544E362F7FA9767EA
:10FD6000FF1F9387E73B9843BE8B01CF044997B0B1
:10FD7000FFFFE7804033AA85268597400000E78093
:10FD8000A0B71305040197000000E78020C897B0D2
:10FD9000FFFFE780403195443DD11C4822858144D6
:10FDA0002390270197800000E780200F83A70B0096
:10FDB000B9D74A8597400000E780A0AB89B71723E1
:10FDC000FFFFE702C32F2A844105B2849700000099
:10FDD000E780C0C311C5228597800000E780E00B53
:10FDE00081460146A685228597800000E780C04EA7
:10FDF0001C4C89C7DC4799C3228582971723FFFFD4
:10FE00006700232E9767FF1F938787129C43014546
:10FE100099C31385070182809767FF1F9387471156
:10FE2000884382801723FFFFE70263299317C600E8
:10FE3000DD8DC2054111C1812A8432C697C0FFFF02
:10FE4000E780E0173246228511829375F60F97C03E
:10FE5000FFFFE780C01441011723FFFF67006328FD
:10FE60001723FFFFE702032479713C083ED2B7074E
:10FE70000C003ED43C083ED683C79500AE842A8948
:10FE800093F7F707A384F500A1659385350448101F
:10FE900097A0FFFFE780E02BC165FD150144176ABD
:10FEA000FF1F130A6A29930A400EAE892E8B2EC6B5
:10FEB00097B0FFFFE780202242059317040141819C
:10FEC000C183B24563E9A702C167FD176387F500E7
:10FED000481097C0FFFFE780800E50100147814611
:10FEE000A6854A8597A0FFFFE780004C4561172350
:10FEF000FFFF6700631E3307540383270A0BBA977B
:10FF000003D6C701630A3601638A3501481097009A
:10FF10000000E78060F1DA85050451BFB285EDBFCE
:10FF20001723FFFFE702231779717C083EC8B70744
:10FF300011003ECA7C083ECC83C79500AA89328551
:10FF400093F7F707A384F5002E8997C0FFFFE7809A
:10FF5000C01485676378F504A165AA84890508083B
:10FF600097A0FFFFE780E01E268597400000E7800E
:10FF700060ED133415000A04A285080897C0FFFF3E
:10FF8000E780E001A685080897C0FFFFE78020030F
:10FF900025CC014781461008CA854E8597A0FFFFF2
:10FFA000E780804045611723FFFF67004312B307D6
:10FFB00054030327CA0ABA9703D70700631C9700A4
:10FFC00003D6270063806505080897000000E780D6
:10FFD000A0E5DE8505042EC697B0FFFFE780A010E0
:10FFE0004205931704014181C183B245E3E1A7FCB7
:10FFF000C167FD17E38FF5F8080897C0FFFFE7809A
:020000040001F9
:1000000000FC41BFB285F9B7C165FD150144176A0F
:10001000FF1F130A6A12930A80022E8BAE8B65BFF4
:100020001723FFFFE702A309184183471700834600
:100030000700A207D58FD207D1832390F50083470D
:100040002700034717008D45A207D98F91832310FE
:10005000F60097C0FFFFE780A0E91723FFFF6700C6
:1000600043081723FFFFE702E303C1640144176954
:10007000FF1F1309690C93098002FD1497B0FFFF5D
:10008000E78060066347A40001451723FFFF670070
:10009000A304330534038327C90A3E95835705001B
:1000A000E38597FE0504D9BF1723FFFFE70283FF0F
:1000B0002A8AAE89B284B68A97400000E78080D849
:1000C00019E591473E851723FFFF6700E3002A8962
:1000D0004E8597C00000E780E08E2A84638E0A0474
:1000E0008D476DD103570500C547E31D47FD034705
:1000F000F9018546AD47E317D7FC8347450081CF1B
:100100004146A6855D0597F00000E780C09E8147C7
:1001100055D9AD4745BF130965012302E500CA85DE
:10012000268597100000E780606231C1A547E38B08
:100130000AF82302040079B705C183570500E3924A
:1001400047F94146A685190597F00000E780A09A77
:1001500081472DD99947BDB74E8597000000E780AC
:1001600080F02A84954739DD130955004DBF41467B
:10017000A68523104401231134011305190097F0BB
:100180000000E780A099228597800000E780A0EA20
:1001900081470DBF1723FFFFE70263F279717C00EF
:1001A0003ECCB7070A003ECE7C003ED083C7950008
:1001B000B2842E8493F7F707A384F5001306A100F9
:1001C0002A892C00268597000000E780A0E5A1651C
:1001D00028088D0597A0FFFFE780A0F79040835582
:1001E000A10003558100854697000000E78000ECE0
:1001F000AA84AA85280897C0FFFFE78040DA035643
:10020000A10083558100280897000000E780C0C145
:10021000300801478146A2854A8597A0FFFFE78005
:10022000A018854748103ED42302910202D697D0E9
:10023000FFFFE78060BD45611723FFFF670063EAAA
:100240001723FFFFE702A3E779717C003ECCB707D5
:100250000A003ECE7C003ED083C79500B2842E8437
:1002600093F7F707A384F5001306A1002A892C0051
:10027000268597000000E780E0DAA16528088D0553
:1002800097A0FFFFE780E0EC90408355A100035565
:100290008100814697000000E78040E1AA84AA859A
:1002A000280897C0FFFFE78080CF0356A100835541
:1002B0008100280897000000E78000B73008014758
:1002C0008146A2854A8597A0FFFFE780E00D481090
:1002D0002302910202D402D697D0FFFFE780C0B27A
:1002E00045611723FFFF6700C3DF1723FFFFE70206
:1002F00003DD97000000E78060DB1723FFFF670046
:1003000043DE9767FF1F9387E7C2884382801723E6
:10031000FFFFE702C3DA835725004111AE842A8428
:100320002307B10017F5FFFF130525466C002316C0
:10033000F10097A0FFFFE780204991C422859780B4
:100340000000E780E0D6FD572310F40013062002DA
:100350008145130554009720FFFFE78040D94101F4
:100360001723FFFF6700E3D71723FFFFE70283D3BD
:1003700079717C003ECCB7070A003ECE7C003ED0AF
:1003800083C79500AA89AE8493F7F7073285A384C3
:10039000F5001306A1002C0097000000E78080C83C
:1003A00003558100114497400000E780A0A915C5BE
:1003B0000355A100014497B00000E780A06011CD73
:1003C000035705008357810045446318F7008545AE
:1003D00097000000E780E0F30144216993053900AC
:1003E000280897A0FFFFE780C0D6A285280897C0FD
:1003F000FFFFE780C0BA0356A1008355810028089B
:1004000097000000E78040A2300801478146A6859A
:100410004E8597A0FFFFE78020F948104AD42302B9
:10042000810202D697D0FFFFE780009E4561172327
:10043000FFFF670063CA1723FFFFE702A3C69767A2
:10044000FF1F9387E7AE2A8488432E8915C503577B
:1004500045038357C4016311F702232605022318BD
:100460000502410597D00000E780209C6306090043
:1004700097800000E78060DB81449769FF1F9389C4
:10048000A9CB130A800297B0FFFFE780C0C563C401
:10049000A4049767FF1F938767B29C4399C70355CE
:1004A000C40197200000E780C0BD630709002285D2
:1004B00097800000E780C0A01306400E814522858A
:1004C0009720FFFFE780A0C2FD57231EF4001723EB
:1004D000FFFF670063C03385440383A7C90A3E95C5
:1004E000035705008357C4016317F700CA859700B7
:1004F0000000E78000E2850479B71723FFFFE702D9
:1005000063BA83C795004111AA8993F7F707A384BB
:10051000F5003285AE8497C0FFFFE78000B885679D
:100520006378F5042A8997400000E780A091014490
:1005300001CD83D7040031446388270185459700A6
:100540000000E78080EF01444E85A2864A86A6859A
:1005500097D0FFFFE780A09CA1679387170448000E
:100560003EC42302810002C697D0FFFFE780C08906
:1005700041011723FFFF670023B61723FFFFE702A0
:1005800063B29767FF1F9387A79A804329C40145E9
:1005900097C00000E780002181470148C1641CDC4E
:1005A000232E0403232004041769FF1F1309C9B86D
:1005B00001449309400EFD1497B0FFFFE780A0B1FE
:1005C000634FA400814517F5FFFF1305857F97A0B2
:1005D000FFFFE780601F1723FFFF6700E3AF3305CE
:1005E00034038327090B3E958357C5016387970022
:1005F000854597000000E78040E4050475BF9357E8
:10060000050113D78700A380F50093170501C18367
:10061000A1832380E5002381F500A381A5008280CA
:100620001723FFFFE702A3A92300050083C71500D6
:10063000A300F50083C725002301F50083C735001B
:10064000A301F50083C745002302F50083C75500C9
:10065000A302F50083C7650093059500A303050079
:100660002303F50023040500328597000000E7808E
:1006700040F91723FFFF6700C3A61723FFFFE70218
:1006800063A24111E9540DCD85CD93F9C5FF2E84A8
:100690002A89AA84338AA900B7EA040063189A0257
:1006A0000D88854411CCB7E704009C5F82972AC669
:1006B00022866C003305390197E00000E780004690
:1006C000268541011723FFFF670003A183A78A0343
:1006D0009104829793170501C183A183A38EF4FE31
:1006E00093570501238FF4FEA183238EA4FEA38FCD
:1006F000F4FE6DB763E6D5021723FFFFE702239CE4
:10070000B28741113686BE8536C697E00000E78085
:10071000E040B246410136851723FFFF6700639C26
:10072000814636858280838705001387F5003D0565
:10073000FD8793F77708834607007D158606B58FFA
:10074000A300F5006307B7007D17834717009D835B
:10075000DDB782801723FFFFE7026396B7E7040047
:1007600083A7070932872A863A85829713351500B1
:100770001723FFFF6700E39615C181478DC117233B
:10078000FFFFE702C393414697E00000E78000398E
:1007900085473E851723FFFF6700A39481473E8569
:1007A00082801DCD1723FFFFE702639141468145FB
:1007B0002A849720FFFFE7808093414681451305F7
:1007C00004039720FFFFE78080920147C16723223F
:1007D000040438C87CC805451723FFFF67006390F1
:1007E0000145828081473DCDB5CD1723FFFFE7024C
:1007F000038DB2842E891306800581452A849720B3
:10080000FFFFE780C08ECA8524C4268597000000BC
:10081000E780C0F64146814522859720FFFFE780AB
:10082000008D3044A285228597000000E780C0F249
:1008300093040401A285268597000000E780E0EE7E
:10084000A6851305040297000000E78000EE2285CC
:1008500097000000E78020F585473E851723FFFFBE
:10086000670023883E8582801723FFFFE70283838A
:100870004111E9540DCD85CD93F9C5FF2E842A8908
:10088000AA84338AA900B7EA0400639844030D8858
:10089000814411CCB7E704009C5F82972AC6228668
:1008A0006C003305390197E00000E780202726859A
:1008B00041011723FFFF6700238283A78A03910466
:1008C000829793170501C183A183A38EF4FE9357EA
:1008D0000501238FF4FEA183238EA4FEA38FF4FED3
:1008E0006DB765CD1713FFFFE702C37BB28411E636
:1008F00005451713FFFF6700237E2A842E890145D3
:10090000EDD93C487848B3E6E700E5D69386F7FF93
:10091000B3B7F6007D17032A4404BA9734C87CC8DD
:1009200063050A06C14913050A03B38949412295A3
:10093000637D3601B2862E86A68597000000E7808B
:10094000A0DB7C40BE9464C065B7CE862E86CE8583
:1009500097000000E78040DAC114D2944E99232218
:100960000404A2879306040103C7070003C6070314
:100970008507318FA38FE7FEE398F6FE3044A2850A
:10098000228597000000E78020DD2699C1493306C3
:10099000994063EC9900A9DCA686A685130504039B
:1009A00097000000E78040D579BF8147B306F40087
:1009B0003307F6000347070083C5060085072D8F20
:1009C0002380E600E39437FF3044A2852285970018
:1009D0000000E78060D8C1145DBF014582800DC171
:1009E0001713FFFFE702A36D1306800581459710DB
:1009F000FFFFE780C06F05451713FFFF6700636EB9
:100A000001458280814749C5C1C51713FFFFE70231
:100A1000036BFC4141462E84AA846399C704138664
:100A20000501A2878146C14503C7070003C5070327
:100A30008507298F3305D600034505008506298FD4
:100A4000A38FE7FEE392B6FE3044A2852685970089
:100A50000000E78060D0228597000000E78060F802
:100A600085473E851713FFFF6700A36713850703BC
:100A70001D8E814522959710FFFFE78040677C40DF
:100A8000130700F813060402A2972388E70251BF58
:100A90003E8582801713FFFFE70263626D712E842B
:100AA000B284AA8590102800368997000000E7805C
:100AB000A0D309EDD55725A050400C402800970041
:100AC0000000E78040E27DD5FD142104F5F42C0000
:100AD0004A8597000000E78020F3814761DD3E856D
:100AE00051611713FFFF6700C35F1713FFFFE70292
:100AF000035D41112EC432C62C000546970000004C
:100B0000E78080F941011713FFFF6700835D17132A
:100B1000FFFFE702C35A01112A842EC602C802CA87
:100B200002CC02CE97E00000E780E032B2462A868F
:100B3000A285080897000000E78060FB1375F50F99
:100B400005611713FFFF6700C3591713FFFFE70283
:100B500003577971B2872A8421462308B10013050F
:100B60001101BE853AC436C697E00000E78000FB5D
:100B7000B24693059101368597000000E78060A892
:100B80002285141035460C0897000000E78020F6F7
:100B90002A84224701E921460C103A8597E000009B
:100BA000E780C0F7228545611713FFFF6700635395
:100BB0001713FFFFE702A3507171AE84AA850A855F
:100BC000328497000000E78060BB11C90A86A685C1
:100BD000228597000000E78020B8814711E1C547D2
:100BE0003E854D611713FFFF6700A34F1713FFFFEB
:100BF000E702E3491D712A8AB289BE8435468547DA
:100C0000130511012E8CB68A3A8BC28C468D2308AF
:100C1000F10097E00000E78060F010100C085285AA
:100C2000231F010097000000E780C0F82A843DEDF3
:100C3000A1476313FD089307900591E0E54735460A
:100C4000E2851305110113990A012308F1001359D4
:100C5000090197E00000E78060EC13578900939743
:100C60008A00D98F90080C085285231FF100970045
:100C70000000E78020F42A8415E9A1E49387FA00B4
:100C800091831379F9003EC6631309004149668BCD
:100C90008144C14B854DB247639F970C6A868C0097
:100CA00033855C0197E00000E78040E722852561FD
:100CB0001713FFFF6700634193079004C9F0A5472E
:100CC000BDBF834701050947C14B2308F100834796
:100CD0001105A58FA308F10093872400814463E1E7
:100CE000FB04014714083386E6008C08B386E40051
:100CF000BA95DA9683C6060083C505000507AD8E52
:100D00002300D600E390E7FE4147639CE704900888
:100D10000C08528597000000E780C0E925D181A02A
:100D2000B3069B00BA871008B305F60090083E96FC
:100D300003C506000346060085078506298E238025
:100D4000C500E39277FF998F90080C085285BE94F6
:100D500097000000E78000E68947014749D12A84CF
:100D6000B1B790083E96034606001408BE9623804D
:100D7000C600850759BFB24785046387971481472A
:100D80001808B306F70098083E973386F900034722
:100D90000700034606008507318F2380E600E391B4
:100DA00077FF90080C08528597000000E78080E0EC
:100DB0005DF53546E285130511012308B10197E081
:100DC0000000E780A0D51397040141839397840026
:100DD0002183D98F10180C085285231FF10097002A
:100DE0000000E78020DD25FD814710183387F900DA
:100DF0003E960347070003460600B306FB0085073F
:100E0000318F2380E600E39277FF65A81808B306C8
:100E1000F70098083E973386F9000347070003461A
:100E200006008507318F2380E600E3E127FFCA87AC
:100E3000639E770990080C08528597000000E780B0
:100E400060D711FD81479800B306F700900818108D
:100E50003E973E9603470700034606008507318FFD
:100E60002380E600E39177FF3546E2851305110103
:100E70002308B10197E00000E78040CA13970401FE
:100E80004183939784002183D98F10180C085285D1
:100E9000231FF10097000000E780C0D1E31105ECAB
:100EA000814710183387F9003E9603470700034631
:100EB0000600B306FB008507318F2380E600E3E2DE
:100EC00027FFC109410BC1BB814785B79408BE9676
:100ED00083C6060018083E972300D700850789BF00
:100EE000638006321713FFFFE702631A59712A84E1
:100EF000BE89B28B85473546130511022E8B468C71
:100F00004289BA8A368A2300F10297E00000E7801E
:100F1000E0C010180C102285231701029700000072
:100F2000E78040C963180512A147631FFC069307B9
:100F3000900563930900E5473546DA8513051102EC
:100F400093140A012300F102C18097E00000E780BA
:100F5000E0BC93178A0013D78400D98F90080C1037
:100F600022852317F10297000000E780A0C47DE1ED
:100F7000639209049307FA00BD88918391E0C1440C
:100F8000C207C183DE8C814A3EC6414DB24763E24F
:100F9000FA0E6286B3854B01881097E00000E78067
:100FA00080B54DC93D557DA093079004E39609F89F
:100FB000A54759B7834701050947C14C2300F102F2
:100FC00083471105B3C7F900A300F10293872900F5
:100FD000814963E1FC04814618103306D7008C0870
:100FE0003387D900B69556970347070083C5050098
:100FF00085062D8F2300E600E390D7FE41476390DE
:10100000E70690080C10228597000000E78080BA60
:1010100035D189A0B3863A01BA871010B305F6001E
:1010200090083E9603C50600034606008507850620
:10103000298E2380C500E39297FF3387EC40900808
:101040000C102285BA9997000000E780A0B6894766
:10105000014741D165611713FFFF6700030790083F
:101060003E96034606001410BE962380C6008507F0
:1010700079B7B247850A93990A01939D8A0093D95B
:1010800009016391570F85473546DA85130511022B
:101090002300F10293D9890097E00000E78000A8BF
:1010A000B3ED3D0190000C1022852317B10397008A
:1010B0000000E78020B059FD8147A68963EA9706C2
:1010C00026860C084A8597E00000E78020A5814726
:1010D0001810B306F700100898083E973E9603478D
:1010E0000700034606008507318F2380E600E3E111
:1010F00097FE639FA90590080C10228597000000B9
:10110000E78040AB21F981479810B306F7009008BB
:1011100018183E973E9603470700034606008507CA
:10112000318F2380E600E391A7FF4109C10CB9BDCF
:1011300018089000B306F7003E963387FC0003477B
:101140000700034606008507318F2380E600B5B708
:1011500098084E97034707001C10CE972380E7009E
:10116000850941BF85473546DA85130511022300FD
:10117000F10293D9890097E00000E780209AB3ED4F
:101180003D0190000C1022852317B1039700000049
:10119000E78040A2E31005EC814718089000B306F1
:1011A000F7003E963387FC0003470700034606001E
:1011B0008507318F2380E600E391A7FF41460C08A5
:1011C0004A8597E00000E780609581471810B306D4
:1011D000F700100898083E973E960347070003461D
:1011E00006008507318F2380E600E391A7FF900872
:1011F0000C10228597000000E780C09B1DD599BD8B
:101200007D5582801713FFFFE70263EB01112A84EB
:101210002E8593055100328902C002C202C402C663
:101220009304740097F0FFFFE780A03D1D46A6855C
:101230001305910097E00000E780408E10088A8532
:101240004A8597000000E780E09619ED93071400A7
:10125000180883C607000346070085070507B18EF7
:10126000A38FD7FEE397F4FE05611713FFFF670016
:1012700043E71713FFFFE702E3E22E848C4141119D
:10128000AA89838715003289914463D30700A1445A
:101290009757FF1F9387C7209C43A1C7C1CA8D479B
:1012A0002310F10083C725004A852301F10083C77D
:1012B0003500A301F10083C745002302F10083C775
:1012C0005500A302F10083C7650093059100A303B5
:1012D00001002303F1002304010097F0FFFFE780E2
:1012E00040320C404A860A8597F0FFFFE780803342
:1012F0000328040083564400A6881D08814701473F
:10130000E51642868A854E8597000000E780408E6C
:101310002A8919E5A685228597B0FFFFE780E0C1FD
:101320004A8541011713FFFF670003DB4A860A85E0
:1013300097F0FFFFE780002F6DB71713FFFFE7025D
:1013400063D62E848C414111AA8983871500328986
:10135000914463D30700A1449757FF1F9387471415
:101360009C43A1C7C1C68D472310F10083C7250048
:101370004A852301F10083C73500A301F10083C72B
:1013800045002302F10083C75500A302F10083C783
:10139000650093059100A30301002303F1002304DA
:1013A000010097F0FFFFE780C0250C404A860A85C0
:1013B00097F0FFFFE78000278356440003280400CE
:1013C0008A85858EC2061D08C1822312D400A68894
:1013D00081470147E51642864E8597000000E78069
:1013E00060B041011713FFFF670003CF4A860A85EB
:1013F00097F0FFFFE78000234DBF1713FFFFE702C1
:1014000003CCB335B000011185052A891315F60107
:10141000336515012308B1009305110136843AC6DE
:1014200032C03EC442C297F0FFFFE780801DA24752
:101430001248425593D68700230BF1009305910182
:1014400093578800A30AD100A30BF100230C0101DC
:1014500097F0FFFFE780E01A3247024603280400B6
:10146000B337E000835644009207914411C2A1446F
:101470004A85A68842860C0897F0FFFFE7804077F0
:101480002A8919E5A685228597B0FFFFE780E0AAA3
:101490004A8505611713FFFF6700A3C41713FFFFF9
:1014A000E70243C001113EC68647B335B00085054B
:1014B000AA891315F6015D8D2308B100930511016A
:1014C00036843A89B28442C446C297F0FFFFE7806F
:1014D000401322489248164593578800A30AF1000A
:1014E0009305910193D78800230B0101A30BF10011
:1014F000230C110197F0FFFFE780A0103247104046
:1015000083564400B337E00092070328090091484E
:1015100091C0A1480C084E8597000000E780809C90
:10152000AA8401E9835544004A8597B0FFFFE7800C
:10153000C0A0268505611713FFFF6700E3B9AA95D0
:101540009307F00F171701001307C7F16317B500D2
:1015500013C5F7FF1375F50F828005058346F5FF68
:10156000B58FBA9783C70700D5B703574500144115
:101570009307F00F171601001306C6EE36974207C1
:101580004183139506014181631BE500AD8FB2973E
:1015900003C50700130515F3133515008280850672
:1015A00003C5F6FFA98FB29783C70700D9BF1713EA
:1015B000FFFFE702C3B0B28736842E86BA86AA85BB
:1015C0003E85BA8497F0FFFFE7806052634F0500C5
:1015D000228597E00000E78000882A86A686A285FB
:1015E000268597F0FFFFE78080501713FFFF670005
:1015F00043AF1713FFFFE702E3AA5D712A8BAE8AA0
:1016000017150100130585E32C00B284368ABA89C8
:101610003E8997F0FFFFE780C04F2A845DE13410D8
:101620004146DA85280097F0FFFFE780404C2A8486
:1016300049E98547A303F100A6C293077100240876
:10164000BEC4A68685470D462C18281002DC02DE93
:10165000D6C0BEC697F0FFFFE78000442A8435E17C
:1016600083477102A6860D4693F7F7072300FA0019
:10167000C1473EDE2C188947281026DCA303F10061
:1016800097F0FFFFE78040412A8405ED4146A6859B
:101690004E8597D00000E78060488D47A6860D46AE
:1016A0002C182810A303F10097F0FFFFE780C03E3D
:1016B0002A8401E94146A6854A8597D00000E78043
:1016C000E045228561611713FFFF6700E3A0171350
:1016D000FFFFE702C39E97F700009387E712984346
:1016E00083C7470079712A89AE8417150100130555
:1016F00065D50C083AC42306F10097F0FFFFE78098
:1017000040412A8405ED14104146CA85080897F027
:10171000FFFFE780C03D2A8415E1140815462C0020
:10172000081097F0FFFFE780803C2A8401E92146FA
:101730002C08268597D00000E780403E2285456131
:101740001713FFFF6700E3991713FFFFE7022397C3
:1017500097F700009387470B9C477971AA842E84E2
:1017600017150100130585CE0C083EC697F0FFFF44
:10177000E780203A0DE914104146A685080897F045
:10178000FFFFE780C03605E1140811466C00081021
:1017900097F0FFFFE780A03519E58347F10193F744
:1017A000F7032300F40045611713FFFF67006393FD
:1017B0001713FFFFE702A3903688A148814701472E
:1017C000E54697F0FFFFE780A0421713FFFF670091
:1017D00043911713FFFFE702838E3688A1488147A4
:1017E0000147E54697F0FFFFE780C06F1713FFFF43
:1017F0006700238F1713FFFFE702638C01112A8410
:101800002E850C0832C697F0FFFFE780803009ED87
:101810003247971601009386E6C11008C14522851C
:1018200097000000E780E0D805611713FFFF67000D
:10183000438B1713FFFFE70283884111C1472EC076
:1018400032C48A8509463EC23EC697F0FFFFE78054
:10185000A02441011713FFFF6700A3881713FFFFA0
:10186000E702E3854111AE8613061009AA850A85B1
:1018700002C002C202C402C697F0FFFFE780202721
:1018800041011713FFFF6700C3851713FFFFE7022E
:1018900003833287971601009386C6BB2E86930575
:1018A000000297000000E780C0D01713FFFF670019
:1018B00043831713FFFFE70283807971C1472ACC66
:1018C0002ED032D42C080D4628003ECE3ED23ED635
:1018D00002C402C602C802CA97F0FFFFE780C01B1D
:1018E00045611703FFFF6700C37F1703FFFFE70290
:1018F000037D0111AA842E8417150100130505B676
:101900008A8597F0FFFFE780C02015E5140841465F
:10191000A6850A8597F0FFFFE780601D09ED8347E4
:10192000E1010347F101A207D98FCA07C983617793
:10193000D98F2310F40005611703FFFF6700637A56
:1019400015CD1703FFFFE70283779747FF1F9387A4
:10195000E76290439745FF1F938585621745FF1FF8
:101960001305C55D97D00000E78000C51745FF1F30
:101970001305C55C1703FFFF6700A3761745FF1F1C
:101980001305C55B82808DCD1703FFFFE70223732C
:101990009747FF1F9387875E944301112E840A8621
:1019A0009745FF1F9385C55D97D00000E78040C62F
:1019B0000A850294014505611703FFFF6700637202
:1019C0007D5582801703FFFFE702636F97D0000009
:1019D000E78080D19747FF1F23A2A75A17F5FFFF83
:1019E0001305E5C997B00000E780C0741703FFFF37
:1019F0006700236F1747FF1F1307875A93171500B8
:101A000008433E95FD572310F50082801703FFFF22
:101A1000E702E36A2A84084009E51703FFFF67002D
:101A2000436C1C4158401CC06313E5005CC08347F5
:101A3000550023200500F99BA302F50097A0FFFFA6
:101A4000E780207CC9BF1703FFFFE702A365974724
:101A5000FF1F9387E75698432A8411CB83473500AD
:101A600093F7070289C703550500894502971305B7
:101A7000440197B00000E780403B835504000355C4
:101A8000E40097300000E780A00C485819C597A0E3
:101A9000FFFFE7800077232A0402130584039700E1
:101AA0000000E780E0F68144B1499790FFFFE780AE
:101AB000C06D63CBA402834734002320040493F752
:101AC00027FCA301F40000489790FFFFE780E06C3B
:101AD00013161500814522859700FFFFE7802061DE
:101AE0001703FFFF6700435FB38734030329040331
:101AF00085043E994A8597000000E78060F1230441
:101B0000090065B78347350093F7070299E301455C
:101B100082808357E500E39CB7FEC167FD1763161B
:101B2000F60005458280054599A81703FFFFE702E7
:101B3000035993170601C187B2842A840149635966
:101B4000F002835705009DCB01456367F60003450E
:101B500084003E953325A6001375F50F0DA01C4893
:101B600013171900BA9783D70700E38E97FA050970
:101B70009790FFFFE7806062E343A9FE01451703EA
:101B8000FFFF670003561703FFFFE702A351AE896B
:101B9000AA849790FFFFE78000562A8497D0FFFF22
:101BA000E780A02EAA86014713068401970500004E
:101BB000938585E41745FF1F1305C53E9790FFFFEA
:101BC000E780801C2A8925C98C441304C50022851E
:101BD0009E0593F5050897A0FFFFE780403CCC40A9
:101BE00083877400E18163DD070493E5050822859E
:101BF00097A0FFFFE780A03A0D4693854400228519
:101C000097A0FFFFE780C03683D50400228597A008
:101C1000FFFFE780E03D83D52400228597A0FFFFEA
:101C2000E780003D03D6490083A50900228597A0DF
:101C3000FFFFE780E0334A851703FFFF6700C349D2
:101C400093F5F5076DB71703FFFFE702434701114F
:101C50002A84328532C697A0FFFFE780E02797806D
:101C6000FFFFE7806034835704001747FF1F130707
:101C7000A74C3246231BF100930700F8A30DF10097
:101C80001C471843231AA1008983858BB307F740AB
:101C9000B28548083ECE231C0100230D01009700A9
:101CA0000000E78080EE05611703FFFF67006343D4
:101CB0001703FFFFE702033F004101453DC49304C2
:101CC000C40026853289AE8997A0FFFFE780C02433
:101CD00095452A8A2685035B040197A0FFFFE780CC
:101CE0002021268597A0FFFFE780603E8D45AA8AC8
:101CF000268597A0FFFFE780A01F268597A0FFFFFE
:101D0000E780E03C5C48420A135A0A01D2975CC45F
:101D100023186401814763983A0146054D813306D3
:101D200025419337160013F5F70F1703FFFF6700E0
:101D3000A33A1703FFFFE702033689692A8BAE8BAC
:101D4000328AB68A81440144314CFD199790FFFFD5
:101D5000E780A04363CDA4009790FFFFE780E045B4
:101D6000018D33B5AA001703FFFF6700433633899F
:101D7000840383270B003E9963170A008347890079
:101D800085043E94E1B703560A00DE854A8533F6A2
:101D9000C90097000000E780E0F16DD10545E1B78B
:101DA0001703FFFFE702A33101112A847C000355CA
:101DB000E5003ECAB70707003ECC7C003ECE972028
:101DC0000000E78020082A898545480897A0FFFF82
:101DD000E78020399945480897A0FFFFE780E01584
:101DE000AA844A8597200000E780A0082380A400E9
:101DF0009747FF1F938747349C434166130606F0BD
:101E00009396870113D78701558F93D68700F18E5C
:101E1000558FA207B706FF00F58FD98F11462C000A
:101E2000138514003EC497D00000E78020CF5008EF
:101E3000A38204008945228597000000E780E0E046
:101E400019C9AA851305840397A0FFFFE780E03135
:101E50003C4085073CC005611703FFFF670063280E
:101E60001703FFFFE702A3259790FFFFE780E03409
:101E70002A8405049790FFFFE78020333305A402EE
:101E8000F14791453305F50297200000E78020BA1D
:101E900011E565551703FFFF6700A3249747FF1F50
:101EA00023A8A7109790FFFFE78020312A8405041C
:101EB0009790FFFFE780602F3305A4028945060550
:101EC00097200000E780A0B669D59747FF1F23A998
:101ED000A70C9790FFFFE780402E2A840504979077
:101EE000FFFFE780802C3304A4029747FF1F239B4A
:101EF000870A9790FFFFE780402C2A849790FFFF86
:101F0000E780A02A930714003385A7029747FF1F95
:101F1000239BA70897070100938707181747FF1F00
:101F20002326F7080145BDB71703FFFFE702831714
:101F3000AA842E8901449749FF1F9389E91F130A38
:101F400080069790FFFFE78040266347A400014585
:101F50001703FFFF670043183305440383A70902F3
:101F60004A86A6853E9597000000E780E0B919E112
:101F70000504C1BF0545E9BF1703FFFFE702A31131
:101F8000AA8A2E8BB28B368C3A8A814401448149CD
:101F9000974CFF1F938C4C1A130D80069790FFFFF0
:101FA000E780A02063C9A40011E085494E8517038E
:101FB000FFFF6700C3113389A40383A70C025E8669
:101FC000D6853E994A8597000000E780E0B31DC1A1
:101FD0009790FFFFE780601E0544636D4501D28640
:101FE0006286DA851305090397000000E780A0D414
:101FF00011C1854985045DB71703FFFFE702830A16
:10200000C16441112A8901449749FF1F9389C9126C
:10201000130A8006FD1436C632C42EC29790FFFF05
:10202000E780A01892452246B2466348A4000145C5
:1020300041011703FFFF6700230A3305440383A709
:1020400009023E9509C683473500C18B9DC791C6DD
:102050008347350093F707028DC3630699008357C2
:10206000E500639C27010357050001CB63E7E5000A
:1020700083478500BA97E3CDF5FA050469BF1703D6
:10208000FFFFE7022302C1642A8901449749FF1F29
:102090009389890A130A8006FD149790FFFFE78051
:1020A000C0106346A4001703FFFF6700E302330577
:1020B000440383A709023E958357E500638A97008E
:1020C000630499006396270197000000E780E0977A
:1020D0000504E1B71703FFFFE70263FB89692A8A5A
:1020E000AE8A328BB68B8144174CFF1F130CCC0485
:1020F000930C8006314DFD199790FFFFE780E00AB1
:1021000063C6A4001703FFFF670023FC3389940311
:1021100083270C028355CA015A863E994A85970047
:102120000000E780609E31C1814D15A03384AD036E
:102130008327090303D60B00D68533F6C9003E94E6
:10214000228597000000E780E0B609E9850D9790A9
:10215000FFFFE7808003E3CBADFC01A82285970059
:102160000000E780E08A23040400850471B71703A8
:10217000FFFFE70243F24169AA8A014A174BFF1F9A
:10218000130B8BFB7D19C14B054C9790FFFFE7802C
:10219000C0016346AA001703FFFF670043F39309DA
:1021A0008006B3073A0383290B02BE9983D7E9005F
:1021B000638E270163842A01639A570103A489036C
:1021C00001E84E8597000000E780C0BD050A75BF95
:1021D00083570401639977099304C400268597A067
:1021E000FFFFE78060D385452A8D2685835C040147
:1021F00097A0FFFFE780C0CF268597A0FFFFE7806D
:10220000A0E762056185635905048D45268597A081
:10221000FFFFE780E0CD8945268597A0FFFFE78097
:1022200020CD8945268597A0FFFFE78060CC8545B6
:10223000268597A0FFFFE780E0CC8347050009478C
:1022400093F7F707639AE7009945268597A0FFFF64
:10225000E78040CBA30285014848337D2D01231838
:1022600094016A9548C40040A1BF1703FFFFE7022D
:1022700003E537E404008327041D82979747FF1F77
:1022800083C787D81715FF1F13050528A300F5007E
:102290008327441C82978327841C81461306F00FF2
:1022A0008145014582971703FFFF670083E31747C6
:1022B000FF1F130767C518439745FF1F83C5C5D484
:1022C0009747FF1F9387C7D2834687030346970329
:1022D0006397D5009747FF1F2388C7D2828083C5A5
:1022E00087010347A7036317B6009747FF1F238D96
:1022F000E7D0828003C687016317C7009747FF1F97
:102300002384D7D0828083C68701130750026319C4
:10231000D700930760021747FF1F2307F7CE82807D
:1023200083C68701130660026315D6009307700207
:10233000DDB783C7870155BF9747FF1F938747CBFB
:10234000D44B0947638DE6081703FFFFE70223D745
:102350001749FF1F130909C73E8483470900918B62
:102360009DCFB7E4040083A7041D829783A7441C74
:102370001745FF1F130585C5829783A7841C8146D7
:102380001746FF1F034686C681450145829721C532
:1023900083470900ED9B1747FF1F2305F7C28347BB
:1023A000040093F7F70F85CB91471747FF1F232BA7
:1023B000F7C497000000E78080EB97000000E780FB
:1023C00040EFB7E70400BC4F414691451745FF1F5A
:1023D000034585C282971703FFFF670083D0828081
:1023E0001703FFFFE702A3CD8D4741116306F504F4
:1023F000C5476308F50285476310F5029747FF1F3D
:102400002386A7C0B7E70400BC4B9305001017450F
:10241000FF1F034565BE829741011703FFFF670059
:1024200043CC85471747FF1F2302F7BEB7E70400D9
:10243000BC4B93050020E1BF9747FF1F938747BB25
:10244000D44B1147638DE600B7E7040083A7071D4F
:102450008297B7E70400BC4B930500044DBF0549C4
:102460001747FF1F232027BB83C7070032C62E84D0
:1024700093F7F70FD5D3B7E4040083A7041D7D14A9
:102480001374F40F8297E37689FCB245994703C62B
:102490001500E3F0C7FCFC4409061745FF1F1305B0
:1024A00025B78297BC48930500081745FF1F0345D1
:1024B000A5B4829779BF1703FFFFE70243C0174710
:1024C000FF1F1307E7B24047184B1C409746FF1FFA
:1024D00023A6F6B26316E4001747FF1F2322F7B2C4
:1024E000130584FE9790FFFFE78000AA035564FF61
:1024F0009780FFFFE780807297A0FFFFE78060D0A2
:102500001703FFFF6700E3BD1703FFFFE70223BBCD
:102510009747FF1F9387C7ADD84BDC4789C7970004
:102520000000E78080F985471747FF1F232CF7AC91
:102530009747FF1F9387479D9C43930500021745CC
:10254000FF1F034565AB83C787031747FF1F230D95
:10255000F7AAB7E70400BC4B82971703FFFF670099
:1025600043B89747FF1F23A7A7A882801703FFFF41
:10257000E70243B337E404007C4CA1451745FF1F35
:10258000034585A782977C48A1451745FF1F034552
:10259000A5A69744FF1F9384A4A58297DC4489EBEA
:1025A00097000000E78080D91703FFFF6700C3B2E0
:1025B00003D567FF9780FFFFE7804066AA896DD14A
:1025C000D84891476310F7027C4C91451745FF1F8F
:1025D000034585A282977C4891451745FF1F034517
:1025E000A5A1829703A9490103D409018947B7E945
:1025F00004001747FF1F2327F7A083A7091D210405
:102600004204829783C784011715FF1F1305C5EF86
:1026100061191717FF1FA309F7EE83A7491C418013
:1026200082979747FF1F2383079E83A7C91C814674
:1026300009469375F40F4A85829711E99747FF1F62
:1026400083C707AD89C79700FF1FE780A058B7E78A
:102650000400BC4F2146A1451745FF1F0345C599FE
:10266000829799B71703FFFFE70263A593F7052049
:1026700001112E8481CF97000000E78020E91345E7
:10268000042005611703FFFF6700A3A593F705105A
:10269000A9CF9744FF1F9384A495DC4897000000BE
:1026A000E78020C11747FF1F13070786184383C71A
:1026B0008401034787036318F700DC4489C7970048
:1026C0000000E78080DF85471747FF1F232CF79224
:1026D000B7E70400BC4B930500021745FF1F0345F5
:1026E000A59182971345041069BF93F70508BDC7EC
:1026F0009747FF1F83C7D791E91719469745FF1FD3
:10270000938525911305D10093F4F70F1749FF1F07
:102710000349099097C00000E78040409397040167
:10272000C1831747FF1F1307278F231DF100231CA9
:10273000F1009747FF1F9387A78B3ACE3ACAD84339
:102740002306010009CBDC439315890154080D468B
:10275000E185680082971345040825B793F72500A3
:10276000A5C39747FF1F9387A788D84B8947630660
:10277000F7029747FF1F83C7E78413F7270011EF7E
:10278000918B99CFB7E70400BC4F1306000A894527
:102790001745FF1F03454586829713452400D5B58D
:1027A0009737FF1F938747769C4383C78703174755
:1027B000FF1F230BF78497000000E78060DBF1BF69
:1027C00093F7050281CB97000000E78060DA13459C
:1027D000040245BD93F7850081CB97000000E78098
:1027E000E0D21345840071BD93F7150081CB9700AB
:1027F0000000E780A0B41345140061B593F74500CD
:1028000081CB97000000E78060B31345440095BD7D
:1028100093F7050495C39737FF1F83C7677D91CB57
:1028200097000000E780A0A491471737FF1F232BD4
:10283000F77C13450404B1B593F705010145E38224
:1028400007E49737FF1F9387A77AD84B9147631008
:10285000F7049737FF1F9387E7769C4313D727002A
:102860008583D98F858B91E7B7E7040083A7071D80
:102870008297B7E70400FC4F91451735FF1F0345CA
:10288000A577829785471737FF1F232DF7761345C6
:102890000401C5BB9747FF1F238CA78682801703BF
:1028A000FFFFE702C3819737FF1F23A907749737FC
:1028B000FF1F23A7077485471734FF1F1304C46441
:1028C0001737FF1F2320F7741C4083C78703173770
:1028D000FF1F230BF7729790FFFFE780409329C5F6
:1028E0009717FF1F23A6A7C21C401705000013055A
:1028F000A5D783C787031737FF1F2307F77017175D
:10290000FF1FA303F7C09737FF1FA383076EB7E727
:10291000040083A7070882979737FF1F238EA76CB1
:1029200017F3FEFF6700E37BB7C7898E938767EDD8
:102930001717FF1F232EF7BC45BF1737FF1F03478D
:10294000276B795555E79737FF1F9387676A03C74A
:10295000170005079736FF1FA38CE66803C717000B
:102960008D463377D7029736FF1FA383E66883C669
:1029700017001737FF1F13072759184393F6F60F51
:10298000A9EE834787031737FF1F230FF766854795
:102990001737FF1F230EF7649737FF1F9387876250
:1029A0009C430145998BA9E717F3FEFFE7022371CA
:1029B00037E404007C48C1451735FF1F0345C56354
:1029C00082973C4885451735FF1F0345E56282978E
:1029D000014517F3FEFF6700C37083C717008546E4
:1029E0006395F6008347970379BF8347A70361BFC9
:1029F00082809737FF1F83C7A75FA1CF17F3FEFF22
:102A0000E702E36B37E404009737FF1F2382075E7A
:102A10007C4885451735FF1F0345055E82977C4C32
:102A200091451735FF1F0345255D82977C489145E9
:102A30001735FF1F0345455C82973C48C145173554
:102A4000FF1F0345655B8297014517F3FEFF670093
:102A500043697955828017F3FEFFE70243662A84B3
:102A6000035565FF9780FFFFE780401B9737FF1FE7
:102A700093870758D847BE841DEF9790FFFFE780E4
:102A800080779C48232004009DEB9737FF1F23A9E4
:102A900087569737FF1F23A38756B7E70400BC4B21
:102AA00089451735FF1F034525558297014517F3C3
:102AB000FEFF67000363630A8700184375BF80C386
:102AC0009737FF1F23AE8752C9BF7955CDB717F38C
:102AD000FEFFE702C35E9737FF1F9387A763884314
:102AE0002326050023240500510597A00000E78058
:102AF000C03317F3FEFF6700C35E17F3FEFFE70264
:102B0000035C1734FF1F1304E4601C40411199CF8C
:102B10009C472302B5002AC61CC197000000E7802D
:102B200040FB1C409C4B99C332458297410117F3EF
:102B3000FEFF6700035B17F3FEFFE70243584111F6
:102B4000444D328532842EC69790FFFFE780C052F5
:102B50002AC422859790FFFFE780205403A84400F1
:102B6000630C0800B245835744001840224683D5C1
:102B70004500AA8626850298410117F3FEFF6700EB
:102B8000435617F3FEFFE7028353404D1DC808C0AC
:102B900097050000938565031305440197A0000085
:102BA000E78040169737FF1F9387C7569C43014520
:102BB00089E79737FF1F23AF875417F3FEFF67009E
:102BC00043527D55DDBF17F3FEFFE702434F01116E
:102BD00068009305F00F02C602C802CA02CC02CEFA
:102BE00097000000E780A0F1056117F3FEFF670082
:102BF000434F9737FF1F9387E7519C43D847A167FF
